:100000000C94697A0C94197C0C94297C0C94000053
:100010000C9400000C9400000C9400000C94000060
:100020000C9400000C9400000C9400000C94000050
:100030000C9400000C9400000C942E7C0C94000096
:100040000C9400000C9400000C9400000C94000030
:100050000C9400000C9400000C9400000C94000020
:100060000C9400000C9400000C9400000C94000010
:100070000C9400000C9400000C9400000C94000000
:100080000C9400000C9400000C94000079A95ADA3A
:10009000997DA95ADE6379C0B086BFB17F79A95A2C
:1000A000DA997DA95ADE6379C0B086BFB17F79A99C
:1000B0005ADA997DA95ADE6379C0B086BFB17F79DB
:1000C000A95ADA997DA95ADE6379C0B086BFB17F9B
:1000D00079A95ADA997DA95ADE6379C0B086BFB191
:1000E0007F79A95ADA997DA95ADE6379C0B086BFB3
:1000F000B17F79A95ADA997DA95ADE6379C0B086B1
:10010000BFB17F79A95ADA997DA95ADE6379C0B067
:1001100086BFB17F0300000003030000000302025A
:1001200002020202000300000003030000000302B9
:1001300002020202020003000000030300000003A9
:10014000020202020202000300000003030000009A
:100150000302020202020200020202020202020280
:10016000020202020202020203020202020202026E
:10017000020202020202020202030202020202025E
:10018000020202020202020202020302020202024E
:1001900002020202020202020202020379A95ADAF0
:1001A000997DA95ADE6379C0B086BFB17F79A95A1B
:1001B000DA997DA95ADE6379C0B086BFB17F79A98B
:1001C0005ADA997DA95ADE6379C0B086BFB17F79CA
:1001D000A95ADA997DA95ADE6379C0B086BFB17F8A
:1001E00079A95ADA997DA95ADE6379C0B086BFB180
:1001F0007F79AA5ADA997DAA5ADE6378C0B087BFA0
:10020000B17F79AA5ADA997DAA5ADE6377C0B0889D
:10021000BFB17F79AB5ADA997DAB5ADE6376C0B055
:1002200089BFB17F79AC5ADA997DAC5ADE6375C06B
:10023000B08ABFB17F79AC5ADA997DAC5ADE63746B
:10024000C0B08BBFB17F79AD5ADA997DAD5ADE630C
:1002500073C0B08CBFB17F79AE5ADA997DAE5ADEE9
:100260006372C0B08DBFB17F79AE5ADA997DAE5A54
:10027000DE6371C0B08EBFB17F79AF5ADA997DAFBE
:100280005ADE6370C0B08FBFB17F79AF5ADA997D03
:10029000AF5ADE636FC0B090BFB17F79B05ADA99C0
:1002A0007DB05ADE636EC0B091BFB17F79B15ADACA
:1002B000997DB15ADE636DC0B092BFB17F79B15AFA
:1002C000DA997DB15ADE636CC0B093BFB17F79B269
:1002D0005ADA997DB25ADE636BC0B094BFB17F79B0
:1002E000B35ADA997DB35ADE636AC0B095BFB17F65
:1002F00079B35ADA997DB35ADE636AC0B095BFB15B
:100300007F79B45ADA997DB45ADE6369C0B096BF7A
:10031000B17F79B45ADA997DB45ADE6368C0B09778
:10032000BFB17F79B55ADA997DB55ADE6367C0B03F
:1003300098BFB17F79B65ADA997DB65ADE6366C046
:10034000B099BFB17F79B65ADA997DB65ADE636546
:10035000C0B09ABFB17F79B75ADA997DB75ADE63D8
:1003600064C0B09BBFB17F79B85ADA997DB85ADEC4
:100370006363C0B09CBFB17F79B85ADA997DB85A2F
:10038000DE6362C0B09DBFB17F79B95ADA997DB999
:100390005ADE6361C0B09EBFB17F79B95ADA997DE8
:1003A000B95ADE6360C0B09FBFB17F79BA5ADA999B
:1003B0007DBA5ADE635FC0B0A0BFB17F79BB5ADAA5
:1003C000997DBB5ADE635EC0B0A1BFB17F79BB5AD5
:1003D000DA997DBB5ADE635DC0B0A2BFB17F79BC44
:1003E0005ADA997DBC5ADE635CC0B0A3BFB17F7995
:1003F000BD5ADA997DBD5ADE635BC0B0A4BFB17F40
:1004000079BD5ADA997DBD5ADE635BC0B0A4BFB135
:100410007F79BC5ADA997DBC5ADE635CC0B0A3BF59
:10042000B17F79BC5ADA997DBC5ADE635DC0B0A257
:10043000BFB17F79BB5ADA997DBB5ADE635EC0B02B
:10044000A1BFB17F79BA5ADA997DBA5ADE635FC02B
:10045000B0A0BFB17F79BA5ADA997DBA5ADE63602B
:10046000C0B09FBFB17F79B95ADA997DB95ADE63BE
:1004700061C0B09EBFB17F79B85ADA997DB85ADEB3
:100480006362C0B09DBFB17F79B85ADA997DB85A1E
:10049000DE6363C0B09CBFB17F79B75ADA997DB78C
:1004A0005ADE6364C0B09BBFB17F79B75ADA997DD9
:1004B000B75ADE6365C0B09ABFB17F79B65ADA9990
:1004C0007DB65ADE6366C0B099BFB17F79B55ADA9E
:1004D000997DB55ADE6367C0B098BFB17F79B55AD0
:1004E000DA997DB55ADE6368C0B097BFB17F79B441
:1004F0005ADA997DB45ADE6369C0B096BFB17F798C
:10050000B35ADA997DB35ADE636AC0B095BFB17F42
:1005100079B35ADA997DB35ADE636AC0B095BFB138
:100520007F79B25ADA997DB25ADE636BC0B094BF5C
:10053000B17F79B25ADA997DB25ADE636CC0B0935A
:10054000BFB17F79B15ADA997DB15ADE636DC0B01F
:1005500092BFB17F79B05ADA997DB05ADE636EC02E
:10056000B091BFB17F79B05ADA997DB05ADE636F2E
:10057000C0B090BFB17F79AF5ADA997DAF5ADE63D0
:1005800070C0B08FBFB17F79AE5ADA997DAE5ADEB6
:100590006371C0B08EBFB17F79AE5ADA997DAE5A21
:1005A000DE6372C0B08DBFB17F79AD5ADA997DAD8F
:1005B0005ADE6373C0B08CBFB17F79AD5ADA997DD2
:1005C000AD5ADE6374C0B08BBFB17F79AC5ADA9993
:1005D0007DAC5ADE6375C0B08ABFB17F79AB5ADAA1
:1005E000997DAB5ADE6376C0B089BFB17F79AB5AD3
:1005F000DA997DAB5ADE6377C0B088BFB17F79AA44
:100600005ADA997DAA5ADE6378C0B087BFB17F7984
:10061000A95ADA997DA95ADE6379C0B086BFB17F45
:1006200079A95ADA997DA95ADE6379C0B07BBFB146
:100630008379A95ADA997DA95ADE6379C0B065BF7A
:10064000B18B79A95ADA997DA95ADE6379C0B05A7B
:10065000BFB19079A95ADA997DA95ADE6379C0B001
:100660004EBFB19479A95ADA997DA95ADE6379C04F
:10067000B043BFB19879A95ADA997DA95ADE637956
:10068000C0B038BFB19D79A95ADA997DA95ADE6305
:1006900079C0B02DBFB19779A95ADA997DA95ADEF0
:1006A0006379C0B021BFB1A679A95ADA997DA95A58
:1006B000DE6379C0B021BFB1A679A95ADA997DA9C4
:1006C0005ADE6379C0B021BFB1A679A95ADA997D03
:1006D000A95ADE6379C0B021BFB1A679A95ADA99C7
:1006E0007DA95ADE6379C0B021BFB1A679A95ADAD3
:1006F000997DA95ADE6379C0B021BFB1A679A95A04
:10070000DA997DA95ADE6379C0B021BFB1A679A973
:100710005ADA997DA95ADE6379C0B021BFB1A679B2
:10072000A95ADA997DA95ADE6379C0B021BFB1A672
:1007300079A95ADA997DA95ADE6379C0B021C0B18E
:10074000A679A95ADA997DA95ADE6379C0B021C386
:10075000B1A679A95ADA997DA95ADE6379C0B02188
:10076000C5B1A679A95ADA997DA95ADE6379C0B0D4
:1007700021C7B1A679A95ADA997DA95ADE6379C051
:10078000B021C9B1A679A95ADA997DA95ADE63794F
:10079000C0B021CBB1A679A95ADA997DA95ADE63F6
:1007A00079C0B021CDB1A679A95ADA997DA95ADECE
:1007B0006379C0B021CFB1A679A95ADA997DA95A37
:1007C000DE6379C0B021CCB1A679A95ADA997DA9A6
:1007D0005ADE6379C0B021C5B1A679A95ADA997DEC
:1007E000A95ADE6379C0B021C1B1A679A95ADA99B4
:1007F0007DA95ADE6379C0B021BDB1A679A95ADAC4
:10080000997DA95ADE6379C0B021BAB1A679A95AF7
:10081000DA997DA95ADE6379C0B021B6B1A679A96B
:100820005ADA997DA95ADE6379C0B021B2B1A679AE
:10083000A95ADA997DA95ADE6379C0B021AEB1A672
:1008400079A95ADA997DA95ADE6379C0B021B1B18C
:10085000A679A95ADA997DA95ADE6379C0B021B880
:10086000B1A679A95ADA997DA95ADE6379C0B02177
:10087000BCB1A679A95ADA997DA95ADE6379C0B0CC
:1008800021C0B1A679A95ADA997DA95ADE6379C047
:10089000B021C3B1A679A95ADA997DA95ADE637944
:1008A000C0B021C7B1A679A95ADA997DA95ADE63E9
:1008B00079C0B021CBB1A679A95ADA997DA95ADEBF
:1008C0006379C0B021CFB1A679A95ADA997DA95A26
:1008D000DE6379C0B021CEB1A679A95ADA997DA993
:1008E0005ADE6379C0B021CBB1A679A95ADA997DD5
:1008F000A95ADE6379C0B021C9B1A679A95ADA999B
:100900007DA95ADE6379C0B021C7B1A679A95ADAA8
:10091000997DA95ADE6379C0B021C5B1A679A95ADB
:10092000DA997DA95ADE6379C0B021C3B1A679A94D
:100930005ADA997DA95ADE6379C0B021C1B1A6798E
:10094000A95ADA997DA95ADE6379C0B021BFB1A650
:1009500079A95ADA997DA95ADE6384C0B02CBFB157
:100960009E79A95ADA997DA95ADE639AC0B042BF2E
:10097000B18D79A95ADA997DA95ADE63A5C0B04D27
:10098000BFB18479A95ADA997DA95ADE63B1C0B0A2
:1009900059BFB17B79A95ADA997DA95ADE63BCC0E7
:1009A000B064BFB17379A95ADA997DA95ADE63C7D9
:1009B000C0B06FBFB16A79A95ADA997DA95ADE63CE
:1009C000D2C0B07ABFB16179A95ADA997DA95ADE4D
:1009D00063DEC0B086BFB15879A95ADA997DA95AA9
:1009E000DE63DEC0B086BFB15879A95ADA997DA915
:1009F0005ADE63DEC0B086BFB15879A95ADA997D54
:100A0000A95ADE63DEC0B086BFB15879A95ADA9917
:100A10007DA95ADE63DEC0B086BFB15879A95ADA23
:100A2000997DA95ADE63DEC0B086BFB15879A95A54
:100A3000DA997DA95ADE63DEC0B086BFB15879A9C4
:100A40005ADA997DA95ADE63DEC0B086BFB1587903
:100A5000A95ADA997DA95ADE63DEC0B086BFB158C3
:100A600079A95ADA997DA95ADE63DEC1B086BFB191
:100A70005879A95ADA997DA95ADE63DEC4B086BFD7
:100A8000B15879A95ADA997DA95ADE63DEC6B086D3
:100A9000BFB15879A95ADA997DA95ADE63DEC8B088
:100AA00086BFB15879A95ADA997DA95ADE63DECAA0
:100AB000B086BFB15879A95ADA997DA95ADE63DEAA
:100AC000CCB086BFB15879A95ADA997DA95ADE63AC
:100AD000DECEB086BFB15879A95ADA997DA95ADE1F
:100AE00063DED0B086BFB15879A95ADA997DA95A88
:100AF000DE63DECDB086BFB15879A95ADA997DA9F7
:100B00005ADE63DEC6B086BFB15879A95ADA997D3C
:100B1000A95ADE63DEC2B086BFB15879A95ADA9904
:100B20007DA95ADE63DEBEB086BFB15879A95ADA14
:100B3000997DA95ADE63DEBBB086BFB15879A95A48
:100B4000DA997DA95ADE63DEB7B086BFB15879A9BC
:100B50005ADA997DA95ADE63DEB3B086BFB15879FF
:100B6000A95ADA997DA95ADE63DEAFB086BFB158C3
:100B700079A95ADA997DA95ADE63DEB2B086BFB18F
:100B80005879A95ADA997DA95ADE63DEB9B086BFD1
:100B9000B15879A95ADA997DA95ADE63DEBDB086CB
:100BA000BFB15879A95ADA997DA95ADE63DEC1B07E
:100BB00086BFB15879A95ADA997DA95ADE63DEC495
:100BC000B086BFB15879A95ADA997DA95ADE63DE99
:100BD000C8B086BFB15879A95ADA997DA95ADE639F
:100BE000DECCB086BFB15879A95ADA997DA95ADE10
:100BF00063DED0B086BFB15879A95ADA997DA95A77
:100C0000DE63DECFB086BFB15879A95ADA997DA9E3
:100C10005ADE63DECCB086BFB15879A95ADA997D25
:100C2000A95ADE63DECAB086BFB15879A95ADA99EB
:100C30007DA95ADE63DEC8B086BFB15879A95ADAF9
:100C4000997DA95ADE63DEC6B086BFB15879A95A2C
:100C5000DA997DA95ADE63DEC4B086BFB15879A99E
:100C60005ADA997DA95ADE63DEC2B086BFB15879DF
:100C7000A95ADA997DA95ADE63DEC0B086BFB158A1
:100C800079A95ADA997DA95ADE63D3C0B086BFB17B
:100C90005C79A95ADA997DA95ADE63BDC0B086BFD6
:100CA000B16479A95ADA997DA95ADE63B2C0B086D7
:100CB000BFB16979A95ADA997DA95ADE63A6C0B095
:100CC00086BFB16D79A95ADA997DA95ADE639BC0B6
:100CD000B086BFB17179A95ADA997DA95ADE6390BD
:100CE000C0B086BFB17679A95ADA997DA95ADE6378
:100CF00085C0B086BFB17A79A95ADA997DA95ADE42
:100D00006379C0B086BFB17F79A95ADA997DA95AB3
:100D1000DE6379C0B086BFB17F79A95ADA997DA91F
:100D20005ADE6379C0B086BFB17F79A95ADA997D5E
:100D3000A95ADE6379C0B086BFB17F79A95ADA9922
:100D40007DA95ADE6379C0B086BFB17F0300000081
:100D50000303000000030303030303030403000071
:100D60000003030000000303030303030304030061
:100D70000000030300000003030303030303040351
:100D80000000000303000000030303030303030444
:100D9000030400000303040000030203030203032F
:100DA000040304000003030400000302030302031E
:100DB000030403040000030304000003020303020E
:100DC00003030403040000030304000003020303FD
:100DD00002030304030400000303040000030203EE
:100DE00003020303040304000003030400000302DE
:100DF00003030203030403040000030304000003CD
:100E000002030302030304030400000303040000BD
:100E100003020303020303040304000003030400AA
:100E2000000302030302030304030400000303049A
:100E3000000003020303020303040304000003038E
:100E4000040000030203030203030403040000037D
:100E5000030400000302030302030304030400006D
:100E6000030304000003020303020303040304005A
:100E7000000303040000030203030203030403044A
:100E8000000003030400000302030302030304033E
:100E9000040000030304000003020303020303042D
:100EA000030400000303040000030203030203031E
:100EB000040304000003030400000302030302030D
:100EC00003040304000003030400000302030302FD
:100ED00003030403040000030304000003020303EC
:100EE00002030304030400000303040000030203DD
:100EF00003020303040304000003030400000302CD
:100F000003030203030403040000030304000003BB
:100F100002030302030304030400000303040000AC
:100F20000302030302030304030400000303040099
:100F30000003020303020303040304000003030489
:100F4000000003020303020303040304000003037D
:100F5000040000030203030203030403040000036C
:100F6000030400000302030302030304030400005C
:100F70000303040000030203030203030403040049
:100F80000003030400000302030302030304030439
:100F9000000003030400000302030302030304032D
:100FA000040000030304000003020303020303041C
:100FB000030300000303030000030203030203030F
:100FC00004030300000303030000030203030203FE
:100FD00003040303000003030300000302030302EE
:100FE00003030403030000030303000003020303DD
:100FF00002030304030300000303030000030203CE
:1010000003020303040303000003030300000302BD
:1010100003030203030403030000030303000003AC
:10102000020303020303040303000003030300009D
:10103000030203030203030403030000030303008A
:10104000000302030302030304030300000303037A
:10105000000003020303020303040303000003036D
:10106000030000030203030203030403030000035D
:10107000030300000302030302030304030300004D
:10108000030303000003020303020303040303003A
:10109000000303030000030203030203030403032A
:1010A000000003030300000302030302030304031D
:1010B000030000030303000003020303020303040D
:1010C00003030000030303000003020303020303FE
:1010D00004030300000303030000030203030203ED
:1010E00003040303000003030300000302030302DD
:1010F00003030403030000030303000003020303CC
:1011000002030304030300000303030000030203BC
:1011100003020303040303000003030300000302AC
:10112000030302030304030300000303030000039B
:10113000020303020303040303000003030300008C
:101140000302030302030304030300000303030079
:101150000003020303020303040303000003030369
:10116000000003020303020303040303000003035C
:10117000030000030203030203030403030000034C
:10118000030300000302030302030304030300003C
:101190000303030000030203030203030403030029
:1011A0000003030300000302030302030304030319
:1011B000000003030300000302030302030304030C
:1011C00003000003030300000302030302030304FC
:1011D00003030000030303000003020303030303EC
:1011E00003030300000303030000030203030303DC
:1011F00003030303000003030300000302030303CC
:1012000003030303030000030303000003020303BB
:1012100003030303030300000303030000030203AB
:10122000030303030303030000030303000003029B
:10123000030303030303030300000303030000038A
:10124000020303030303030303000003030300007B
:101250000302030303030303030300000303030068
:101260000003020303030303030303000003030358
:10127000000003020303030303030303000003034B
:10128000030000030203030303030303030000033B
:10129000030300000302030303030303030300002B
:1012A0000303030000030203030303030303030018
:1012B0000003030300000302030303030303030308
:1012C00000000303030000030203030303030303FB
:1012D00003000003030300000302030303030303EB
:1012E00003030000030303000003020303030303DB
:1012F00003030300000303030000030203030303CB
:1013000003030303000003030300000302030303BA
:1013100003030303030000030303000003020303AA
:10132000030303030303000003030300000302039A
:10133000030303030303030000030303000003028A
:101340000303030303030303000003030300000379
:10135000020303030303030303000003030300006A
:101360000302030303030303030300000303030057
:101370000003020303030303030303000003030347
:10138000000003020303030303030303000003033A
:10139000030000030203030303030303030000032A
:1013A000030300000302030303030303030300001A
:1013B0000303030000030203030303030303030007
:1013C00000030303000003020303030303030303F7
:1013D00000000303030000030203030303030303EA
:1013E00003000003030300000302030303030303DA
:1013F00003030000030303000003020303030303CA
:1014000003030300000303030000030203030303B9
:1014100003030303000003030300000302030303A9
:101420000303030303000003030300000302030399
:101430000303030303030000030303000003020389
:101440000303030303030300000303030000030279
:101450000303030303030303000003030300000368
:101460000203030303030303030000030303000059
:101470000302030303030303030300000303030046
:101480000003020303030303030303000003030336
:101490000000030203030303030303030000030329
:1014A0000300000302030303030303030300000319
:1014B0000303000003020303030303030303000009
:1014C00003030300000302030303030303030300F6
:1014D00000030303000003020303030303030303E6
:1014E00000000303030000030203030303030303D9
:1014F00003000003030300000302030303030303C9
:1015000003030000030303000003030303030303B7
:1015100003030300000303030000030303030303A7
:101520000303030300000303030000030303030397
:101530000303030303000003030300000303030387
:101540000303030303030000030303000003030377
:101550000303030303030300000303030000030367
:101560000303030303030303000003030300000357
:101570000303030303030303030000030303000047
:101580000303030303030303030300000303030034
:101590000003030303030303030303000003030324
:1015A0000000030303030303030303030000030317
:1015B0000300000303030303030303030300000307
:1015C00003030000030303030303030303030000F7
:1015D00003030300000303030303030303030300E4
:1015E00000030303000003030303030303030303D4
:1015F00000000303030000030303030303030303C7
:1016000003000003030300000303030303030303B6
:1016100003030000030303000003030303030303A6
:101620000303030000030303000003030303030396
:101630000303030300000303030000030303030386
:101640000303030303000003030300000303030376
:101650000303030303030000030303000003030366
:101660000303030303030300000303030000030356
:101670000303030303030303000003030300000346
:101680000303030303030303030000030303000036
:101690000303030303030303030300000303030023
:1016A0000003030303030303030303000003030313
:1016B0000000030303030303030303030000030306
:1016C00003000003030303030303030303000003F6
:1016D00003030000030303030303030303030000E6
:1016E00003030300000303030303030303030300D3
:1016F00000030303000003030303030303030303C3
:1017000000000303030000030303030303030303B5
:1017100003000003030300000303030303030303A5
:101720000303000003030300000303030303030395
:101730000303030000030303000003030303030385
:101740000303030300000303030000030303030375
:101750000303030303000003030300000303030365
:101760000303030303030000030303000003030355
:101770000303030303030300000303030000030345
:101780000303030303030303000003030300000335
:101790000303030303030303030000030303000025
:1017A0000303030303030303030300000303030012
:1017B0000003030303030303030303000003030302
:1017C00000000303030303030303030300000303F5
:1017D00003000003030303030303030303000003E5
:1017E00003030000030303030303030303030000D5
:1017F00003030300000303030303030303030300C2
:1018000000030303000003030303030303030303B1
:1018100000000303030000030303030303030303A4
:101820000300000303030000030303030303030394
:101830000303000003030300000303030303030384
:101840000103030000030303000003030303030376
:101850000301030300000303030000030303030366
:101860000303010303000003030300000303030356
:101870000303030103030000030303000003030346
:101880000303030301030300000303030000030336
:101890000303030303010303000003030300000326
:1018A0000303030303030103030000030303000016
:1018B00003030303030303010302020203030202FF
:1018C00002030303030303030303020202030302ED
:1018D00002020303030303030303030202020303DD
:1018E00002020203030303030303030302020203CE
:1018F00003020202030303030303030379AA5DD86F
:10190000997DAA5DDC6379C0B086BFB17F79AA5F9B
:10191000D7997DAA5FDB6379C0B086BFB17F79AA12
:1019200062D5997DAA62D96379C0B086BFB17F794B
:10193000AB64D4997DAB64D86379C0B086BFB17F06
:1019400079AB66D3997DAB66D76379C0B086BFB1FA
:101950007F79AC68D2997DAC68D66379C0B086BF18
:10196000B17F79AC6AD0997DAC6AD46379C0B08616
:10197000BFB17F79AC6CCF997DAC6CD36379C0B0CB
:1019800086BFB17F79AD6ECE997DAD6ED26379C0E1
:10199000B086BFB17F79AD6FCD997DAD6FD16379E1
:1019A000C0B086BFB17F7AAD6FCD9A7EAD6FD16486
:1019B0007AC0B087BFB17F7BAD6FCD9B80AD6FD15B
:1019C000667AC0B087BFB17F7CAD6FCD9C82AD6FB2
:1019D000D1687BC0B088BFB17F7DAD6FCD9D83AD39
:1019E0006FD16A7BC0B088BFB17F7FAD6FCD9F855F
:1019F000AD6FD16C7BC0B088BFB17F80AD6FCDA023
:101A000087AD6FD16E7CC0B089BFB17F81AD6FCD26
:101A1000A188AD6FD1707CC0B089BFB17F82AD6F3E
:101A2000CDA28AAD6FD1727DC0B08ABFB17F84ADC7
:101A30006FCDA48CAD6FD1747DC0B08ABFB17F85EE
:101A4000AD6FCDA58DAD6FD1757DC0B08ABFB17FB3
:101A500086AD6FCDA68FAD6FD1777EC0B08BBFB195
:101A60007F87AD6FCDA791AD6FD1797EC0B08BBFB1
:101A7000B17F88AD6FCDA892AD6FD17B7FC0B08CA8
:101A8000BFB17F8AAD6FCDAA94AD6FD17D7FC0B05D
:101A90008CBFB17F8BAD6FCDAB96AD6FD17F7FC06B
:101AA000B08CBFB17F8CAD6FCDAC97AD6FD1818065
:101AB000C0B08DBFB17F8DAD6FCDAD99AD6FD1830E
:101AC00080C0B08DBFB17F8FAD6FCDAF9BAD6FD1FB
:101AD0008581C0B08EBFB17F90AD6FCDB09CAD6F32
:101AE000D18681C0B08EBFB17F91AD6FCDB19EADBB
:101AF0006FD18881C0B08EBFB17F91AD6FCDB19EE7
:101B0000B17BCC8881C0B08EBFB17F91AD6FCDB1BC
:101B10009EB586C98881C0B08EBFB17F91AD6FCDB3
:101B2000B19EB88FC68881C0B08EBFB17F91AD6FB6
:101B3000CDB19EBB97C48881C0B08EBFB17F91AD3F
:101B40006FCDB19EBE9EC28881C0B08EBFB17F9165
:101B5000AD6FCDB19EBD95C98881C0B08EBFB17F3C
:101B600091AD6FCDB19EBC8CD08881C0B08EBFB11D
:101B70007F91AD6FCDB19EBA81D88881C0B08EBF44
:101B8000B17F91AD6FCDB19EB874E08881C0B08E49
:101B9000BFB17F91AD6FCDB19EB564EA8881C0B011
:101BA0008EBFB17F000000000000000000000303B2
:101BB0000303030303000000000000000000000313
:101BC0000303030303030000000000000000000003
:101BD00003030303030303000000000000000000F0
:101BE00000030303030303030000000000000000E0
:101BF00000000303030303030300000000000000D0
:101C000000000003030303030303000000000000BF
:101C100000000000030303030303030000000000AF
:101C2000000000000003030303030303000000009F
:101C3000000000000000030303030303030000008F
:101C4000000000000000000303030303030300007F
:101C50000000000000000000040404040404030069
:101C60000000000000000000000404040404040359
:101C7000000000000000000000000404040404044C
:101C8000030000000000000000000004040404043D
:101C9000040300000000000000000000040404042D
:101CA000040403000000000000000000000404041D
:101CB000040404030000000000000000000004040D
:101CC00004040404030000000000000000000004FD
:101CD00004040404040300000000000000000000ED
:101CE00004040404040403000000000000000000D9
:101CF00000040404040404030000000000000000C9
:101D000000000404040404040300000000000000B8
:101D100000000004040404040403000000000000A8
:101D20000000000004040404040403000000000098
:101D30000000000000040404040404030000000088
:101D40000000000000000404040404040300000078
:101D50000000000000000004040404040403000068
:101D60000000000000000000040404040404030058
:101D70000000000000000000000404040404040348
:101D8000000000000000000000000404040404043B
:101D9000030000000000000000000004040404042C
:101DA000040300000000000000000000040404041C
:101DB000040403000000000000000000000404040C
:101DC00004040403000000000000000000000404FC
:101DD00004040404030000000000000000000004EC
:101DE00004040404040300000000000000000000DC
:101DF00004040404040403000000000000000000C8
:101E000000040404040404030000000000000000B7
:101E100000000404040404040300000000000000A7
:101E20000000000404040404040300000000000097
:101E30000000000004040404040403000000000087
:101E40000000000000040404040404038EAD6FCC01
:101E5000AE9BB565E98581C0B08EBFB17F8BAC6F9D
:101E6000CBAB98B467E78280C0B08DBFB17F88AB41
:101E70006FCAA895B468E67F7FC0B08CBFB17F857C
:101E8000AB6EC9A593B469E47B7EC0B08BBFB17F54
:101E900082AA6EC9A290B46AE3787DC0B08ABFB14D
:101EA0007F80AA6EC8A08DB36AE1757DC0B08ABF7D
:101EB000B17F7DA96DC79D8AB36BE0717CC0B0898D
:101EC000BFB17F7AA86DC79A87B36CDE6E7BC0B056
:101ED00088BFB17F77A86CC69784B26DDD6B7AC07E
:101EE000B087BFB17F74A76BC59381B26DDC687991
:101EF000C0B086BFB17F71A66AC5907EB16EDB644B
:101F000079C0B086BFB17F6EA669C48D7BB16ED932
:101F10006178C0B085BFB17F6BA568C48A78B16FA6
:101F2000D85E77C0B084BFB17F68A467C38675B040
:101F30006FD75B76C0B083BFB17F65A366C3837381
:101F4000B06FD65975C0B082BFB17F62A365C38040
:101F500070AF6FD55675C0B082BFB17F60A264C349
:101F60007C6DAF6FD45374C0B081BFB17F5DA1628F
:101F7000C2796AAE6FD35073C0B080BFB17F5AA030
:101F800061C27667AE6FD24D72C0B07FBFB17F576E
:101F90009F5FC27364AD6FD14A71C0B07EBFB17F25
:101FA00057A677B97364AD6FD14A71C0B07EBFB127
:101FB0007F57AC88B37364AD6FD14A71C0B07EBF38
:101FC000B17F57B196AF7364AD6FD14A71C0B07E27
:101FD000BFB17F57B6A2AC7364AD6FD14A71C0B0C8
:101FE0007EBFB17F57BBACAB7364AD6FD14A71C0DC
:101FF000B07EBFB17F57BBA2B57364AD6FD14A71DC
:10200000C0B07EBFB17F57BB97C07364AD6FD14A7C
:1020100071C0B07EBFB17F57BA8ACB7364AD6FD148
:102020004A71C0B07EBFB17F57B87AD77364AD6FC5
:10203000D14A71C0B07EBFB17F57B564E67364AD5D
:102040006FD14A71C0B07EBFB17F5AB565E5766782
:10205000AD6FD04D72C0B07FBFB17F5DB467E37923
:102060006AAC6FCF5073C0B080BFB17F60B468E21C
:102070007C6DAB6FCE5374C0B081BFB17F62B46969
:10208000E08070AB6ECD5675C0B082BFB17F65B4D5
:102090006ADF8373AA6ECD5975C0B082BFB17F6805
:1020A000B36ADD8675AA6ECC5B76C0B083BFB17FA4
:1020B0006BB36BDC8A78A96DCB5E77C0B084BFB19F
:1020C0007F6EB36CDA8D7BA86DCB6178C0B085BFB5
:1020D000B17F71B26DD9907EA86CCA6479C0B086A8
:1020E000BFB17F74B26DD89381A76BC96879C0B056
:1020F00086BFB17F77B16ED79784A66AC96B7AC065
:10210000B087BFB17F7AB16ED59A87A669C86E7B5A
:10211000C0B088BFB17F7DB16FD49D8AA568C871FA
:102120007CC0B089BFB17F80B06FD3A08DA467C7DA
:10213000757DC0B08ABFB17F82B06FD2A290A36616
:10214000C7787DC0B08ABFB17F85AF6FD1A593A39B
:1021500065C77B7EC0B08BBFB17F88AF6FD0A895BD
:10216000A264C77F7FC0B08CBFB17F8BAE6FCFAB97
:1021700098A162C68280C0B08DBFB17F8EAE6FCE97
:10218000AE9BA061C68581C0B08EBFB17F91AD6F9F
:10219000CDB19E9F5FC68881C0B08EBFB17F91AD2B
:1021A0006FCDB19EA677BD8881C0B08EBFB17F9143
:1021B000AD6FCDB19EAC88B78881C0B08EBFB17F06
:1021C00091AD6FCDB19EB196B38881C0B08EBFB1D5
:1021D0007F91AD6FCDB19EB6A2B08881C0B08EBFE9
:1021E000B17F91AD6FCDB19EBBACAF8881C0B08ED9
:1021F000BFB17F91AD6FCDB19EBBA2B98881C0B098
:102200008EBFB17F91AD6FCDB19EBB97C48881C0A9
:10221000B08EBFB17F91AD6FCDB19EBA8ACF8881AC
:10222000C0B08EBFB17F91AD6FCDB19EB87ADB8863
:1022300081C0B08EBFB17F91AD6FCDB19EB564EA64
:102240008881C0B08EBFB17F000000000000000098
:102250000000040404040404030000000000000063
:102260000000000404040404040300000000000053
:102270000000000004040404040403000000000043
:102280000000000000040404040404030000000033
:102290000000000000000404040404040300000023
:1022A0000000000000000004040404040403000013
:1022B0000000000000000000040404040404030003
:1022C00000000000000000000004040404040403F3
:1022D00000000000000000000000040404040404E6
:1022E00003000000000000000000000404040404D7
:1022F00004030000000000000000000004040404C7
:1023000004040300000000000000000000040404B6
:1023100004040403000000000000000000000404A6
:102320000404040403000000000000000000000496
:102330000404040404030000000000000000000086
:102340000404040404040300000000000000000072
:102350000004040404040403000000000000000062
:102360000000040404040404030000000000000052
:102370000000000404040404040300000000000042
:102380000000000004040404040403000000000032
:102390000000000000040404040404030000000022
:1023A0000000000000000404040404040300000012
:1023B0000000000000000004040404040403000002
:1023C00000000000000000000404040404040300F2
:1023D00000000000000000000004040404040403E2
:1023E00000000000000000000000040404040404D5
:1023F00003000000000000000000000404040404C6
:1024000004030000000000000000000004040404B5
:1024100004040300000000000000000000040404A5
:102420000404040300000000000000000000040495
:102430000404040403000000000000000000000485
:102440000404040404030000000000000000000075
:102450000404040404040300000000000000000061
:102460000004040404040403000000000000000051
:102470000000040404040404030000000000000041
:102480000000000404040404040300000000000031
:102490000000000004040404040403000000000021
:1024A0000000000000040404040404030000000011
:1024B0000000000000000404040404040300000001
:1024C00000000000000000040404040404030000F1
:1024D00000000000000000000404040404040300E1
:1024E00000000000000000000004040404040403D1
:1024F00000000000000000000000040404040404C4
:1025000003000000000000000000000404040404B4
:1025100004030000000000000000000004040404A4
:102520000404030000000000000000000004040494
:102530000404040300000000000000000000040484
:102540000404040403000000000000000000000474
:102550000404040404030000000000000000000064
:102560000404040404040300000000000000000050
:102570000004040404040403000000000000000040
:102580000000040404040404030000000000000030
:102590000000000404040404040300000000000020
:1025A0000000000004040404040403000000000010
:1025B0000000000000040404040404030000000000
:1025C00000000000000004040404040403000000F0
:1025D00000000000000000040404040404030000E0
:1025E00000000000000000000404040404040300D0
:1025F00000000000000000000004040404040403C0
:1026000000000000000000000000040404040404B2
:1026100003000000000000000000000404040404A3
:102620000403000000000000000000000404040493
:102630000404030000000000000000000004040483
:10264000040404038EAD6FCCAE9BB565E98581C0F3
:10265000B08EBFB17F8BAC6FCBAB98B467E7828095
:10266000C0B08DBFB17F88AB6FCAA895B468E67F54
:102670007FC0B08CBFB17F85AB6EC9A593B469E450
:102680007B7EC0B08BBFB17F82AA6EC9A290B46AB4
:10269000E3787DC0B08ABFB17F80AA6EC8A08DB339
:1026A0006AE1757DC0B08ABFB17F7DA96DC79D8A83
:1026B000B36BE0717CC0B089BFB17F7AA86DC79A57
:1026C00087B36CDE6E7BC0B088BFB17F77A86CC665
:1026D0009784B26DDD6B7AC0B087BFB17F74A76B92
:1026E000C59381B26DDC6879C0B086BFB17F71A639
:1026F0006AC5907EB16EDB6479C0B086BFB17F6E73
:10270000A669C48D7BB16ED96178C0B085BFB17F39
:102710006BA568C48A78B16FD85E77C0B084BFB14A
:102720007F68A467C38675B06FD75B76C0B083BF80
:10273000B17F65A366C38373B06FD65975C0B0828D
:10274000BFB17F62A365C38070AF6FD55675C0B04F
:1027500082BFB17F60A264C37C6DAF6FD45374C07D
:10276000B081BFB17F5DA162C2796AAE6FD3507391
:10277000C0B080BFB17F5AA061C27667AE6FD24D44
:1027800072C0B07FBFB17F579F5FC27364AD6FD11E
:102790004A71C0B07EBFB17F57A471BA7364AD6F88
:1027A000D14A71C0B07EBFB17F57A87EB47364AD0B
:1027B0006FD14A71C0B07EBFB17F57AC8AAF73642E
:1027C000AD6FD14A71C0B07EBFB17F57AF94AB73CC
:1027D00064AD6FD14A71C0B07EBFB17F57B29DA8C2
:1027E0007364AD6FD14A71C0B07EBFB17F57B196EF
:1027F000AF7364AD6FD14A71C0B07EBFB17F57B1C6
:102800008EB57364AD6FD14A71C0B07EBFB17F57D2
:10281000B085BD7364AD6FD14A71C0B07EBFB17F6A
:1028200057AF7BC47364AD6FD14A71C0B07EBFB186
:102830007F57AD6FCD7364AD6FD14A71C0B07EBFAD
:10284000B17F59AD6FCD7565AD6FD14B72C0B07FA3
:10285000BFB17F5AAD6FCD7666AD6FD14C72C0B04F
:102860007FBFB17F5CAD6FCD7868AD6FD14E73C067
:10287000B080BFB17F5EAD6FCD7A69AD6FD14F7360
:10288000C0B080BFB17F5FAD6FCD7C6AAD6FD150FE
:1028900073C0B080BFB17F61AD6FCD7E6BAD6FD1C6
:1028A0005174C0B081BFB17F63AD6FCD806DAD6F2E
:1028B000D15374C0B081BFB17F64AD6FCD826EADB6
:1028C0006FD15475C0B082BFB17F66AD6FCD846FDC
:1028D000AD6FD15575C0B082BFB17F68AD6FCD8689
:1028E00070AD6FD15675C0B082BFB17F69AD6FCD8D
:1028F0008771AD6FD15776C0B083BFB17F6BAD6FBD
:10290000CD8973AD6FD15976C0B083BFB17F6DAD46
:102910006FCD8B74AD6FD15A77C0B084BFB17F6E6D
:10292000AD6FCD8D75AD6FD15B77C0B084BFB17F1A
:1029300070AD6FCD8F76AD6FD15C77C0B084BFB115
:102940007F72AD6FCD9178AD6FD15E78C0B085BF2D
:10295000B17F73AD6FCD9379AD6FD15F78C0B08526
:10296000BFB17F75AD6FCD957AAD6FD16079C0B0D5
:1029700086BFB17F77AD6FCD977BAD6FD16179C0E9
:10298000B086BFB17F79AD6FCD997DAD6FD16379E1
:10299000C0B086BFB17F79AD6ECE997DAD6ED2638A
:1029A00079C0B086BFB17F79AC6CCF997DAC6CD368
:1029B0006379C0B086BFB17F79AC6AD0997DAC6ACB
:1029C000D46379C0B086BFB17F79AC68D2997DAC51
:1029D00068D66379C0B086BFB17F79AB66D3997D85
:1029E000AB66D76379C0B086BFB17F79AB64D49949
:1029F0007DAB64D86379C0B086BFB17F79AA62D558
:102A0000997DAA62D96379C0B086BFB17F79AA5F88
:102A1000D7997DAA5FDB6379C0B086BFB17F79AA01
:102A20005DD8997DAA5DDC6379C0B086BFB17F793E
:102A3000A95ADA997DA95ADE6379C0B086BFB17F01
:102A4000000000000000000000000404040404046E
:102A5000030000000000000000000004040404045F
:102A6000040300000000000000000000040404044F
:102A7000040403000000000000000000000404043F
:102A8000040404030000000000000000000004042F
:102A9000040404040300000000000000000000041F
:102AA000040404040403000000000000000000000F
:102AB00004040404040403000000000000000000FB
:102AC00000040404040404030000000000000000EB
:102AD00000000404040404040300000000000000DB
:102AE00000000004040404040403000000000000CB
:102AF00000000000040404040404030000000000BB
:102B000000000000000404040404040300000000AA
:102B1000000000000000040404040404030000009A
:102B2000000000000000000404040404040300008A
:102B3000000000000000000004040404040403007A
:102B4000000000000000000000040404040404036A
:102B5000000000000000000000000404040404045D
:102B6000030000000000000000000004040404044E
:102B7000040300000000000000000000040404043E
:102B8000040403000000000000000000000404042E
:102B9000040404030000000000000000000004041E
:102BA000040404040300000000000000000000040E
:102BB00004040404040300000000000000000000FE
:102BC00004040404040403000000000000000000EA
:102BD00000040404040404030000000000000000DA
:102BE00000000404040404040300000000000000CA
:102BF00000000004040404040403000000000000BA
:102C000000000000040404040404030000000000A9
:102C10000000000000040404040404030000000099
:102C20000000000000000404040404040300000089
:102C30000000000000000004040404040403000079
:102C40000000000000000000040404040404030069
:102C50000000000000000000000404040404040359
:102C6000000000000000000000000404040404044C
:102C7000030000000000000000000004040404043D
:102C8000040300000000000000000000040404042D
:102C9000040403000000000000000000000404041D
:102CA000040404030000000000000000000004040D
:102CB00004040404030000000000000000000004FD
:102CC00004040404040300000000000000000000ED
:102CD00004040404040403000000000000000000D9
:102CE00000040404040404030000000000000000C9
:102CF00000000404040404040300000000000000B9
:102D000000000004040404040403000000000000A8
:102D10000000000004040404040403000000000098
:102D20000000000000040404040404030000000088
:102D30000000000000000404040404040300000078
:102D40000000000000000004040404040403000068
:102D50000000000000000000040404040404030058
:102D60000000000000000000000404040404040348
:102D7000000000000000000000000404040404043B
:102D8000030000000000000000000004040404042C
:102D9000040302020202020202020202030303030C
:102DA00003030302020202020202020202030303FD
:102DB00003030303020202020202020202020303ED
:102DC00003030303030202020202020202020203DD
:102DD00003030303030302020202020202020202CD
:102DE00003030303030303020202020202020202BC
:102DF00002030303030303030202020202020202AC
:102E0000020203030303030303020202020202029B
:102E1000020202030303030303030202020202028B
:102E2000020202020303030303030302020202027B
:102E300002020202020303030303030379A95ADA1D
:102E4000997DA95ADE6379C0B086BFB17F79A95A4E
:102E5000DA997DA95ADE6379C0B086BFB17F79A9BE
:102E60005ADA997DA95ADE6379C0B086BFB17F79FD
:102E7000A95ADA997DA95ADE6379C0B086BFB17FBD
:102E800079A95ADA997DA95ADE6379C0B086BFB1B3
:102E90007F79A95ADA997DA95ADE6379C0B086BFD5
:102EA000B17F79A95ADA997DA95ADE6379C0B086D3
:102EB000BFB17F79A95ADA997DA95ADE6379C0B08A
:102EC00086BFB17F79A95ADA997DA95ADE6379C0A4
:102ED000B086BFB17F79A95ADA997DA95ADE6379A4
:102EE000C0B086BFB17F76A95ADA967BA95ADE6157
:102EF00079C0B086BFB17F74A95ADA9479A95ADE35
:102F00005F79C0B086BFB17F71A95ADA9177A95AAB
:102F1000DE5D79C0B086BFB17F6FA95ADA8F75A91F
:102F20005ADE5B79C0B086BFB17F6CA95ADA8C7368
:102F3000A95ADE5979C0B086BFB17F6AA95ADA8A28
:102F400071A95ADE5779C0B086BFB17F67A95ADA36
:102F5000876FA95ADE5579C0B086BFB17F65A95A7F
:102F6000DA856DA95ADE5379C0B086BFB17F62A9F8
:102F70005ADA826BA95ADE5179C0B086BFB17F6040
:102F8000A95ADA8069A95ADE4F79C0B086BFB17FED
:102F900060AD6BD18069A95ADE4F79C0B086BFB1F0
:102FA0007F60B078CA8069A95ADE4F79C0B086BF09
:102FB000B17F60B383C48069A95ADE4F79C0B086FF
:102FC000BFB17F60B58CBE8069A95ADE4F79C0B0B1
:102FD00086BFB17F60B795BA8069A95ADE4F79C0C4
:102FE000B086BFB17F5EB691BC7E69A95ADE4F79CB
:102FF000C0B086BFB17F5DB58CBE7D69A95ADE4F7A
:1030000079C0B086BFB17F5BB488C17B69A95ADE45
:103010004F79C0B086BFB17F5AB383C47A69A95AC9
:10302000DE4F79C0B086BFB17F58B17DC77869A93E
:103030005ADE4F79C0B086BFB17F57B078CA776982
:10304000A95ADE4F79C0B086BFB17F55AF72CD753A
:1030500069A95ADE4F79C0B086BFB17F54AD6BD13C
:103060007369A95ADE4F79C0B086BFB17F52AB6396
:10307000D57269A95ADE4F79C0B086BFB17F51A918
:103080005ADA7069A95ADE4F79C0B086BFB17F5451
:10309000A95ADA736CA95ADE5279C0B086BFB17FE3
:1030A00057A95ADA766FA95ADE5579C0B086BFB1F2
:1030B0007F5AA95ADA7972A95ADE5879C0B086BF08
:1030C000B17F5DA95ADA7C75A95ADE5B79C0B086FA
:1030D000BFB17F60A95ADA7F78A95ADE5E79C0B0A5
:1030E00086BFB17F63A95ADA827BA95ADE6179C0B3
:1030F000B086BFB17F66A95ADA857DA95ADE6479A8
:10310000C0B086BFB17F69A95ADA8880A95ADE6744
:1031100079C0B086BFB17F6CA95ADA8B83A95ADE19
:103120006A79C0B086BFB17F6FA95ADA8E86A95A74
:10313000DE6D79C0B086BFB17F72A95ADA9189A9D4
:103140005ADE7079C0B086BFB17F75A95ADA948C07
:10315000A95ADE7379C0B086BFB17F78A95ADA97D1
:103160008FA95ADE7679C0B086BFB17F7AA95ADAC4
:103170009A92A95ADE7979C0B086BFB17F7DA95AEB
:10318000DA9D95A95ADE7C79C0B086BFB17F80A94F
:103190005ADAA098A95ADE7F79C0B086BFB17F8382
:1031A000A95ADAA39BA95ADE8279C0B086BFB17F43
:1031B00086A95ADAA69EA95ADE8579C0B086BFB123
:1031C0007F89A95ADAA9A1A95ADE8879C0B086BF39
:1031D000B17F8CA95ADAACA4A95ADE8B79C0B0862B
:1031E000BFB17F8CA95ADAACA1AD6BD58879C0B0DC
:1031F00086BFB17F8CA95ADAAC9EB078CE8479C0F4
:10320000B086BFB17F8CA95ADAAC9BB383C88179F1
:10321000C0B086BFB17F8CA95ADAAC98B58CC27E9B
:1032200079C0B086BFB17F8CA95ADAAC95B795BE8C
:103230007B79C0B086BFB17F8CA95ADAAC95B691C4
:10324000C07B79C0B086BFB17F8CA95ADAAC95B586
:103250008CC27B79C0B086BFB17F8CA95ADAAC959D
:10326000B488C57B79C0B086BFB17F8CA95ADAAC6F
:1032700095B383C87B79C0B086BFB17F8CA95ADA79
:10328000AC95B17DCB7B79C0B086BFB17F8CA95A9C
:10329000DAAC95B078CE7B79C0B086BFB17F8CA90F
:1032A0005ADAAC95AF72D17B79C0B086BFB17F8C52
:1032B000A95ADAAC95AD6BD57B79C0B086BFB17F2A
:1032C0008CA95ADAAC95AB63D97B79C0B086BFB113
:1032D0007F8CA95ADAAC95A95ADE7B79C0B086BF3B
:1032E000B17F8BA95ADAAB94A95ADE7A79C0B0863D
:1032F000BFB17F8AA95ADAAA93A95ADE7979C0B0F8
:1033000086BFB17F89A95ADAA991A95ADE7879C016
:10331000B086BFB17F88A95ADAA890A95ADE76791B
:10332000C0B086BFB17F87A95ADAA78FA95ADE75C8
:1033300079C0B086BFB17F86A95ADAA68EA95ADEB7
:103340007479C0B086BFB17F85A95ADAA58CA95A15
:10335000DE7379C0B086BFB17F84A95ADAA48BA985
:103360005ADE7179C0B086BFB17F83A95ADAA38AC9
:10337000A95ADE7079C0B086BFB17F82A95ADAA29D
:1033800089A95ADE6F79C0B086BFB17F81A95ADAA8
:10339000A188A95ADE6E79C0B086BFB17F80A95AD4
:1033A000DAA086A95ADE6C79C0B086BFB17F7FA94A
:1033B0005ADA9F85A95ADE6B79C0B086BFB17F7E8D
:1033C000A95ADA9E84A95ADE6A79C0B086BFB17F55
:1033D0007DA95ADA9D83A95ADE6979C0B086BFB14A
:1033E0007F7CA95ADA9C81A95ADE6779C0B086BF72
:1033F000B17F7BA95ADA9B80A95ADE6679C0B08674
:10340000BFB17F7AA95ADA9A7FA95ADE6579C0B02E
:1034100086BFB17F79A95ADA997EA95ADE6479C04C
:10342000B086BFB17F79A95ADA997DA95ADE63794E
:10343000C0B086BFB17F79A95ADA997DA95ADE63F7
:1034400079C0B086BFB17F79A95ADA997DA95ADED1
:103450006379C0B086BFB17F79A95ADA997DA95A3C
:10346000DE6379C0B086BFB17F79A95ADA997DA9A8
:103470005ADE6379C0B086BFB17F79A95ADA997DE7
:10348000A95ADE6379C0B086BFB17F79A95ADA99AB
:103490007DA95ADE6379C0B086BFB17F79A95ADAB7
:1034A000997DA95ADE6379C0B086BFB17F79A95AE8
:1034B000DA997DA95ADE6379C0B086BFB17F79A958
:1034C0005ADA997DA95ADE6379C0B086BFB17F7997
:1034D000A95ADA997DA95ADE6379C0B086BFB17F57
:1034E00079A95ADA997DA95ADE6379C0B086BFB14D
:1034F0007F79A95ADA997DA95ADE6379C0B086BF6F
:10350000B17F79A95ADA997DA95ADE6379C0B0866C
:10351000BFB17F79A95ADA997DA95ADE6379C0B023
:1035200086BFB17F79A95ADA997DA95ADE6379C03D
:10353000B086BFB17F000000000000000000000066
:103540000303030303030300000000000000000066
:103550000003030303030303000000000000000056
:103560000000030303030303030000000000000046
:103570000000000303030303030300000000000036
:103580000000000003030303030303000000000026
:103590000000000000030303030303030000000016
:1035A0000000000000000303030303030300000006
:1035B00000000000000000030303030303030000F6
:1035C00000000000000000000303030303030300E6
:1035D00000000000000000000003030303030303D6
:1035E00000000000000000000000030303030303C9
:1035F00003000000000000000000000303030303B9
:1036000003030000000000000000000003030303A8
:103610000303030000000000000000000003030398
:103620000303030300000000000000000000030388
:103630000303030303000000000000000000000378
:103640000303030303030000000000000000000068
:103650000303030303030300000000000000000055
:103660000003030303030303000000000000000045
:103670000000030303030303030000000000000035
:103680000000000303030303030300000000000025
:103690000000000003030303030303000000000015
:1036A0000000000000030303030303030000000005
:1036B00000000000000003030303030303000000F5
:1036C00000000000000000030303030303030000E5
:1036D00000000000000000000303030303030300D5
:1036E00000000000000000000003030303030303C5
:1036F00000000000000000000000030303030303B8
:1037000003000000000000000000000303030303A7
:103710000303000000000000000000000303030397
:103720000303030000000000000000000003030387
:103730000303030300000000000000000000030377
:103740000303030303000000000000000000000367
:103750000303030303030000000000000000000057
:103760000303030303030300000000000000000044
:103770000003030303030303000000000000000034
:103780000000030303030303030000000000000024
:103790000000000303030303030300000000000014
:1037A0000000000003030303030303000000000004
:1037B00000000000000303030303030300000000F4
:1037C00000000000000003030303030303000000E4
:1037D00000000000000000030303030303030000D4
:1037E00000000000000000000303030303030300C4
:1037F00000000000000000000003030303030303B4
:1038000000000000000000000000030303030303A6
:103810000300000000000000000000030303030396
:103820000303000000000000000000000303030386
:103830000303030000000000000000000003030376
:103840000303030300000000000000000000030366
:103850000303030303000000000000000000000356
:103860000303030303030000000000000000000046
:103870000303030303030300000000000000000033
:103880000003030303030303000000000000000023
:103890000000030303030303030000000000000013
:1038A0000000000303030303030300000000000003
:1038B00000000000030303030303030000000000F3
:1038C00000000000000303030303030300000000E3
:1038D00000000000000003030303030303000000D3
:1038E00000000000000000030303030303030000C3
:1038F00000000000000000000303030303030300B3
:1039000000000000000000000003030303030303A2
:103910000000000000000000000003030303030395
:103920000300000000000000000000030303030385
:103930000303000000000000000000000303030375
:103940000303030000000000000000000003030365
:103950000303030300000000000000000000030355
:103960000303030303000000000000000000000345
:103970000303030303030000000000000000000035
:103980000303030303030300000000000000000022
:103990000003030303030303000000000000000012
:1039A0000000030303030303030000000000000002
:1039B00000000003030303030303000000000000F2
:1039C00000000000030303030303030000000000E2
:1039D00000000000000303030303030300000000D2
:1039E00000000000000003030303030303000000C2
:1039F00000000000000000030303030303030000B2
:103A000000000000000000000303030303030300A1
:103A10000000000000000000000303030303030391
:103A20000000000000000000000003030303030384
:103A30000300000000000000000000030303030374
:103A40000303000000000000000000000303030364
:103A50000303030000000000000000000003030354
:103A60000303030300000000000000000000030344
:103A70000303030303000000000000000000000334
:103A80000303030303030000000000000000000024
:103A90000303030303030300000000000000000011
:103AA0000003030303030303000000000000000001
:103AB00000000303030303030300000000000000F1
:103AC00000000003030303030303000000000000E1
:103AD00000000000030303030303030000000000D1
:103AE00000000000000303030303030300000000C1
:103AF00000000000000003030303030303000000B1
:103B000000000000000000030303030303030000A0
:103B10000000000000000000030303030303030090
:103B20000000000000000000000303030303030380
:103B30000000000000000000000003030303030373
:103B40000300000000000000000000030303030363
:103B50000303000000000000000000000303030353
:103B60000303030000000000000000000003030343
:103B70000303030300000000000000000000030333
:103B80000303030303000000000000000000000323
:103B90000303030303030000000000000000000013
:103BA0000303030303030300000000000000000000
:103BB00000030303030303030000000000000000F0
:103BC00000000303030303030300000000000000E0
:103BD00000000003030303030303030202020303C1
:103BE00002020203030303030303030302020203AB
:103BF000030202020303030303030303030202029B
:103C00000303020202030303030303030303020289
:103C10000203030202020303030303030303030279
:103C2000020203030202020303030303030303006C
:103C300079A95CD9997DA95CDD6379C0B086BFB1F3
:103C40007F79AA5DD8997DAA5DDC6379C0B086BF13
:103C5000B17F79AA5ED8997DAA5EDC6379C0B0860F
:103C6000BFB17F79AA5FD7997DAA5FDB6379C0B0C6
:103C700086BFB17F79AA60D7997DAA60DB6379C0DE
:103C8000B086BFB17F79AB62D6997DAB62DA6379DA
:103C9000C0B086BFB17F79AB63D5997DAB63D96383
:103CA00079C0B086BFB17F79AB64D5997DAB64D95B
:103CB0006379C0B086BFB17F79AC65D4997DAC65BE
:103CC000D86379C0B086BFB17F79AC66D4997DAC3A
:103CD00066D86379C0B086BFB17F79AA65D0997D77
:103CE000AE65DC6379C0B086BFB17C79A764CD993D
:103CF0007DAF64E16379C0B086BFB17979A461CB4F
:103D0000997DB161E66379C0B086BFB17679A15C77
:103D1000CA997DB15CEC6379C0B086BFB173799EFE
:103D200055CA997DB255F46379C0B086BFB16F773B
:103D30009E55CA967BB257F26179C0B086BFB16F0B
:103D4000759E55CA947AB259F06079C0B086BFB1F9
:103D50006F739E55CA9279B25AEE5F79C0B086BF32
:103D6000B16F729E55CA9078B15CEC5E79C0B08636
:103D7000BFB16F709E55CA8E76B15DEB5C79C0B0F5
:103D800086BFB16F6E9E55CA8C75B15EE95B79C016
:103D9000B086BFB16F6D9E55CA8A74B160E85A791A
:103DA000C0B086BFB16F6B9E55CA8873B161E659CA
:103DB00079C0B086BFB16F699E55CA8671B061E5A2
:103DC0005779C0B086BFB16F689E55CA8370B06224
:103DD000E35679C0B086BFB16F669E55CA816FB099
:103DE00063E25579C0B086BFB16F649E55CA7F6EDD
:103DF000AF64E15479C0B086BFB16F639E55CA7D90
:103E00006DAF64DF5379C0B086BFB16F619E55CA94
:103E10007B6BAE65DE5179C0B086BFB16F5F9E55DA
:103E2000CA796AAE65DD5079C0B086BFB16F5E9E5B
:103E300055CA7769AE65DC4F79C0B086BFB16F5C9B
:103E40009E55CA7568AD66DB4E79C0B086BFB16F4E
:103E50005A9E55CA7366AD66DA4C79C0B086BFB15A
:103E60006F599E55CA7165AC66D94B79C0B086BF93
:103E7000B16F579E55CA6E64AC66D84A79C0B08699
:103E8000BFB16F57A670BE6E64AC66D84A79C0B039
:103E900086BFB16F57AC82B86E64AC66D84A79C041
:103EA000B086BFB16F57B191B36E64AC66D84A7932
:103EB000C0B086BFB16F57B69DB16E64AC66D84ACC
:103EC00079C0B086BFB16F57BBA7AF6E64AC66D880
:103ED0004A79C0B086BFB16F57BB9DBA6E64AC66FD
:103EE000D84A79C0B086BFB16F57BA91C56E64AC7D
:103EF00066D84A79C0B086BFB16F57B982D06E64B8
:103F0000AC66D84A79C0B086BFB16F57B770DE6E65
:103F100064AC66D84A79C0B086BFB16F57B255F06D
:103F20006E64AC66D84A79C0B086BFB16F58B256DD
:103F3000EE7065AC66D84B79C0B086BFB17059B22F
:103F400058ED7166AC66D84C79C0B086BFB1715A75
:103F5000B259EC7366AC66D84C79C0B086BFB1710B
:103F60005BB25AEB7467AC66D84D79C0B086BFB10E
:103F7000725CB25BEA7568AC66D84E79C0B086BF39
:103F8000B1725EB15CE87769AC66D84F79C0B08633
:103F9000BFB1735FB15DE7786AAC66D85079C0B0E5
:103FA00086BFB17360B15EE67A6BAC66D85179C0FA
:103FB000B086BFB17461B15EE57B6BAC66D85179F8
:103FC000C0B086BFB17462B15FE47C6CAC66D8529D
:103FD00079C0B086BFB17563B160E37E6DAC66D861
:103FE0005379C0B086BFB17564B161E27F6EAC66D3
:103FF000D85479C0B086BFB17665B061E1816FAC4D
:1040000066D85579C0B086BFB17667B062E0826F7E
:10401000AC66D85579C0B086BFB17768B062DF832F
:1040200070AC66D85679C0B086BFB17769B063DE30
:104030008571AC66D85779C0B086BFB1786AAF6376
:10404000DD8672AC66D85879C0B086BFB1796BAFE7
:1040500064DD8873AC66D85979C0B086BFB1796C1D
:10406000AF64DC8974AC66D85A79C0B086BFB17AC7
:104070006DAF64DB8A74AC66D85A79C0B086BFB1C4
:104080007A6EAE65DA8C75AC66D85B79C0B086BFE7
:10409000B17B70AE65D98D76AC66D85C79C0B086E0
:1040A000BFB17B71AE65D98F77AC66D85D79C0B092
:1040B00086BFB17C72AE65D89078AC66D85E79C0A8
:1040C000B086BFB17C73AD66D79178AC66D85E79A7
:1040D000C0B086BFB17D74AD66D69379AC66D85F4B
:1040E00079C0B086BFB17D75AD66D6947AAC66D81E
:1040F0006079C0B086BFB17E76AC66D5967BAC6683
:10410000D86179C0B086BFB17E77AC66D4977CACFD
:1041100066D86279C0B086BFB17F79AC66D4997D2C
:10412000AC66D86379C0B086BFB17F79AC65D499ED
:104130007DAC65D86379C0B086BFB17F79AB64D5FB
:10414000997DAB64D96379C0B086BFB17F79AB6329
:10415000D5997DAB63D96379C0B086BFB17F79ABA8
:1041600062D6997DAB62DA6379C0B086BFB17F79E0
:10417000AA60D7997DAA60DB6379C0B086BFB17FA2
:1041800079AA5FD7997DAA5FDB6379C0B086BFB19A
:104190007F79AA5ED8997DAA5EDC6379C0B086BFBC
:1041A000B17F79AA5DD8997DAA5DDC6379C0B086BC
:1041B000BFB17F79A95CD9997DA95CDD6379C0B075
:1041C00086BFB17F79A95ADA997DA95ADE6379C091
:1041D000B086BFB17F79A95ADA997DA95ADE637991
:1041E000C0B086BFB17F79A95ADA997DA95ADE633A
:1041F00079C0B086BFB17F79A95ADA997DA95ADE14
:104200006379C0B086BFB17F79A95ADA997DA95A7E
:10421000DE6379C0B086BFB17F79A95ADA997DA9EA
:104220005ADE6379C0B086BFB17F03030303030383
:10423000030303030303030303030303030303034E
:10424000030303030303030303030303030303033E
:10425000030303030303030303030303030303032E
:10426000030303030303030303030303030303031E
:10427000030303030303030303030303030303030E
:1042800003030303030303030303030303030303FE
:1042900003030303030303030303030303030303EE
:1042A00003030303030303030303030303030303DE
:1042B00003030303030303030303030303030303CE
:1042C00003030303030303030303030303030303BE
:1042D00003030303030000000303000000030303C0
:1042E00003030303030300000003030000000303B0
:1042F00003030303030303000000030300000003A0
:10430000030303030303030300000003030000008F
:10431000030303030303030303000000030300007C
:104320000003030303030303030000000000000075
:104330000000000303030303030300000000000068
:104340000000000003030303030303000000000058
:104350000000000000030303030303030000000048
:104360000000000000000303030303030300000038
:104370000000000000000003030303030303000028
:104380000000000000000000030303030303030018
:104390000000000000000000000303030303030308
:1043A00000000000000000000000030303030303FB
:1043B00003000000000000000000000303030303EB
:1043C00003030000000000000000000003030303DB
:1043D00003030300000000000000000000030303CB
:1043E00003030303000000000000000000000303BB
:1043F00003030303030000000000000000000003AB
:10440000030303030303000000000000000000009A
:104410000303030303030300000000000000000087
:104420000003030303030303000000000000000077
:104430000000030303030303030000000000000067
:104440000000000303030303030300000000000057
:104450000000000003030303030303000000000047
:104460000000000000030303030303030000000037
:104470000000000000000303030303030300000027
:104480000000000000000003030303030303000017
:104490000000000000000000030303030303030007
:1044A00000000000000000000003030303030303F7
:1044B00000000000000000000000030303030303EA
:1044C00003000000000000000000000303030303DA
:1044D00003030000000000000000000003030303CA
:1044E00003030300000000000000000000030303BA
:1044F00003030303000000000000000000000303AA
:104500000303030303000000000000000000000399
:104510000303030303030000000000000000000089
:104520000303030303030300000000000000000076
:104530000003030303030303000000000000000066
:104540000000030303030303030000000000000056
:104550000000000303030303030300000000000046
:104560000000000003030303030303000000000036
:104570000000000000030303030303030000000026
:104580000000000000000303030303030300000016
:104590000000000000000003030303030303000006
:1045A00000000000000000000303030303030300F6
:1045B00000000000000000000003030303030303E6
:1045C00000000000000000000000030303030303D9
:1045D00003000000000000000000000303030303C9
:1045E00003030000000000000000000003030303B9
:1045F00003030300000000000000000000030303A9
:104600000303030300000000000000000000030398
:104610000303030303000000000000000000000388
:104620000303030303030000000000000000000078
:104630000303030303030300000000000000000065
:104640000003030303030303000000000000000055
:104650000000030303030303030000000000000045
:104660000000000303030303030300000000000035
:104670000000000003030303030303000000000025
:104680000000000000030303030303030000000015
:104690000000000000000303030303030300000005
:1046A00000000000000000030303030303030000F5
:1046B00000000000000000000303030303030300E5
:1046C00000000000000000000003030303030303D5
:1046D00000000000000000000000030303030303C8
:1046E00003000000000000000000000303030303B8
:1046F00003030000000000000000000003030303A8
:104700000303030000000000000000000003030397
:104710000303030300000000000000000000030387
:104720000303030303000000000000000000000377
:104730000303030303030000000000000000000067
:104740000303030303030300000000000000000054
:104750000003030303030303000000000000000044
:104760000000030303030303030000000000000034
:104770000000000303030303030300000000000024
:104780000000000003030303030303000000000014
:104790000000000000030303030303030000000004
:1047A00000000000000003030303030303000000F4
:1047B00000000000000000030303030303030000E4
:1047C00000000000000000000303030303030303D1
:1047D00002020203030202020303030303030303AF
:1047E000030202020303020202030303030303039F
:1047F000030302020203030202020303030303038F
:10480000030303020202030302020203030303037E
:10481000030303030202020303020202030303036E
:104820000303030379A95DD8997DA95DDC6379C091
:10483000B086BFB17F79AA5FD6997DAA5FDA637926
:10484000C0B086BFB17F79AA62D5997DAA62D963CB
:1048500079C0B086BFB17F79AA64D3997DAA64D7A5
:104860006379C0B086BFB17F79AB66D2997DAB6604
:10487000D66379C0B086BFB17F79AB68D0997DAB84
:1048800068D46379C0B086BFB17F79AB6ACF997DB8
:10489000AB6AD36379C0B086BFB17F79AB6BCD997A
:1048A0007DAB6BD16379C0B086BFB17F79AC6DCC85
:1048B000997DAC6DD06379C0B086BFB17F79AC6FA4
:1048C000CB997DAC6FCF6379C0B086BFB17F7AAC36
:1048D0006FCB9A7EAC6FCF6479C0B086BFB17F7B5F
:1048E000AC6FCB9B80AC6FCF6679C0B086BFB17F19
:1048F0007CAC6FCB9C82AC6FCF6878C0B085BFB109
:104900007F7DAC6FCB9D83AC6FCF6A78C0B085BF25
:10491000B17F7FAC6FCB9F85AC6FCF6C77C0B0841D
:10492000BFB17F80AC6FCBA087AC6FCF6E77C0B0CC
:1049300084BFB17F81AC6FCBA188AC6FCF7077C0E3
:10494000B084BFB17F82AC6FCBA28AAC6FCF7276DE
:10495000C0B083BFB17F84AC6FCBA48CAC6FCF747D
:1049600076C0B083BFB17F85AC6FCBA58DAC6FCF68
:104970007575C0B082BFB17F86AC6FCBA68FAC6FB0
:10498000CF7775C0B082BFB17F87AC6FCBA791AC3A
:104990006FCF7975C0B082BFB17F88AC6FCBA89262
:1049A000AC6FCF7B74C0B081BFB17F8AAC6FCBAA34
:1049B00094AC6FCF7D74C0B081BFB17F8BAC6FCB37
:1049C000AB96AC6FCF7F73C0B080BFB17F8CAC6F44
:1049D000CBAC97AC6FCF8173C0B080BFB17F8DACD3
:1049E0006FCBAD99AC6FCF8373C0B080BFB17F8FF9
:1049F000AC6FCBAF9BAC6FCF8572C0B07FBFB17FC8
:104A000090AC6FCBB09CAC6FCF8672C0B07FBFB1A3
:104A10007F91AC6FCBB19EAC6FCF8871C0B07EBFC1
:104A2000B17F91AC6FCBB19EAD7BC68871C0B07EBB
:104A3000BFB17F91AC6FCBB19EAF84BF8871C0B066
:104A40007EBFB17F91AC6FCBB19EAF8DB78871C087
:104A5000B07EBFB17F91AC6FCBB19EB095B1887184
:104A6000C0B07EBFB17F91AC6FCBB19EB09CAA8825
:104A700071C0B07EBFB17F91AC6FCBB19EAD92AE35
:104A80008871C0B07EBFB17F91AC6FCBB19EAA8858
:104A9000B28871C0B07EBFB17F91AC6FCBB19EA622
:104AA0007CB78871C0B07EBFB17F91AC6FCBB19E37
:104AB000A26DBE8871C0B07EBFB17F91AC6FCBB12B
:104AC0009E9D5AC78871C0B07EBFB17F00000000B4
:104AD00000000000000003030303030303000000C1
:104AE00000000000000000030303030303030000B1
:104AF00000000000000000000303030303030300A1
:104B00000000000000000000000303030303030390
:104B10000000000000000000000003030303030383
:104B20000300000000000000000000030303030373
:104B30000303000000000000000000000303030363
:104B40000303030000000000000000000003030353
:104B50000303030300000000000000000000030343
:104B60000303030303000000000000000000000333
:104B70000303030303030000000000000000000023
:104B80000303030303030300000000000000000010
:104B90000003030303030303000000000000000000
:104BA00000000303030303030300000000000000F0
:104BB00000000003030303030303000000000000E0
:104BC00000000000030303030303030000000000D0
:104BD00000000000000303030303030300000000C0
:104BE00000000000000003030303030303000000B0
:104BF00000000000000000030303030303030000A0
:104C0000000000000000000003030303030303008F
:104C1000000000000000000000030303030303037F
:104C20000000000000000000000003030303030372
:104C30000300000000000000000000030303030362
:104C40000303000000000000000000000303030352
:104C50000303030000000000000000000003030342
:104C60000303030300000000000000000000030332
:104C70000303030303000000000000000000000322
:104C80000303030303030000000000000000000012
:104C900003030303030303000000000000000000FF
:104CA00000030303030303030000000000000000EF
:104CB00000000303030303030300000000000000DF
:104CC00000000003030303030303000000000000CF
:104CD00000000000030303030303030000000000BF
:104CE00000000000000303030303030300000000AF
:104CF000000000000000030303030303030000009F
:104D0000000000000000000303030303030300008E
:104D1000000000000000000003030303030303007E
:104D2000000000000000000000030303030303036E
:104D30000000000000000000000003030303030361
:104D40000300000000000000000000030303030351
:104D50000303000000000000000000000303030341
:104D60000303030000000000000000000003030331
:104D7000030303038EAC6FCCAE9B9E5CC68572C0F2
:104D8000B07FBFB17F8BAD6FCCAB989F5EC6827397
:104D9000C0B080BFB17F88AD6FCDA895A060C67F41
:104DA00074C0B081BFB17F85AE6FCEA593A162C63E
:104DB0007B75C0B082BFB17F82AF6FCFA290A1637D
:104DC000C77875C0B082BFB17F80AF6FD0A08DA211
:104DD00065C77576C0B083BFB17F7DB06FD19D8A46
:104DE000A366C77177C0B084BFB17F7AB06FD39A22
:104DF00087A467C76E78C0B085BFB17F77B06FD426
:104E00009784A568C86B79C0B086BFB17F74B16E56
:104E1000D59381A569C86879C0B086BFB17F71B1EB
:104E20006ED6907EA66AC9647AC0B087BFB17F6E25
:104E3000B26DD78D7BA76BC9617BC0B088BFB17FD6
:104E40006BB26DD98A78A76CCA5E7CC0B089BFB1DD
:104E50007F68B26CDA8675A86CCA5B7DC0B08ABF09
:104E6000B17F65B36CDB8373A96DCB597DC0B08A0C
:104E7000BFB17F62B36BDD8070A96DCC567EC0B0D0
:104E80008BBFB17F60B36ADE7C6DAA6ECC537FC0EE
:104E9000B08CBFB17F5DB469E0796AAB6ECD5080F4
:104EA000C0B08DBFB17F5AB468E17667AB6FCE4DAD
:104EB00081C0B08EBFB17F57B467E37364AC6FCF6E
:104EC0004A81C0B08EBFB17F57B77BD47364AC6FDB
:104ED000CF4A81C0B08EBFB17F57B98BC87364AC65
:104EE0006FCF4A81C0B08EBFB17F57BA97BD736490
:104EF000AC6FCF4A81C0B08EBFB17F57BAA2B27338
:104F000064AC6FCF4A81C0B08EBFB17F57B9ACA837
:104F10007364AC6FCF4A81C0B08EBFB17F57B5A16B
:104F2000AA7364AC6FCF4A81C0B08EBFB17F57B057
:104F300095AD7364AC6FCF4A81C0B08EBFB17F575F
:104F4000AB86B17364AC6FCF4A81C0B08EBFB17F06
:104F500057A574B87364AC6FCF4A81C0B08EBFB12F
:104F60007F579D5AC37364AC6FCF4A81C0B08EBF68
:104F7000B17F5A9E5CC27667AC6FD04D81C0B08E57
:104F8000BFB17F5D9F5EC2796AAD6FD05080C0B007
:104F90008DBFB17F60A060C27C6DAD6FD1537FC00B
:104FA000B08CBFB17F62A162C28070AE6FD2567EFC
:104FB000C0B08BBFB17F65A163C38373AF6FD3599B
:104FC0007DC0B08ABFB17F68A265C38675AF6FD45C
:104FD0005B7DC0B08ABFB17F6BA366C38A78B06FB8
:104FE000D55E7CC0B089BFB17F6EA467C38D7BB036
:104FF0006FD7617BC0B088BFB17F71A568C4907E58
:10500000B06FD8647AC0B087BFB17F74A569C4930C
:1050100081B16ED96879C0B086BFB17F77A66AC505
:105020009784B16EDA6B79C0B086BFB17F7AA76B17
:10503000C59A87B26DDB6E78C0B085BFB17F7DA7A2
:105040006CC69D8AB26DDD7177C0B084BFB17F80C0
:10505000A86CC6A08DB26CDE7576C0B083BFB17F80
:1050600082A96DC7A290B36CDF7875C0B082BFB162
:105070007F85A96DC8A593B36BE17B75C0B082BF76
:10508000B17F88AA6EC8A895B36AE27F74C0B08168
:10509000BFB17F8BAB6EC9AB98B469E48273C0B00B
:1050A00080BFB17F8EAB6FCAAE9BB468E58572C01E
:1050B000B07FBFB17F91AC6FCBB19EB467E7887111
:1050C000C0B07EBFB17F91AC6FCBB19EB77BD888AB
:1050D00071C0B07EBFB17F91AC6FCBB19EB98BCCAC
:1050E0008871C0B07EBFB17F91AC6FCBB19EBA97D3
:1050F000C18871C0B07EBFB17F91AC6FCBB19EBA99
:10510000A2B68871C0B07EBFB17F91AC6FCBB19EAB
:10511000B9ACAC8871C0B07EBFB17F91AC6FCBB180
:105120009EB5A1AE8871C0B07EBFB17F91AC6FCB90
:10513000B19EB095B18871C0B07EBFB17F91AC6FA8
:10514000CBB19EAB86B58871C0B07EBFB17F91AC4C
:105150006FCBB19EA574BC8871C0B07EBFB17F918A
:10516000AC6FCBB19E9D5AC78871C0B07EBFB17F76
:10517000000000000000000000000303030303031D
:10518000030000000000000000000003030303030D
:1051900003030000000000000000000003030303FD
:1051A00003030300000000000000000000030303ED
:1051B00003030303000000000000000000000303DD
:1051C00003030303030000000000000000000003CD
:1051D00003030303030300000000000000000000BD
:1051E00003030303030303000000000000000000AA
:1051F000000303030303030300000000000000009A
:105200000000030303030303030000000000000089
:105210000000000303030303030300000000000079
:105220000000000003030303030303000000000069
:105230000000000000030303030303030000000059
:105240000000000000000303030303030300000049
:105250000000000000000003030303030303000039
:105260000000000000000000030303030303030029
:105270000000000000000000000303030303030319
:10528000000000000000000000000303030303030C
:1052900003000000000000000000000303030303FC
:1052A00003030000000000000000000003030303EC
:1052B00003030300000000000000000000030303DC
:1052C00003030303000000000000000000000303CC
:1052D00003030303030000000000000000000003BC
:1052E00003030303030300000000000000000000AC
:1052F0000303030303030300000000000000000099
:105300000003030303030303000000000000000088
:105310000000030303030303030000000000000078
:105320000000000303030303030300000000000068
:105330000000000003030303030303000000000058
:105340000000000000030303030303030000000048
:105350000000000000000303030303030300000038
:105360000000000000000003030303030303000028
:105370000000000000000000030303030303030018
:105380000000000000000000000303030303030308
:1053900000000000000000000000030303030303FB
:1053A00003000000000000000000000303030303EB
:1053B00003030000000000000000000003030303DB
:1053C00003030300000000000000000000030303CB
:1053D00003030303000000000000000000000303BB
:1053E00003030303030000000000000000000003AB
:1053F000030303030303000000000000000000009B
:105400000303030303030300000000000000000087
:105410000003030303030303000000000000000077
:105420000000030303030303030000000000000067
:105430000000000303030303030300000000000057
:105440000000000003030303030303000000000047
:105450000000000000030303030303030000000037
:105460000000000000000303030303030300000027
:105470000000000000000003030303030303000017
:105480000000000000000000030303030303030007
:1054900000000000000000000003030303030303F7
:1054A00000000000000000000000030303030303EA
:1054B00003000000000000000000000303030303DA
:1054C00003030000000000000000000003030303CA
:1054D00003030300000000000000000000030303BA
:1054E00003030303000000000000000000000303AA
:1054F000030303030300000000000000000000039A
:105500000303030303030000000000000000000089
:105510000303030303030300000000000000000076
:105520000003030303030303000000000000000066
:105530000000030303030303030000000000000056
:105540000000000303030303030300000000000046
:105550000000000003030303030303000000000036
:105560000000000000030303030303038EAC6FCCB1
:10557000AE9B9E5CC68572C0B07FBFB17F8BAD6FA6
:10558000CCAB989F5EC68273C0B080BFB17F88AD40
:105590006FCDA895A060C67F74C0B081BFB17F8574
:1055A000AE6FCEA593A162C67B75C0B082BFB17F3E
:1055B00082AF6FCFA290A163C77875C0B082BFB130
:1055C0007F80AF6FD0A08DA265C77576C0B083BF56
:1055D000B17F7DB06FD19D8AA366C77177C0B0845B
:1055E000BFB17F7AB06FD39A87A467C76E78C0B017
:1055F00085BFB17F77B06FD49784A568C86B79C039
:10560000B086BFB17F74B16ED59381A569C8687942
:10561000C0B086BFB17F71B16ED6907EA66AC964F4
:105620007AC0B087BFB17F6EB26DD78D7BA76BC9D3
:10563000617BC0B088BFB17F6BB26DD98A78A76C2F
:10564000CA5E7CC0B089BFB17F68B26CDA8675A8CB
:105650006CCA5B7DC0B08ABFB17F65B36CDB8373FE
:10566000A96DCB597DC0B08ABFB17F62B36BDD80BD
:1056700070A96DCC567EC0B08BBFB17F60B36ADEBF
:105680007C6DAA6ECC537FC0B08CBFB17F5DB46916
:10569000E0796AAB6ECD5080C0B08DBFB17F5AB497
:1056A00068E17667AB6FCE4D81C0B08EBFB17F57DA
:1056B000B467E37364AC6FCF4A81C0B08EBFB17F73
:1056C00057B776D97364AC6FCF4A81C0B08EBFB183
:1056D0007F57B982D07364AC6FCF4A81C0B08EBFA0
:1056E000B17F57BB8DC97364AC6FCF4A81C0B08E98
:1056F000BFB17F57BC96C27364AC6FCF4A81C0B054
:105700008EBFB17F57BD9FBB7364AC6FCF4A81C062
:10571000B08EBFB17F57BA97BD7364AC6FCF4A816B
:10572000C0B08EBFB17F57B78FBF7364AC6FCF4A25
:1057300081C0B08EBFB17F57B386C27364AC6FCFE8
:105740004A81C0B08EBFB17F57B07BC67364AC6F67
:10575000CF4A81C0B08EBFB17F57AC6FCB7364AC02
:105760006FCF4A81C0B08EBFB17F59AC6FCB75652A
:10577000AC6FCF4B81C0B08EBFB17F5AAC6FCB76D0
:1057800066AC6FCF4C81C0B08EBFB17F5CAC6FCBCD
:105790007868AC6FCF4E80C0B08DBFB17F5EAC6F0C
:1057A000CB7A69AC6FCF4F80C0B08DBFB17F5FAC9B
:1057B0006FCB7C6AAC6FCF507FC0B08CBFB17F61C4
:1057C000AC6FCB7E6BAC6FCF517FC0B08CBFB17F65
:1057D00063AC6FCB806DAC6FCF537FC0B08CBFB16B
:1057E0007F64AC6FCB826EAC6FCF547EC0B08BBF8A
:1057F000B17F66AC6FCB846FAC6FCF557EC0B08B82
:10580000BFB17F68AC6FCB8670AC6FCF567DC0B038
:105810008ABFB17F69AC6FCB8771AC6FCF577DC04A
:10582000B08ABFB17F6BAC6FCB8973AC6FCF597D42
:10583000C0B08ABFB17F6DAC6FCB8B74AC6FCF5AE9
:105840007CC0B089BFB17F6EAC6FCB8D75AC6FCFB4
:105850005B7CC0B089BFB17F70AC6FCB8F76AC6F13
:10586000CF5C7BC0B088BFB17F72AC6FCB9178AC9E
:105870006FCF5E7BC0B088BFB17F73AC6FCB9379C5
:10588000AC6FCF5F7BC0B088BFB17F75AC6FCB957D
:105890007AAC6FCF607AC0B087BFB17F77AC6FCB87
:1058A000977BAC6FCF617AC0B087BFB17F79AC6FA7
:1058B000CB997DAC6FCF6379C0B086BFB17F79AC37
:1058C0006DCC997DAC6DD06379C0B086BFB17F7966
:1058D000AB6BCD997DAB6BD16379C0B086BFB17F27
:1058E00079AB6ACF997DAB6AD36379C0B086BFB11B
:1058F0007F79AB68D0997DAB68D46379C0B086BF3F
:10590000B17F79AB66D2997DAB66D66379C0B0863C
:10591000BFB17F79AA64D3997DAA64D76379C0B0F7
:1059200086BFB17F79AA62D5997DAA62D96379C011
:10593000B086BFB17F79AA5FD6997DAA5FDA637915
:10594000C0B086BFB17F79A95DD8997DA95DDC63C0
:1059500079C0B086BFB17F79A95ADA997DA95ADE9C
:105960006379C0B086BFB17F000000000000000076
:105970000000030303030303030000000000000012
:105980000000000303030303030300000000000002
:1059900000000000030303030303030000000000F2
:1059A00000000000000303030303030300000000E2
:1059B00000000000000003030303030303000000D2
:1059C00000000000000000030303030303030000C2
:1059D00000000000000000000303030303030300B2
:1059E00000000000000000000003030303030303A2
:1059F0000000000000000000000003030303030395
:105A00000300000000000000000000030303030384
:105A10000303000000000000000000000303030374
:105A20000303030000000000000000000003030364
:105A30000303030300000000000000000000030354
:105A40000303030303000000000000000000000344
:105A50000303030303030000000000000000000034
:105A60000303030303030300000000000000000021
:105A70000003030303030303000000000000000011
:105A80000000030303030303030000000000000001
:105A900000000003030303030303000000000000F1
:105AA00000000000030303030303030000000000E1
:105AB00000000000000303030303030300000000D1
:105AC00000000000000003030303030303000000C1
:105AD00000000000000000030303030303030000B1
:105AE00000000000000000000303030303030300A1
:105AF0000000000000000000000303030303030391
:105B00000000000000000000000003030303030383
:105B10000300000000000000000000030303030373
:105B20000303000000000000000000000303030363
:105B30000303030000000000000000000003030353
:105B40000303030300000000000000000000030343
:105B50000303030303000000000000000000000333
:105B60000303030303030000000000000000000023
:105B70000303030303030300000000000000000010
:105B80000003030303030303000000000000000000
:105B900000000303030303030300000000000000F0
:105BA00000000003030303030303000000000000E0
:105BB00000000000030303030303030000000000D0
:105BC00000000000000303030303030300000000C0
:105BD00000000000000003030303030303000000B0
:105BE00000000000000000030303030303030000A0
:105BF0000000000000000000030303030303030090
:105C0000000000000000000000030303030303037F
:105C10000000000000000000000003030303030372
:105C20000300000000000000000000030303030362
:105C30000303000000000000000000000303030352
:105C40000303030000000000000000000003030342
:105C50000303030300000000000000000000030332
:105C60000303030303000000000000000000000322
:105C70000303030303030000000000000000000012
:105C800003030303030303000000000000000000FF
:105C900000030303030303030000000000000000EF
:105CA00000000303030303030300000000000000DF
:105CB00000000003030303030303020202020202C3
:105CC00002020202030303030303000202020202B0
:105CD00002020202020303030303030002020202A0
:105CE0000202020202020303030303030002020290
:105CF0000202020202020203030303030300020280
:105D0000020202020202020203030303030300026F
:105D1000020202020202020202030303030303005F
:105D2000020202020202020202020303030303034D
:105D30000002020202020202020202030303030340
:105D40000300020202020202020202020303030330
:105D50000303000202020202020202020203030320
:105D60000303030079A95ADA997DA95ADE6379C041
:105D7000B086BFB17F79A95ADA997DA95ADE6379D5
:105D8000C0B086BFB17F79A95ADA997DA95ADE637E
:105D900079C0B086BFB17F79A95ADA997DA95ADE58
:105DA0006379C0B086BFB17F79A95ADA997DA95AC3
:105DB000DE6379C0B086BFB17F79A95ADA997DA92F
:105DC0005ADE6379C0B086BFB17F79A95ADA997D6E
:105DD000A95ADE6379C0B086BFB17F79A95ADA9932
:105DE0007DA95ADE6379C0B086BFB17F79A95ADA3E
:105DF000997DA95ADE6379C0B086BFB17F79A95A6F
:105E0000DA997DA95ADE6379C0B086BFB17F7AAADC
:105E100060D79A7EAA60DB6479C0B086BFB17F7B11
:105E2000AB64D49B80AB64D86679C0B086BFB17FC9
:105E30007CAC69D29C81AC69D66879C0B086BFB1B0
:105E40007F7EAD6DD09E83AD6DD46979C0B086BFC5
:105E5000B17F7FAE71CE9F84AE71D26B79C0B086B8
:105E6000BFB17F80AF74CCA086AF74D06D79C0B065
:105E700086BFB17F82B077CAA287B077CE6F79C074
:105E8000B086BFB17F83B17BC8A389B17BCC707969
:105E9000C0B086BFB17F84B17EC6A48AB17ECA720B
:105EA00079C0B086BFB17F86B281C5A68CB281C9E8
:105EB0007479C0B086BFB17F87B384C3A78DB38424
:105EC000C77579C0B086BFB17F88B387C2A88FB3CA
:105ED00087C67779C0B086BFB17F89B489C0A990E1
:105EE000B489C47979C0B086BFB17F8BB58CBFABA4
:105EF00092B58CC37B79C0B086BFB17F8CB58EBDA7
:105F0000AC93B58EC17C79C0B086BFB17F8DB691A0
:105F1000BCAD95B691C07E79C0B086BFB17F8FB65B
:105F200093BAAF97B693BE8079C0B086BFB17F9069
:105F3000B796B9B098B796BD8179C0B086BFB17F2A
:105F400091B898B8B19AB898BC8379C0B086BFB1FF
:105F50007F93B89BB6B39BB89BBA8579C0B086BF18
:105F6000B17F93B89BB6B39BBCA5B88579C0B0860A
:105F7000BFB17F93B89BB6B39BC0AEB58579C0B0B7
:105F800086BFB17F93B89BB6B39BC3B6B48579C0C7
:105F9000B086BFB17F93B89BB6B39BC7BEB38579BC
:105FA000C0B086BFB17F93B89BB6B39BC8C5B3855D
:105FB00079C0B086BFB17F93B89BB6B39BC8BCBA5B
:105FC0008579C0B086BFB17F93B89BB6B39BC8B28A
:105FD000C28579C0B086BFB17F93B89BB6B39BC76B
:105FE000A7CA8579C0B086BFB17F93B89BB6B39B73
:105FF000C59BD38579C0B086BFB17F93B89BB6B33C
:106000009BC38EDC8579C0B086BFB17F03020202DC
:106010000303020202030303030303030203020256
:106020000203030202020303030303030302030246
:106030000202030302020203030303030303020336
:106040000202020303020202030303030303030227
:106050000302020203030202020303030303030316
:106060000203020202030302020203030303030307
:1060700003020302020203030202020303030303F7
:1060800003030203020202030302020203030303E7
:1060900003030302030202020303020202030303D7
:1060A00003030303020302020203030202020303C7
:1060B00003030303030200000000000000000000CF
:1060C00003030303030302000000000000000000BC
:1060D00000030303030303020000000000000000AC
:1060E000000003030303030302000000000000009C
:1060F000000000030303030303020000000000008C
:10610000000000000303030303030200000000007B
:10611000000000000003030303030302000000006B
:10612000000000000000030303030303020000005B
:10613000000000000000000303030303030200004B
:10614000000000000000000003030303030302003B
:10615000000000000000000000030303030303022B
:10616000000000000000000000000303030303031D
:10617000020000000000000000000003030303030E
:1061800003020000000000000000000003030303FE
:1061900003030200000000000000000000030303EE
:1061A00003030302000000000000000000000303DE
:1061B00003030303020000000000000000000003CE
:1061C00003030303030200000000000000000000BE
:1061D00003030303030302000000000000000000AB
:1061E000000303030303030200000000000000009B
:1061F000000003030303030302000000000000008B
:10620000000000030303030303020000000000007A
:10621000000000000303030303030200000000006A
:10622000000000000003030303030302000000005A
:10623000000000000000030303030303020000004A
:10624000000000000000000303030303030200003A
:10625000000000000000000003030303030302002A
:10626000000000000000000000030303030303021A
:10627000000000000000000000000303030303030C
:1062800002000000000000000000000303030303FD
:1062900003020000000000000000000003030303ED
:1062A00003030200000000000000000000030303DD
:1062B0000303030290B79AB5B098C28FDA8279C00F
:1062C000B086BFB17F8DB79AB4AD95C290D87F79B3
:1062D000C0B086BFB17F8AB69AB3AA93C291D67B6B
:1062E00079C0B086BFB17F87B59AB1A790C192D46B
:1062F0007879C0B086BFB17F84B49AB0A48DC193C1
:10630000D27579C0B086BFB17F82B499AFA28AC07E
:1063100094D07279C0B086BFB17F7FB399AE9F87AA
:10632000C095CF6F79C0B086BFB17F7CB299AD9C6C
:1063300084BF96CD6B79C0B086BFB17F79B198AC80
:106340009982BF97CB6879C0B086BFB17F76B0978E
:10635000AB967FBE97CA6579C0B086BFB17F73B078
:1063600097AA937CBE98C86279C0B086BFB17F718E
:10637000AF96A99079BD99C65F79C0B086BFB17F4D
:106380006EAE95A88C76BD99C55C79C0B086BFB15C
:106390007F6BAD94A78973BC99C35979C0B086BF90
:1063A000B17F68AC93A78671BB9AC25779C0B0869B
:1063B000BFB17F65AB92A6836EBB9AC05479C0B063
:1063C00086BFB17F62AA91A5806BBA9ABF5179C08E
:1063D000B086BFB17F60A990A57C68B99ABD4E799F
:1063E000C0B086BFB17F5DA88FA47965B99ABC4B58
:1063F00079C0B086BFB17F5AA88EA47662B89BBA26
:106400004879C0B086BFB17F5AAD9D9F7662B89B78
:10641000BA4879C0B086BFB17F5AB3AA9C7662B839
:106420009BBA4879C0B086BFB17F5AB8B59B766237
:10643000B89BBA4879C0B086BFB17F5ABDBF9B76C2
:1064400062B89BBA4879C0B086BFB17F5AC2C89CB7
:106450007662B89BBA4879C0B086BFB17F5AC4BFD4
:10646000A87662B89BBA4879C0B086BFB17F5AC5DA
:10647000B5B37662B89BBA4879C0B086BFB17F5ACF
:10648000C5AABF7662B89BBA4879C0B086BFB17F53
:106490005AC49DCB7662B89BBA4879C0B086BFB16A
:1064A0007F5AC38ED87662B89BBA4879C0B086BF8F
:1064B000B17F5DC28FD67965B79AB94B79C0B08686
:1064C000BFB17F60C290D47C68B79AB84E79C0B033
:1064D00086BFB17F62C291D2806BB69AB75179C044
:1064E000B086BFB17F65C192D0836EB59AB554793D
:1064F000C0B086BFB17F68C193CE8671B49AB457DD
:1065000079C0B086BFB17F6BC094CC8973B499B3A6
:106510005979C0B086BFB17F6EC095CB8C76B399E8
:10652000B25C79C0B086BFB17F71BF96C99079B2B5
:1065300099B15F79C0B086BFB17F73BF97C7937CB5
:10654000B198B06279C0B086BFB17F76BE97C6966B
:106550007FB097AF6579C0B086BFB17F79BE98C470
:106560009982B097AE6879C0B086BFB17F7CBD9983
:10657000C29C84AF96AD6B79C0B086BFB17F7FBD42
:1065800099C19F87AE95AC6F79C0B086BFB17F824D
:10659000BC99BFA28AAD94AB7279C0B086BFB17FFF
:1065A00084BB9ABEA48DAC93AB7579C0B086BFB1E5
:1065B0007F87BB9ABCA790AB92AA7879C0B086BF00
:1065C000B17F8ABA9ABBAA93AA91A97B79C0B086F7
:1065D000BFB17F8DB99AB9AD95A990A97F79C0B0A7
:1065E00086BFB17F90B99AB8B098A88FA88279C0B9
:1065F000B086BFB17F93B89BB6B39BA88EA88579B0
:10660000C0B086BFB17F93B89BB6B39BAD9DA38549
:1066100079C0B086BFB17F93B89BB6B39BB3AAA035
:106620008579C0B086BFB17F93B89BB6B39BB8B530
:106630009F8579C0B086BFB17F93B89BB6B39BBD31
:10664000BF9F8579C0B086BFB17F93B89BB6B39B1F
:10665000C2C8A08579C0B086BFB17F93B89BB6B3DE
:106660009BC4BFAC8579C0B086BFB17F93B89BB6E1
:10667000B39BC5B5B78579C0B086BFB17F93B89BD2
:10668000B6B39BC5AAC38579C0B086BFB17F93B8A6
:106690009BB6B39BC49DCF8579C0B086BFB17F93B5
:1066A000B89BB6B39BC38EDC8579C0B086BFB17F83
:1066B00000000000000000000000030303030303C8
:1066C00003000000000000000000000303030303B8
:1066D00003030000000000000000000003030303A8
:1066E0000303030000000000000000000003030398
:1066F0000303030300000000000000000000030388
:106700000303030303000000000000000000000377
:106710000303030303030000000000000000000067
:106720000303030303030300000000000000000054
:106730000003030303030303000000000000000044
:106740000000030303030303030000000000000034
:106750000000000303030303030300000000000024
:106760000000000003030303030303000000000014
:106770000000000000030303030303030000000004
:1067800000000000000003030303030303000000F4
:1067900000000000000000030303030303030000E4
:1067A00000000000000000000303030303030300D4
:1067B00000000000000000000003030303030303C4
:1067C00000000000000000000000030303030303B7
:1067D00003000000000000000000000303030303A7
:1067E0000303000000000000000000000303030397
:1067F0000303030000000000000000000003030387
:106800000303030300000000000000000000030376
:106810000303030303000000000000000000000366
:106820000303030303030000000000000000000056
:106830000303030303030300000000000000000043
:106840000003030303030303000000000000000033
:106850000000030303030303030000000000000023
:106860000000000303030303030300000000000013
:106870000000000003030303030303000000000003
:1068800000000000000303030303030300000000F3
:1068900000000000000003030303030303000000E3
:1068A00000000000000000030303030303030000D3
:1068B00000000000000000000303030303030300C3
:1068C00000000000000000000003030303030303B3
:1068D00000000000000000000000030303030303A6
:1068E0000300000000000000000000030303030396
:1068F0000303000000000000000000000303030386
:106900000303030000000000000000000003030375
:106910000303030300000000000000000000030365
:106920000303030303000000000000000000000355
:106930000303030303030000000000000000000045
:106940000303030303030300000000000000000032
:106950000003030303030303000000000000000022
:106960000000030303030303030000000000000012
:106970000000000303030303030300000000000002
:1069800000000000030303030303030000000000F2
:1069900000000000000303030303030300000000E2
:1069A00000000000000003030303030303000000D2
:1069B00000000000000000030303030303030000C2
:1069C00000000000000000000303030303030300B2
:1069D00000000000000000000003030303030303A2
:1069E0000000000000000000000003030303030395
:1069F0000300000000000000000000030303030385
:106A00000303000000000000000000000303030374
:106A10000303030000000000000000000003030364
:106A20000303030300000000000000000000030354
:106A30000303030303000000000000000000000344
:106A40000303030303030000000000000000000034
:106A50000303030303030300000000000000000021
:106A60000003030303030303000000000000000011
:106A70000000030303030303030000000000000001
:106A800000000003030303030303000000000000F1
:106A900000000000030303030303030000000000E1
:106AA00000000000000303030303030390B79AB53B
:106AB000B098C28FDA8279C0B086BFB17F8DB79AA5
:106AC000B4AD95C290D87F79C0B086BFB17F8AB689
:106AD0009AB3AA93C291D67B79C0B086BFB17F87A3
:106AE000B59AB1A790C192D47879C0B086BFB17F72
:106AF00084B49AB0A48DC193D27579C0B086BFB169
:106B00007F82B499AFA28AC094D07279C0B086BF98
:106B1000B17F7FB399AE9F87C095CF6F79C0B086A4
:106B2000BFB17F7CB299AD9C84BF96CD6B79C0B06C
:106B300086BFB17F79B198AC9982BF97CB6879C095
:106B4000B086BFB17F76B097AB967FBE97CA6579A6
:106B5000C0B086BFB17F73B097AA937CBE98C8625D
:106B600079C0B086BFB17F71AF96A99079BD99C643
:106B70005F79C0B086BFB17F6EAE95A88C76BD99A7
:106B8000C55C79C0B086BFB17F6BAD94A78973BC7B
:106B900099C35979C0B086BFB17F68AC93A786719D
:106BA000BB9AC25779C0B086BFB17F65AB92A6834E
:106BB0006EBB9AC05479C0B086BFB17F62AA91A55E
:106BC000806BBA9ABF5179C0B086BFB17F60A9907F
:106BD000A57C68B99ABD4E79C0B086BFB17F5DA86B
:106BE0008FA47965B99ABC4B79C0B086BFB17F5A82
:106BF000A88EA47662B89BBA4879C0B086BFB17F30
:106C00005AAB9B9E7662B89BBA4879C0B086BFB13A
:106C10007F5AAFA7997662B89BBA4879C0B086BF51
:106C2000B17F5AB2B2947662B89BBA4879C0B08646
:106C3000BFB17F5AB6BC917662B89BBA4879C0B0F2
:106C400086BFB17F5AB9C58D7662B89BBA4879C004
:106C5000B086BFB17F5AB9BE957662B89BBA487903
:106C6000C0B086BFB17F5ABAB69E7662B89BBA48AA
:106C700079C0B086BFB17F5AB9AEA67662B89BBA6A
:106C80004879C0B086BFB17F5AB9A5AE7662B89BCD
:106C9000BA4879C0B086BFB17F5AB89BB67662B8A1
:106CA0009BBA4879C0B086BFB17F5BB899B77763AC
:106CB000B899BB4979C0B086BFB17F5CB797B87847
:106CC00064B797BC4A79C0B086BFB17F5DB796B94B
:106CD0007A65B796BD4B79C0B086BFB17F5EB79479
:106CE000BA7B66B794BE4C79C0B086BFB17F5FB641
:106CF00093BB7C67B693BF4D79C0B086BFB17F6050
:106D0000B691BC7D68B691C04E79C0B086BFB17FE8
:106D100061B58FBD7E69B58FC14F79C0B086BFB1F7
:106D20007F62B58EBE7F69B58EC24F79C0B086BF17
:106D3000B17F63B58CBF806AB58CC35079C0B08613
:106D4000BFB17F64B48AC0826BB48AC45179C0B0C9
:106D500086BFB17F65B488C1836CB488C55279C0E1
:106D6000B086BFB17F66B387C2846DB387C65379DF
:106D7000C0B086BFB17F67B385C3856EB385C75486
:106D800079C0B086BFB17F68B383C4866FB383C850
:106D90005579C0B086BFB17F69B281C5876FB281B6
:106DA000C95579C0B086BFB17F6AB27FC68870B25C
:106DB0007FCA5679C0B086BFB17F6BB17DC78A717B
:106DC000B17DCB5779C0B086BFB17F6CB17BC88B2A
:106DD00072B17BCC5879C0B086BFB17F6DB079C934
:106DE0008C73B079CD5979C0B086BFB17F6EB07663
:106DF000CB8D74B076CF5A79C0B086BFB17F6FAFFC
:106E000074CC8E75AF74D05B79C0B086BFB17F7023
:106E1000AF72CD8F76AF72D15C79C0B086BFB17FD3
:106E200071AE6FCE9076AE6FD25C79C0B086BFB1D6
:106E30007F72AD6DD09277AD6DD45D79C0B086BFF5
:106E4000B17F73AD6AD19378AD6AD55E79C0B086F3
:106E5000BFB17F74AC67D39479AC67D75F79C0B0AA
:106E600086BFB17F75AB64D4957AAB64D86079C0C6
:106E7000B086BFB17F76AB61D6967BAB61DA6179C4
:106E8000C0B086BFB17F77AA5ED8977CAA5EDC626D
:106E900079C0B086BFB17F79A95ADA997DA95ADE47
:106EA0006379C0B086BFB17F000000000000000021
:106EB00000000303030303030300000000000000BD
:106EC00000000003030303030303000000000000AD
:106ED000000000000303030303030300000000009D
:106EE000000000000003030303030303000000008D
:106EF000000000000000030303030303030000007D
:106F0000000000000000000303030303030300006C
:106F1000000000000000000003030303030303005C
:106F2000000000000000000000030303030303034C
:106F3000000000000000000000000303030303033F
:106F4000030000000000000000000003030303032F
:106F5000030300000000000000000000030303031F
:106F6000030303000000000000000000000303030F
:106F700003030303000000000000000000000303FF
:106F800003030303030000000000000000000003EF
:106F900003030303030300000000000000000000DF
:106FA00003030303030303000000000000000000CC
:106FB00000030303030303030000000000000000BC
:106FC00000000303030303030300000000000000AC
:106FD000000000030303030303030000000000009C
:106FE000000000000303030303030300000000008C
:106FF000000000000003030303030303000000007C
:10700000000000000000030303030303030000006B
:10701000000000000000000303030303030300005B
:10702000000000000000000003030303030303004B
:10703000000000000000000000030303030303033B
:10704000000000000000000000000303030303032E
:10705000030000000000000000000003030303031E
:10706000030300000000000000000000030303030E
:1070700003030300000000000000000000030303FE
:1070800003030303000000000000000000000303EE
:1070900003030303030000000000000000000003DE
:1070A00003030303030300000000000000000000CE
:1070B00003030303030303000000000000000000BB
:1070C00000030303030303030000000000000000AB
:1070D000000003030303030303000000000000009B
:1070E000000000030303030303030000000000008B
:1070F000000000000303030303030300000000007B
:10710000000000000003030303030303000000006A
:10711000000000000000030303030303030000005A
:10712000000000000000000303030303030300004A
:10713000000000000000000003030303030303003A
:10714000000000000000000000030303030303032A
:10715000000000000000000000000303030303031D
:10716000030000000000000000000003030303030D
:1071700003030000000000000000000003030303FD
:1071800003030300000000000000000000030303ED
:1071900003030303000000000000000000000303DD
:1071A00003030303030000000000000000000003CD
:1071B00003030303030300000000000000000000BD
:1071C00003030303030303000000000000000000AA
:1071D000000303030303030300000000000000009A
:1071E000000003030303030303000000000000008A
:1071F000000000030303030303030000000000007A
:107200000000000003030303030303000000000069
:107210000000000000030303030303030000000059
:107220000000000000000303030303030300000049
:107230000000000000000003030303030303000039
:107240000000000000000000030303030303030029
:107250000000000000000000000303030303030319
:10726000000000000000000000000303030303030C
:1072700003000000000000000000000303030303FC
:1072800003030000000000000000000003030303EC
:1072900003030300000000000000000000030303DC
:1072A0000303030379A95ADA997DA95ADE6379C0E9
:1072B000B086BFB17F79A95ADA997DA95ADE637980
:1072C000C0B086BFB17F79A95ADA997DA95ADE6329
:1072D00079C0B086BFB17F79A95ADA997DA95ADE03
:1072E0006379C0B086BFB17F79A95ADA997DA95A6E
:1072F000DE6379C0B086BFB17F79A95ADA997DA9DA
:107300005ADE6379C0B086BFB17F79A95ADA997D18
:10731000A95ADE6379C0B086BFB17F79A95ADA99DC
:107320007DA95ADE6379C0B086BFB17F79A95ADAE8
:10733000997DA95ADE6379C0B086BFB17F79A95A19
:10734000DA997DA95ADE6379C0B086BFB17F7AAA87
:1073500060D79A7EAA60DB6479C0B086BFB17F7BBC
:10736000AB64D49B80AB64D86679C0B086BFB17F74
:107370007CAC69D29C81AC69D66879C0B086BFB15B
:107380007F7EAD6DD09E83AD6DD46979C0B086BF70
:10739000B17F7FAE71CE9F84AE71D26B79C0B08663
:1073A000BFB17F80AF74CCA086AF74D06D79C0B010
:1073B00086BFB17F82B077CAA287B077CE6F79C01F
:1073C000B086BFB17F83B17BC8A389B17BCC707914
:1073D000C0B086BFB17F84B17EC6A48AB17ECA72B6
:1073E00079C0B086BFB17F86B281C5A68CB281C993
:1073F0007479C0B086BFB17F87B384C3A78DB384CF
:10740000C77579C0B086BFB17F88B387C2A88FB374
:1074100087C67779C0B086BFB17F89B489C0A9908B
:10742000B489C47979C0B086BFB17F8BB58CBFAB4E
:1074300092B58CC37B79C0B086BFB17F8CB58EBD51
:10744000AC93B58EC17C79C0B086BFB17F8DB6914B
:10745000BCAD95B691C07E79C0B086BFB17F8FB606
:1074600093BAAF97B693BE8079C0B086BFB17F9014
:10747000B796B9B098B796BD8179C0B086BFB17FD5
:1074800091B898B8B19AB898BC8379C0B086BFB1AA
:107490007F93B89BB6B39BB89BBA8579C0B086BFC3
:1074A000B17F93B89BB6B39BB9A5B28579C0B086BE
:1074B000BFB17F93B89BB6B39BB9AEAA8579C0B074
:1074C00086BFB17F93B89BB6B39BBAB6A28579C08D
:1074D000B086BFB17F93B89BB6B39BB9BE9985798F
:1074E000C0B086BFB17F93B89BB6B39BB9C5918539
:1074F00079C0B086BFB17F93B89BB6B39BB6BC953D
:107500008579C0B086BFB17F93B89BB6B39BB2B24A
:10751000988579C0B086BFB17F93B89BB6B39BAF57
:10752000A79D8579C0B086BFB17F93B89BB6B39B4A
:10753000AB9BA28579C0B086BFB17F93B89BB6B331
:107540009BA88EA88579C0B086BFB17F03020202D6
:107550000303020202030303030303030203020201
:1075600002030302020203030303030303020302F1
:1075700002020303020202030303030303030203E1
:1075800002020203030202020303030303030302D2
:1075900003020202030302020203030303030303C1
:1075A00002030202020303020202030303030303B2
:1075B00003020302020203030202020303030303A2
:1075C0000303020302020203030202020303030392
:1075D0000303030203020202030302020203030382
:1075E0000303030302030202020303020202030372
:1075F000030303030302000000000000000000007A
:107600000303030303030200000000000000000066
:107610000003030303030302000000000000000056
:107620000000030303030303020000000000000046
:107630000000000303030303030200000000000036
:107640000000000003030303030302000000000026
:107650000000000000030303030303020000000016
:107660000000000000000303030303030200000006
:1076700000000000000000030303030303020000F6
:1076800000000000000000000303030303030200E6
:1076900000000000000000000003030303030302D6
:1076A00000000000000000000000030303030303C8
:1076B00002000000000000000000000303030303B9
:1076C00003020000000000000000000003030303A9
:1076D0000303020000000000000000000003030399
:1076E0000303030200000000000000000000030389
:1076F0000303030302000000000000000000000379
:107700000303030303020000000000000000000068
:107710000303030303030200000000000000000055
:107720000003030303030302000000000000000045
:107730000000030303030303020000000000000035
:107740000000000303030303030200000000000025
:107750000000000003030303030302000000000015
:107760000000000000030303030303020000000005
:1077700000000000000003030303030302000000F5
:1077800000000000000000030303030303020000E5
:1077900000000000000000000303030303030200D5
:1077A00000000000000000000003030303030302C5
:1077B00000000000000000000000030303030303B7
:1077C00002000000000000000000000303030303A8
:1077D0000302000000000000000000000303030398
:1077E0000303020000000000000000000003030388
:1077F0000303030290B99AB8B098A88FA88279C001
:10780000B086BFB17F8DB99AB9AD95A990A97F799E
:10781000C0B086BFB17F8ABA9ABBAA93AA91A97B4E
:1078200079C0B086BFB17F87BB9ABCA790AB92AA44
:107830007879C0B086BFB17F84BB9ABEA48DAC936B
:10784000AB7579C0B086BFB17F82BC99BFA28AAD4B
:1078500094AB7279C0B086BFB17F7FBD99C19F875D
:10786000AE95AC6F79C0B086BFB17F7CBD99C29C2C
:1078700084AF96AD6B79C0B086BFB17F79BE98C436
:107880009982B097AE6879C0B086BFB17F76BE9757
:10789000C6967FB097AF6579C0B086BFB17F73BF22
:1078A00097C7937CB198B06279C0B086BFB17F7141
:1078B000BF96C99079B299B15F79C0B086BFB17FE8
:1078C0006EC095CB8C76B399B25C79C0B086BFB1EF
:1078D0007F6BC094CC8973B499B35979C0B086BF1B
:1078E000B17F68C193CE8671B49AB45779C0B0861F
:1078F000BFB17F65C192D0836EB59AB55479C0B0DF
:1079000086BFB17F62C291D2806BB69AB75179C0FF
:10791000B086BFB17F60C290D47C68B79AB84E7908
:10792000C0B086BFB17F5DC28FD67965B79AB94BBB
:1079300079C0B086BFB17F5AC38ED87662B89BBA81
:107940004879C0B086BFB17F5AC49DCB7662B89BE0
:10795000BA4879C0B086BFB17F5AC5AABF7662B8AF
:107960009BBA4879C0B086BFB17F5AC5B5B37662BD
:10797000B89BBA4879C0B086BFB17F5AC4BFA87659
:1079800062B89BBA4879C0B086BFB17F5AC2C89C62
:107990007662B89BBA4879C0B086BFB17F5ABDBF86
:1079A0009B7662B89BBA4879C0B086BFB17F5AB89F
:1079B000B59B7662B89BBA4879C0B086BFB17F5A92
:1079C000B3AA9C7662B89BBA4879C0B086BFB17F33
:1079D0005AAD9D9F7662B89BBA4879C0B086BFB158
:1079E0007F5AA88EA47662B89BBA4879C0B086BF89
:1079F000B17F5DA88FA47965B99ABC4B79C0B08678
:107A0000BFB17F60A990A57C68B99ABD4E79C0B01E
:107A100086BFB17F62AA91A5806BBA9ABF5179C027
:107A2000B086BFB17F65AB92A6836EBB9AC0547916
:107A3000C0B086BFB17F68AC93A78671BB9AC257AE
:107A400079C0B086BFB17F6BAD94A78973BC99C371
:107A50005979C0B086BFB17F6EAE95A88C76BD99BE
:107A6000C55C79C0B086BFB17F71AF96A99079BD72
:107A700099C65F79C0B086BFB17F73B097AA937C77
:107A8000BE98C86279C0B086BFB17F76B097AB961A
:107A90007FBE97CA6579C0B086BFB17F79B198AC17
:107AA0009982BF97CB6879C0B086BFB17F7CB2990D
:107AB000AD9C84BF96CD6B79C0B086BFB17F7FB3DC
:107AC00099AE9F87C095CF6F79C0B086BFB17F82D6
:107AD000B499AFA28AC094D07279C0B086BFB17F8A
:107AE00084B49AB0A48DC193D27579C0B086BFB169
:107AF0007F87B59AB1A790C192D47879C0B086BF7C
:107B0000B17F8AB69AB3AA93C291D67B79C0B08668
:107B1000BFB17F8DB79AB4AD95C290D87F79C0B010
:107B200086BFB17F90B79AB5B098C28FDA8279C01C
:107B3000B086BFB17F93B89BB6B39BC38EDC85790B
:107B4000C0B086BFB17F93B89BB6B39BC49DCF85B1
:107B500079C0B086BFB17F93B89BB6B39BC5AAC3AB
:107B60008579C0B086BFB17F93B89BB6B39BC5B5CE
:107B7000B78579C0B086BFB17F93B89BB6B39BC4BD
:107B8000BFAC8579C0B086BFB17F93B89BB6B39BBD
:107B9000C2C8A08579C0B086BFB17F93B89BB6B389
:107BA0009BBDBF9F8579C0B086BFB17F93B89BB6A0
:107BB000B39BB8B59F8579C0B086BFB17F93B89BA2
:107BC000B6B39BB3AAA08579C0B086BFB17F93B886
:107BD0009BB6B39BAD9DA38579C0B086BFB17F93A3
:107BE000B89BB6B39BA88EA88579C0B086BFB17F7D
:107BF0000000000000000000000003030303030373
:107C00000300000000000000000000030303030362
:107C10000303000000000000000000000303030352
:107C20000303030000000000000000000003030342
:107C30000303030300000000000000000000030332
:107C40000303030303000000000000000000000322
:107C50000303030303030000000000000000000012
:107C600003030303030303000000000000000000FF
:107C700000030303030303030000000000000000EF
:107C800000000303030303030300000000000000DF
:107C900000000003030303030303000000000000CF
:107CA00000000000030303030303030000000000BF
:107CB00000000000000303030303030300000000AF
:107CC000000000000000030303030303030000009F
:107CD000000000000000000303030303030300008F
:107CE000000000000000000003030303030303007F
:107CF000000000000000000000030303030303036F
:107D00000000000000000000000003030303030361
:107D10000300000000000000000000030303030351
:107D20000303000000000000000000000303030341
:107D30000303030000000000000000000003030331
:107D40000303030300000000000000000000030321
:107D50000303030303000000000000000000000311
:107D60000303030303030000000000000000000001
:107D700003030303030303000000000000000000EE
:107D800000030303030303030000000000000000DE
:107D900000000303030303030300000000000000CE
:107DA00000000003030303030303000000000000BE
:107DB00000000000030303030303030000000000AE
:107DC000000000000003030303030303000000009E
:107DD000000000000000030303030303030000008E
:107DE000000000000000000303030303030300007E
:107DF000000000000000000003030303030303006E
:107E0000000000000000000000030303030303035D
:107E10000000000000000000000003030303030350
:107E20000300000000000000000000030303030340
:107E30000303000000000000000000000303030330
:107E40000303030000000000000000000003030320
:107E50000303030300000000000000000000030310
:107E60000303030303000000000000000000000300
:107E700003030303030300000000000000000000F0
:107E800003030303030303000000000000000000DD
:107E900000030303030303030000000000000000CD
:107EA00000000303030303030300000000000000BD
:107EB00000000003030303030303000000000000AD
:107EC000000000000303030303030300000000009D
:107ED000000000000003030303030303000000008D
:107EE000000000000000030303030303030000007D
:107EF000000000000000000303030303030300006D
:107F0000000000000000000003030303030303005C
:107F1000000000000000000000030303030303034C
:107F2000000000000000000000000303030303033F
:107F3000030000000000000000000003030303032F
:107F4000030300000000000000000000030303031F
:107F5000030303000000000000000000000303030F
:107F600003030303000000000000000000000303FF
:107F700003030303030000000000000000000003EF
:107F800003030303030300000000000000000000DF
:107F900003030303030303000000000000000000CC
:107FA00000030303030303030000000000000000BC
:107FB00000000303030303030300000000000000AC
:107FC000000000030303030303030000000000009C
:107FD000000000000303030303030300000000008C
:107FE00000000000000303030303030390B99AB8E1
:107FF000B098A88FA88279C0B086BFB17F8DB99A9A
:10800000B9AD95A990A97F79C0B086BFB17F8ABA72
:108010009ABBAA93AA91A97B79C0B086BFB17F878A
:10802000BB9ABCA790AB92AA7879C0B086BFB17F4B
:1080300084BB9ABEA48DAC93AB7579C0B086BFB13A
:108040007F82BC99BFA28AAD94AB7279C0B086BF63
:10805000B17F7FBD99C19F87AE95AC6F79C0B08667
:10806000BFB17F7CBD99C29C84AF96AD6B79C0B027
:1080700086BFB17F79BE98C49982B097AE6879C047
:10808000B086BFB17F76BE97C6967FB097AF657951
:10809000C0B086BFB17F73BF97C7937CB198B06201
:1080A00079C0B086BFB17F71BF96C99079B299B1DE
:1080B0005F79C0B086BFB17F6EC095CB8C76B39927
:1080C000B25C79C0B086BFB17F6BC094CC8973B409
:1080D00099B35979C0B086BFB17F68C193CE86711C
:1080E000B49AB45779C0B086BFB17F65C192D083CE
:1080F0006EB59AB55479C0B086BFB17F62C291D2D5
:10810000806BB69AB75179C0B086BFB17F60C2901C
:10811000D47C68B79AB84E79C0B086BFB17F5DC2D3
:108120008FD67965B79AB94B79C0B086BFB17F5AFF
:10813000C38ED87662B89BBA4879C0B086BFB17F8B
:108140005AC59BCF7662B89BBA4879C0B086BFB19A
:108150007F5AC7A7C67662B89BBA4879C0B086BFB7
:10816000B17F5AC8B2BE7662B89BBA4879C0B086B1
:10817000BFB17F5AC8BCB67662B89BBA4879C0B066
:1081800086BFB17F5AC8C5AF7662B89BBA4879C07E
:10819000B086BFB17F5AC7BEAF7662B89BBA487986
:1081A000C0B086BFB17F5AC3B6B07662B89BBA483A
:1081B00079C0B086BFB17F5AC0AEB17662B89BBA03
:1081C0004879C0B086BFB17F5ABCA5B47662B89B6F
:1081D000BA4879C0B086BFB17F5AB89BB67662B84C
:1081E0009BBA4879C0B086BFB17F5BB899B7776357
:1081F000B899BB4979C0B086BFB17F5CB797B878F2
:1082000064B797BC4A79C0B086BFB17F5DB796B9F5
:108210007A65B796BD4B79C0B086BFB17F5EB79423
:10822000BA7B66B794BE4C79C0B086BFB17F5FB6EB
:1082300093BB7C67B693BF4D79C0B086BFB17F60FA
:10824000B691BC7D68B691C04E79C0B086BFB17F93
:1082500061B58FBD7E69B58FC14F79C0B086BFB1A2
:108260007F62B58EBE7F69B58EC24F79C0B086BFC2
:10827000B17F63B58CBF806AB58CC35079C0B086BE
:10828000BFB17F64B48AC0826BB48AC45179C0B074
:1082900086BFB17F65B488C1836CB488C55279C08C
:1082A000B086BFB17F66B387C2846DB387C653798A
:1082B000C0B086BFB17F67B385C3856EB385C75431
:1082C00079C0B086BFB17F68B383C4866FB383C8FB
:1082D0005579C0B086BFB17F69B281C5876FB28161
:1082E000C95579C0B086BFB17F6AB27FC68870B207
:1082F0007FCA5679C0B086BFB17F6BB17DC78A7126
:10830000B17DCB5779C0B086BFB17F6CB17BC88BD4
:1083100072B17BCC5879C0B086BFB17F6DB079C9DE
:108320008C73B079CD5979C0B086BFB17F6EB0760D
:10833000CB8D74B076CF5A79C0B086BFB17F6FAFA6
:1083400074CC8E75AF74D05B79C0B086BFB17F70CE
:10835000AF72CD8F76AF72D15C79C0B086BFB17F7E
:1083600071AE6FCE9076AE6FD25C79C0B086BFB181
:108370007F72AD6DD09277AD6DD45D79C0B086BFA0
:10838000B17F73AD6AD19378AD6AD55E79C0B0869E
:10839000BFB17F74AC67D39479AC67D75F79C0B055
:1083A00086BFB17F75AB64D4957AAB64D86079C071
:1083B000B086BFB17F76AB61D6967BAB61DA61796F
:1083C000C0B086BFB17F77AA5ED8977CAA5EDC6218
:1083D00079C0B086BFB17F79A95ADA997DA95ADEF2
:1083E0006379C0B086BFB17F0000000000000000CC
:1083F0000000030303030303030000000000000068
:108400000000000303030303030300000000000057
:108410000000000003030303030303000000000047
:108420000000000000030303030303030000000037
:108430000000000000000303030303030300000027
:108440000000000000000003030303030303000017
:108450000000000000000000030303030303030007
:1084600000000000000000000003030303030303F7
:1084700000000000000000000000030303030303EA
:1084800003000000000000000000000303030303DA
:1084900003030000000000000000000003030303CA
:1084A00003030300000000000000000000030303BA
:1084B00003030303000000000000000000000303AA
:1084C000030303030300000000000000000000039A
:1084D000030303030303000000000000000000008A
:1084E0000303030303030300000000000000000077
:1084F0000003030303030303000000000000000067
:108500000000030303030303030000000000000056
:108510000000000303030303030300000000000046
:108520000000000003030303030303000000000036
:108530000000000000030303030303030000000026
:108540000000000000000303030303030300000016
:108550000000000000000003030303030303000006
:1085600000000000000000000303030303030300F6
:1085700000000000000000000003030303030303E6
:1085800000000000000000000000030303030303D9
:1085900003000000000000000000000303030303C9
:1085A00003030000000000000000000003030303B9
:1085B00003030300000000000000000000030303A9
:1085C0000303030300000000000000000000030399
:1085D0000303030303000000000000000000000389
:1085E0000303030303030000000000000000000079
:1085F0000303030303030300000000000000000066
:108600000003030303030303000000000000000055
:108610000000030303030303030000000000000045
:108620000000000303030303030300000000000035
:108630000000000003030303030303000000000025
:108640000000000000030303030303030000000015
:108650000000000000000303030303030300000005
:1086600000000000000000030303030303030000F5
:1086700000000000000000000303030303030300E5
:1086800000000000000000000003030303030303D5
:1086900000000000000000000000030303030303C8
:1086A00003000000000000000000000303030303B8
:1086B00003030000000000000000000003030303A8
:1086C0000303030000000000000000000003030398
:1086D0000303030300000000000000000000030388
:1086E0000303030303000000000000000000000378
:1086F0000303030303030000000000000000000068
:108700000303030303030300000000000000000054
:108710000003030303030303000000000000000044
:108720000000030303030303030000000000000034
:108730000000000303030303030300000000000024
:108740000000000003030303030303000000000014
:108750000000000000030303030303030000000004
:1087600000000000000003030303030303000000F4
:1087700000000000000000030303030303030000E4
:1087800000000000000000000303030303030300D4
:1087900000000000000000000003030303030303C4
:1087A00000000000000000000000030303030303B7
:1087B00003000000000000000000000303030303A7
:1087C0000303000000000000000000000303030397
:1087D0000303030000000000000000000003030387
:1087E0000303030379A95CD9997DA95CDD6379C092
:1087F000B086BFB17F79AA5DD8997DAA5DDC637927
:10880000C0B086BFB17F79AA5ED8997DAA5EDC63CD
:1088100079C0B086BFB17F79AA5FD7997DAA5FDBA7
:108820006379C0B086BFB17F79AA60D7997DAA600D
:10883000DB6379C0B086BFB17F79AB62D6997DAB7F
:1088400062DA6379C0B086BFB17F79AB63D5997DB9
:10885000AB63D96379C0B086BFB17F79AB64D5997A
:108860007DAB64D96379C0B086BFB17F79AC65D484
:10887000997DAC65D86379C0B086BFB17F79AC66AD
:10888000D4997DAC66D86379C0B086BFB17F79AE2C
:1088900065D8997DAA65D46379C0B086BFB1837964
:1088A000AF64DD997DA764D16379C0B086BFB1861E
:1088B00079B161E2997DA461CF6379C0B086BFB11F
:1088C0008979B15CE8997DA15CCE6379C0B086BF3F
:1088D000B18C79B255F0997D9E55CE6379C0B08642
:1088E000BFB18F7AB257EE9A7E9E55CE6479C0B0F2
:1088F00086BFB18F7BB259EC9B809E55CE6679C006
:10890000B086BFB18F7CB25AEA9C829E55CE687900
:10891000C0B086BFB18F7DB15CE89D839E55CE6AA5
:1089200079C0B086BFB18F7FB15DE79F859E55CE80
:108930006C79C0B086BFB18F80B15EE5A0879E55CF
:10894000CE6E79C0B086BFB18F81B160E4A1889E40
:1089500055CE7079C0B086BFB18F82B161E2A28A74
:108960009E55CE7279C0B086BFB18F84B061E1A44C
:108970008C9E55CE7479C0B086BFB18F85B062DF52
:10898000A58D9E55CE7579C0B086BFB18F86B06378
:10899000DEA68F9E55CE7779C0B086BFB18F87AFE8
:1089A00064DDA7919E55CE7979C0B086BFB18F881E
:1089B000AF64DBA8929E55CE7B79C0B086BFB18FE5
:1089C0008AAE65DAAA949E55CE7D79C0B086BFB1D5
:1089D0008F8BAE65D9AB969E55CE7F79C0B086BFE2
:1089E000B18F8CAE65D8AC979E55CE8179C0B086DC
:1089F000BFB18F8DAD66D7AD999E55CE8379C0B08E
:108A000086BFB18F8FAD66D6AF9B9E55CE8579C0A0
:108A1000B086BFB18F90AC66D5B09C9E55CE86799E
:108A2000C0B086BFB18F91AC66D4B19E9E55CE8842
:108A300079C0B086BFB18F91AC66D4B19EA670C22A
:108A40008879C0B086BFB18F91AC66D4B19EAC823C
:108A5000BC8879C0B086BFB18F91AC66D4B19EB1ED
:108A600091B78879C0B086BFB18F91AC66D4B19E02
:108A7000B69DB58879C0B086BFB18F91AC66D4B1D0
:108A80009EBBA7B38879C0B086BFB18F91AC66D4C6
:108A9000B19EBB9DBE8879C0B086BFB18F91AC66D8
:108AA000D4B19EBA91C98879C0B086BFB18F91AC5C
:108AB00066D4B19EB982D48879C0B086BFB18F9197
:108AC000AC66D4B19EB770E28879C0B086BFB18F72
:108AD00091AC66D4B19EB255F48879C0B086BFB16E
:108AE0008F90AC66D4B09DB256F28779C0B086BF85
:108AF000B18F8FAC66D4AF9CB258F18679C0B08686
:108B0000BFB18E8FAC66D4AF9BB259F08579C0B03F
:108B100086BFB18E8EAC66D4AE9AB25AEF8379C05E
:108B2000B086BFB18D8DAC66D4AD99B25BEE827963
:108B3000C0B086BFB18D8CAC66D4AC97B15CEC8113
:108B400079C0B086BFB18C8BAC66D4AB96B15DEB0F
:108B50008079C0B086BFB18C8AAC66D4AA95B15E6C
:108B6000EA7E79C0B086BFB18B8AAC66D4AA94B1D4
:108B70005EE97D79C0B086BFB18B89AC66D4A9931C
:108B8000B15FE87C79C0B086BFB18A88AC66D4A8F2
:108B900092B160E77A79C0B086BFB18A87AC66D4FB
:108BA000A791B161E67979C0B086BFB18986AC661C
:108BB000D4A690B061E57879C0B086BFB18986ACA3
:108BC00066D4A68EB062E47779C0B086BFB18885DE
:108BD000AC66D4A58DB062E37579C0B086BFB187AD
:108BE00084AC66D4A48CB063E27479C0B086BFB1A3
:108BF0008783AC66D4A38BAF63E17379C0B086BFC3
:108C0000B18682AC66D4A28AAF64E17279C0B086C4
:108C1000BFB18681AC66D4A189AF64E07079C0B081
:108C200086BFB18581AC66D4A188AF64DF6F79C09F
:108C3000B086BFB18580AC66D4A087AE65DE6E79A4
:108C4000C0B086BFB1847FAC66D49F85AE65DD6D54
:108C500079C0B086BFB1847EAC66D49E84AE65DD3B
:108C60006B79C0B086BFB1837DAC66D49D83AE65A1
:108C7000DC6A79C0B086BFB1837DAC66D49D82AD1D
:108C800066DB6979C0B086BFB1827CAC66D49C815A
:108C9000AD66DA6879C0B086BFB1827BAC66D49B22
:108CA00080AD66DA6679C0B086BFB1817AAC66D431
:108CB0009A7FAC66D96579C0B086BFB18179AC6660
:108CC000D4997EAC66D86479C0B086BFB18079ACE7
:108CD00066D4997DAC66D86379C0B086BFB17F7920
:108CE000AC65D4997DAC65D86379C0B086BFB17FDF
:108CF00079AB64D5997DAB64D96379C0B086BFB1D7
:108D00007F79AB63D5997DAB63D96379C0B086BFFA
:108D1000B17F79AB62D6997DAB62DA6379C0B086F8
:108D2000BFB17F79AA60D7997DAA60DB6379C0B0B3
:108D300086BFB17F79AA5FD7997DAA5FDB6379C0CF
:108D4000B086BFB17F79AA5ED8997DAA5EDC6379CF
:108D5000C0B086BFB17F79AA5DD8997DAA5DDC637A
:108D600079C0B086BFB17F79A95CD9997DA95CDD56
:108D70006379C0B086BFB17F79A95ADA997DA95AC3
:108D8000DE6379C0B086BFB17F79A95ADA997DA92F
:108D90005ADE6379C0B086BFB17F79A95ADA997D6E
:108DA000A95ADE6379C0B086BFB17F79A95ADA9932
:108DB0007DA95ADE6379C0B086BFB17F79A95ADA3E
:108DC000997DA95ADE6379C0B086BFB17F79A95A6F
:108DD000DA997DA95ADE6379C0B086BFB17F0303FB
:108DE0000303030303030303030303030303030353
:108DF0000303030303030303030303030303030343
:108E00000303030303030303030303030303030332
:108E10000303030303030303030303030303030322
:108E20000303030303030303030303030303030312
:108E30000303030303030303030303030303030302
:108E400003030303030303030303030303030303F2
:108E500003030303030303030303030303030303E2
:108E600003030303030303030303030303030303D2
:108E700003030303030303030303030303030303C2
:108E800003030303030303030300000003030000C1
:108E900000030303030303030303000000030300B1
:108EA00000000303030303030303030000000303A1
:108EB0000000000303030303030303030000000394
:108EC0000300000003030303030303030300000084
:108ED0000303000000030303030303030300000074
:108EE000000000000000000303030303030300006D
:108EF000000000000000000003030303030303005D
:108F0000000000000000000000030303030303034C
:108F1000000000000000000000000303030303033F
:108F2000030000000000000000000003030303032F
:108F3000030300000000000000000000030303031F
:108F4000030303000000000000000000000303030F
:108F500003030303000000000000000000000303FF
:108F600003030303030000000000000000000003EF
:108F700003030303030300000000000000000000DF
:108F800003030303030303000000000000000000CC
:108F900000030303030303030000000000000000BC
:108FA00000000303030303030300000000000000AC
:108FB000000000030303030303030000000000009C
:108FC000000000000303030303030300000000008C
:108FD000000000000003030303030303000000007C
:108FE000000000000000030303030303030000006C
:108FF000000000000000000303030303030300005C
:10900000000000000000000003030303030303004B
:10901000000000000000000000030303030303033B
:10902000000000000000000000000303030303032E
:10903000030000000000000000000003030303031E
:10904000030300000000000000000000030303030E
:1090500003030300000000000000000000030303FE
:1090600003030303000000000000000000000303EE
:1090700003030303030000000000000000000003DE
:1090800003030303030300000000000000000000CE
:1090900003030303030303000000000000000000BB
:1090A00000030303030303030000000000000000AB
:1090B000000003030303030303000000000000009B
:1090C000000000030303030303030000000000008B
:1090D000000000000303030303030300000000007B
:1090E000000000000003030303030303000000006B
:1090F000000000000000030303030303030000005B
:10910000000000000000000303030303030300004A
:10911000000000000000000003030303030303003A
:10912000000000000000000000030303030303032A
:10913000000000000000000000000303030303031D
:10914000030000000000000000000003030303030D
:1091500003030000000000000000000003030303FD
:1091600003030300000000000000000000030303ED
:1091700003030303000000000000000000000303DD
:1091800003030303030000000000000000000003CD
:1091900003030303030300000000000000000000BD
:1091A00003030303030303000000000000000000AA
:1091B000000303030303030300000000000000009A
:1091C000000003030303030303000000000000008A
:1091D000000000030303030303030000000000007A
:1091E000000000000303030303030300000000006A
:1091F000000000000003030303030303000000005A
:109200000000000000000303030303030300000049
:109210000000000000000003030303030303000039
:109220000000000000000000030303030303030029
:109230000000000000000000000303030303030319
:10924000000000000000000000000303030303030C
:1092500003000000000000000000000303030303FC
:1092600003030000000000000000000003030303EC
:1092700003030300000000000000000000030303DC
:1092800003030303000000000000000000000303CC
:1092900003030303030000000000000000000003BC
:1092A00003030303030300000000000000000000AC
:1092B0000303030303030300000000000000000099
:1092C0000003030303030303000000000000000089
:1092D0000000030303030303030000000000000079
:1092E0000000000303030303030300000000000069
:1092F0000000000003030303030303000000000059
:109300000000000000030303030303030000000048
:109310000000000000000303030303030300000038
:109320000000000000000003030303030303000028
:109330000000000000000000030303030303030018
:109340000000000000000000000303030303030308
:1093500000000000000000000000030303030303FB
:1093600003000000000000000000000303030303EB
:1093700003030000000000000000000003030303DB
:1093800003030303020202030302020203030303B3
:1093900003030303030202020303020202030303A3
:1093A0000303030303030202020303020202030393
:1093B0000303030303030302020203030202020383
:1093C0000303030303030303020202030302020273
:1093D000030303030303030379A95ADA997DA95A06
:1093E000DE6379C0B086BFB17F79A95ADA997DA9C9
:1093F0005ADE6379C0B086BFB17F79A95ADA997D08
:10940000A95ADE6379C0B086BFB17F79A95ADA99CB
:109410007DA95ADE6379C0B086BFB17F79A95ADAD7
:10942000997DA95ADE6379C0B086BFB17F79A95A08
:10943000DA997DA95ADE6379C0B086BFB17F79A978
:109440005ADA997DA95ADE6379C0B086BFB17F79B7
:10945000A95ADA997DA95ADE6379C0B086BFB17F77
:1094600079A95ADA997DA95ADE6379C0B086BFB16D
:109470007F79A95ADA997DA95ADE6379C0B086BF8F
:10948000B17F7AA95ADA9A7FA95ADE6579C0B08687
:10949000BFB17F7CA95ADA9C82A95ADE6879C0B034
:1094A00086BFB17F7EA95ADA9E85A95ADE6B79C044
:1094B000B086BFB17F80A95ADAA088A95ADE6E793A
:1094C000C0B086BFB17F82A95ADAA28BA95ADE71D9
:1094D00079C0B086BFB17F84A95ADAA48EA95ADEBA
:1094E0007479C0B086BFB17F86A95ADAA691A95A0D
:1094F000DE7779C0B086BFB17F88A95ADAA894A96F
:109500005ADE7A79C0B086BFB17F8AA95ADAAA97A3
:10951000A95ADE7D79C0B086BFB17F8CA95ADAAC7A
:109520009AA95ADE8079C0B086BFB17F8CA95ADA79
:10953000AC9AAD6BD58079C0B086BFB17F8CA95A8B
:10954000DAAC9AB078CE8079C0B086BFB17F8CA9F2
:109550005ADAAC9AB383C88079C0B086BFB17F8C29
:10956000A95ADAAC9AB58CC28079C0B086BFB17FF7
:109570008CA95ADAAC9AB795BE8079C0B086BFB1D3
:109580007F8CA95ADAAC9BB691C08179C0B086BFF6
:10959000B17F8CA95ADAAC9DB58CC28379C0B086F4
:1095A000BFB17F8CA95ADAAC9EB488C58479C0B0AB
:1095B00086BFB17F8CA95ADAACA0B383C88679C0C4
:1095C000B086BFB17F8CA95ADAACA1B17DCB8879C6
:1095D000C0B086BFB17F8CA95ADAACA3B078CE896F
:1095E00079C0B086BFB17F8CA95ADAACA4AF72D172
:1095F0008B79C0B086BFB17F8CA95ADAACA6AD6BAF
:10960000D58C79C0B086BFB17F8CA95ADAACA7AB34
:1096100063D98E79C0B086BFB17F8CA95ADAACA964
:10962000A95ADE8F79C0B086BFB17F89A95ADAA95D
:10963000A6A95ADE8C79C0B086BFB17F86A95ADA56
:10964000A6A2A95ADE8979C0B086BFB17F83A95A84
:10965000DAA39FA95ADE8679C0B086BFB17F80A900
:109660005ADAA09CA95ADE8279C0B086BFB17F7D4C
:10967000A95ADA9D99A95ADE7F79C0B086BFB17F19
:109680007AA95ADA9A96A95ADE7C79C0B086BFB117
:109690007F78A95ADA9792A95ADE7979C0B086BF45
:1096A000B17F75A95ADA948FA95ADE7579C0B08650
:1096B000BFB17F72A95ADA918CA95ADE7279C0B013
:1096C00086BFB17F6FA95ADA8E89A95ADE6F79C039
:1096D000B086BFB17F6CA95ADA8B86A95ADE6C7945
:1096E000C0B086BFB17F69A95ADA8882A95ADE68FC
:1096F00079C0B086BFB17F66A95ADA857FA95ADEE4
:109700006579C0B086BFB17F63A95ADA827CA95A55
:10971000DE6279C0B086BFB17F60A95ADA7F79A9CD
:109720005ADE5F79C0B086BFB17F5DA95ADA7C7519
:10973000A95ADE5B79C0B086BFB17F5AA95ADA79DF
:1097400072A95ADE5879C0B086BFB17F57A95ADADC
:10975000766FA95ADE5579C0B086BFB17F54A95A39
:10976000DA736CA95ADE5279C0B086BFB17F51A9B5
:109770005ADA7069A95ADE4F79C0B086BFB17F54FA
:10978000AD6BD17369A95ADE4F79C0B086BFB17F86
:1097900057B078CA7769A95ADE4F79C0B086BFB191
:1097A0007F5AB383C47A69A95ADE4F79C0B086BFA5
:1097B000B17F5DB58CBE7D69A95ADE4F79C0B08698
:1097C000BFB17F60B795BA8069A95ADE4F79C0B042
:1097D00086BFB17F60B691BC8069A95ADE4F79C05F
:1097E000B086BFB17F60B58CBE8069A95ADE4F7963
:1097F000C0B086BFB17F60B488C18069A95ADE4F0E
:1098000079C0B086BFB17F60B383C48069A95ADED6
:109810004F79C0B086BFB17F60B17DC78069A95A5A
:10982000DE4F79C0B086BFB17F60B078CA8069A9C9
:109830005ADE4F79C0B086BFB17F60AF72CD80690C
:10984000A95ADE4F79C0B086BFB17F60AD6BD180C1
:1098500069A95ADE4F79C0B086BFB17F60AB63D5CE
:109860008069A95ADE4F79C0B086BFB17F60A95A1E
:10987000DA8069A95ADE4F79C0B086BFB17F61A98D
:109880005ADA816AA95ADE5079C0B086BFB17F62C8
:10989000A95ADA826BA95ADE5179C0B086BFB17F6E
:1098A00064A95ADA836CA95ADE5279C0B086BFB176
:1098B0007F65A95ADA856DA95ADE5379C0B086BF93
:1098C000B17F66A95ADA866EA95ADE5479C0B0868D
:1098D000BFB17F67A95ADA876FA95ADE5579C0B040
:1098E00086BFB17F69A95ADA8870A95ADE5679C055
:1098F000B086BFB17F6AA95ADA8A71A95ADE577950
:10990000C0B086BFB17F6BA95ADA8B72A95ADE58F4
:1099100079C0B086BFB17F6CA95ADA8C73A95ADEC0
:109920005979C0B086BFB17F6DA95ADA8D74A95A32
:10993000DE5A79C0B086BFB17F6FA95ADA8F75A998
:109940005ADE5B79C0B086BFB17F70A95ADA9076D3
:10995000A95ADE5C79C0B086BFB17F71A95ADA918D
:1099600077A95ADE5D79C0B086BFB17F72A95ADA95
:109970009278A95ADE5E79C0B086BFB17F74A95AC9
:10998000DA9479A95ADE5F79C0B086BFB17F75A934
:109990005ADA957AA95ADE6079C0B086BFB17F766F
:1099A000A95ADA967BA95ADE6179C0B086BFB17F29
:1099B00077A95ADA977CA95ADE6279C0B086BFB11E
:1099C0007F79A95ADA997DA95ADE6379C0B086BF3A
:1099D000B17F79A95ADA997DA95ADE6379C0B08638
:1099E000BFB17F79A95ADA997DA95ADE6379C0B0EF
:1099F00086BFB17F79A95ADA997DA95ADE6379C009
:109A0000B086BFB17F79A95ADA997DA95ADE637908
:109A1000C0B086BFB17F79A95ADA997DA95ADE63B1
:109A200079C0B086BFB17F79A95ADA997DA95ADE8B
:109A30006379C0B086BFB17F79A95ADA997DA95AF6
:109A4000DE6379C0B086BFB17F79A95ADA997DA962
:109A50005ADE6379C0B086BFB17F79A95ADA997DA1
:109A6000A95ADE6379C0B086BFB17F79A95ADA9965
:109A70007DA95ADE6379C0B086BFB17F79A95ADA71
:109A8000997DA95ADE6379C0B086BFB17F79A95AA2
:109A9000DA997DA95ADE6379C0B086BFB17F79A912
:109AA0005ADA997DA95ADE6379C0B086BFB17F7951
:109AB000A95ADA997DA95ADE6379C0B086BFB17F11
:109AC00079A95ADA997DA95ADE6379C0B086BFB107
:109AD0007F000000000000000000000003030303FB
:109AE0000303030000000000000000000003030364
:109AF0000303030300000000000000000000030354
:109B00000303030303000000000000000000000343
:109B10000303030303030000000000000000000033
:109B20000303030303030300000000000000000020
:109B30000003030303030303000000000000000010
:109B40000000030303030303030000000000000000
:109B500000000003030303030303000000000000F0
:109B600000000000030303030303030000000000E0
:109B700000000000000303030303030300000000D0
:109B800000000000000003030303030303000000C0
:109B900000000000000000030303030303030000B0
:109BA00000000000000000000303030303030300A0
:109BB0000000000000000000000303030303030390
:109BC0000000000000000000000003030303030383
:109BD0000300000000000000000000030303030373
:109BE0000303000000000000000000000303030363
:109BF0000303030000000000000000000003030353
:109C00000303030300000000000000000000030342
:109C10000303030303000000000000000000000332
:109C20000303030303030000000000000000000022
:109C3000030303030303030000000000000000000F
:109C400000030303030303030000000000000000FF
:109C500000000303030303030300000000000000EF
:109C600000000003030303030303000000000000DF
:109C700000000000030303030303030000000000CF
:109C800000000000000303030303030300000000BF
:109C900000000000000003030303030303000000AF
:109CA000000000000000000303030303030300009F
:109CB000000000000000000003030303030303008F
:109CC000000000000000000000030303030303037F
:109CD0000000000000000000000003030303030372
:109CE0000300000000000000000000030303030362
:109CF0000303000000000000000000000303030352
:109D00000303030000000000000000000003030341
:109D10000303030300000000000000000000030331
:109D20000303030303000000000000000000000321
:109D30000303030303030000000000000000000011
:109D400003030303030303000000000000000000FE
:109D500000030303030303030000000000000000EE
:109D600000000303030303030300000000000000DE
:109D700000000003030303030303000000000000CE
:109D800000000000030303030303030000000000BE
:109D900000000000000303030303030300000000AE
:109DA000000000000000030303030303030000009E
:109DB000000000000000000303030303030300008E
:109DC000000000000000000003030303030303007E
:109DD000000000000000000000030303030303036E
:109DE0000000000000000000000003030303030361
:109DF0000300000000000000000000030303030351
:109E00000303000000000000000000000303030340
:109E10000303030000000000000000000003030330
:109E20000303030300000000000000000000030320
:109E30000303030303000000000000000000000310
:109E40000303030303030000000000000000000000
:109E500003030303030303000000000000000000ED
:109E600000030303030303030000000000000000DD
:109E700000000303030303030300000000000000CD
:109E800000000003030303030303000000000000BD
:109E900000000000030303030303030000000000AD
:109EA000000000000003030303030303000000009D
:109EB000000000000000030303030303030000008D
:109EC000000000000000000303030303030300007D
:109ED000000000000000000003030303030303006D
:109EE000000000000000000000030303030303035D
:109EF0000000000000000000000003030303030350
:109F0000030000000000000000000003030303033F
:109F1000030300000000000000000000030303032F
:109F2000030303000000000000000000000303031F
:109F3000030303030000000000000000000003030F
:109F400003030303030000000000000000000003FF
:109F500003030303030300000000000000000000EF
:109F600003030303030303000000000000000000DC
:109F700000030303030303030000000000000000CC
:109F800000000303030303030300000000000000BC
:109F900000000003030303030303000000000000AC
:109FA000000000000303030303030300000000009C
:109FB000000000000003030303030303000000008C
:109FC000000000000000030303030303030000007C
:109FD000000000000000000303030303030300006C
:109FE000000000000000000003030303030303005C
:109FF000000000000000000000030303030303034C
:10A00000000000000000000000000303030303033E
:10A01000030000000000000000000003030303032E
:10A02000030300000000000000000000030303031E
:10A03000030303000000000000000000000303030E
:10A0400003030303000000000000000000000303FE
:10A0500003030303030000000000000000000003EE
:10A0600003030303030300000000000000000000DE
:10A0700003030303030303000000000000000000CB
:10A0800000030303030303030000000000000000BB
:10A0900000000303030303030300000000000000AB
:10A0A000000000030303030303030000000000009B
:10A0B000000000000303030303030300000000008B
:10A0C000000000000003030303030303000000007B
:10A0D000000000000000030303030303030000006B
:10A0E000000000000000000303030303030300005B
:10A0F000000000000000000003030303030303004B
:10A10000000000000000000000030303030303033A
:10A11000000000000000000000000303030303032D
:10A12000030000000000000000000003030303031D
:10A13000030300000000000000000000030303030D
:10A1400003030300000000000000000000030303FD
:10A1500003030303000000000000000000000303ED
:10A1600003030303030000000000000000000003DD
:10A1700003030303030303020202030302020203B5
:10A1800003030303030303030202020303020202A5
:10A190000303030303030303030202020303020294
:10A1A0000203030303030303030302020203030284
:10A1B0000202030303030303030303020202030374
:10A1C00002020203030303030303030079A95ADA1B
:10A1D000997DA95ADE6379C0B086BFB17F79A95A4B
:10A1E000D9997DA95ADD6379C0B086BFB17F79A9BD
:10A1F0005AD9997DA95ADD6379C0B086BFB17F79FC
:10A20000A85AD9997DA85ADD6379C0B086BFB17FBD
:10A2100079A85AD9997DA85ADD6379C0B086BFB1B3
:10A220007F79A85AD9997DA85ADD6379C0B086BFD5
:10A23000B17F79A85AD8997DA85ADC6379C0B086D5
:10A24000BFB17F79A85AD8997DA85ADC6379C0B08C
:10A2500086BFB17F79A85AD8997DA85ADC6379C0A6
:10A26000B086BFB17F79A85AD8997DA85ADC6379A6
:10A27000C0B086BFB17F79A85AD7997DA85ADB6351
:10A2800079C0B086BFB17F79A75AD7997DA75ADB2D
:10A290006379C0B086BFB17F79A75AD7997DA75A95
:10A2A000DB6379C0B086BFB17F79A75AD7997DA704
:10A2B0005ADB6379C0B086BFB17F79A75AD7997D41
:10A2C000A75ADB6379C0B086BFB17F79A75AD69908
:10A2D0007DA75ADA6379C0B086BFB17F79AB6BCD09
:10A2E000997DAB6BD16379C0B086BFB17F79AE7811
:10A2F000C6997DAE78CA6379C0B086BFB17F79B1A7
:10A3000083BF997DB183C36379C0B086BFB17F79C4
:10A31000B38DBA997DB38DBE6379C0B086BFB17F6E
:10A3200079B596B4997DB596B86379C0B086BFB15A
:10A330007F79B79FB0997DB79FB46379C0B086BF6E
:10A34000B17F79B8A7AB997DB8A7AF6379C0B08664
:10A35000BFB17F79BAAEA7997DBAAEAB6379C0B011
:10A3600086BFB17F79BBB5A2997DBBB5A66379C025
:10A37000B086BFB17F79BDBC9E997DBDBCA263791B
:10A38000C0B086BFB17F79BEC29A997DBEC29E63BE
:10A3900079C0B086BFB17F79BFC996997DBFC99A90
:10A3A0006379C0B086BFB17F79C0CF92997DC0CFAD
:10A3B000966379C0B086BFB17F79C2D58E997DC2D0
:10A3C000D5926379C0B086BFB17F79C3DB8B997DAD
:10A3D000C3DB8F6379C0B086BFB17F79C4E0879952
:10A3E0007DC4E08B6379C0B086BFB17F79C2DF875F
:10A3F000997DC2DF8B6376C0AF89BFB07F79BDDD49
:10A4000088997DBDDD8C6370C0AD8FBFAE7F79BA9A
:10A41000DB88997DBADB8C636DC0AC92BFAD7F7970
:10A42000B7DA89997DB7DA8D6369C0AA96BFAB7F29
:10A4300079B4D88A997DB4D88E6366C0A999BFAA29
:10A440007F79B2D78A997DB2D78E6363C0A89CBF4B
:10A45000A97F79AFD68B997DAFD68F6360C0A79F58
:10A46000BFA87F79ACD48C997DACD490635CC0A537
:10A47000A3BFA67F79A9D38C997DA9D3906359C036
:10A48000A4A6BFA57F79A6D18D997DA6D19163564B
:10A49000C0A3A9BFA47F79A4D08D997DA4D09163D6
:10A4A00052C0A2ADBFA37F79A1CF8E997DA1CF92DB
:10A4B000634FC0A0B0BFA17F799ECD8F997D9ECD07
:10A4C00093634CC09FB3BFA07F799BCC8F997D9B3A
:10A4D000CC936349C09EB6BF9F7F7998CA90997DFF
:10A4E00098CA946345C09DBABF9E7F7995C99199DA
:10A4F0007D95C9956342C09BBDBF9C7F7993C891F0
:10A50000997D93C895633FC09AC0BF9B7F7990C6E1
:10A5100092997D90C696633BC099C4BF9A7F798D0E
:10A52000C592997D8DC5966338C098C7BF997F79CC
:10A530008AC393997D8AC3976335C096CABF977FB4
:10A540007987C294997D87C2986332C095CDBF96B2
:10A550007F7985C194997D85C198632EC094D1BFC0
:10A56000957F7982BF95997D82BF99632BC093D4E3
:10A57000BF947F797FBE96997D7FBE9A6328C091F4
:10A58000D7BF927F797CBC96997D7CBC9A6324C0AE
:10A5900090DBBF917F7979BB97997D79BB9B6321D4
:10A5A000C08FDEBF907F7977BA97997D77BA9B632A
:10A5B0001EC08EE1BF8F7F7974B898997D74B89C66
:10A5C000631BC08CE4BF8D7F7971B799997D71B79A
:10A5D0009D6317C08BE8BF8C7F796EB599997D6EAE
:10A5E000B59D6314C08AEBBF8B7F796BB49A997D5C
:10A5F0006BB49E6311C089EEBF8A7F7968B29B9964
:10A600007D68B29F630DC087F2BF887F7969B19D75
:10A61000997D69B1A1630FC087F0BF887F796BAF67
:10A62000A2997D6BAFA66313C088ECBF897F796C5C
:10A63000ADA4997D6CADA86316C088E9BF897F7908
:10A640006DACA7997D6DACAB6318C089E7BF8A7FFD
:10A65000796EAAAA997D6EAAAE631AC08AE5BF8BED
:10A660007F796FA9AC997D6FA9B0631DC08AE2BFE5
:10A670008B7F7970A7AF997D70A7B3631FC08BE004
:10A68000BF8C7F7971A6B2997D71A6B66321C08C0B
:10A69000DEBF8D7F7972A4B4997D72A4B86324C0A3
:10A6A0008CDBBF8D7F7973A3B7997D73A3BB6326C2
:10A6B000C08DD9BF8E7F7974A1BA997D74A1BE6314
:10A6C00028C08DD7BF8E7F7975A0BC997D75A0C03D
:10A6D000632BC08ED4BF8F7F79769EBF997D769E87
:10A6E000C3632DC08FD2BF907F79779DC2997D774C
:10A6F0009DC6632FC08FD0BF907F79789BC4997D12
:10A70000789BC86332C090CDBF917F79799AC79901
:10A710007D799ACB6334C091CBBF927F797A99CA05
:10A72000997D7A99CE6336C091C9BF927F797B9724
:10A73000CC997D7B97D06339C092C6BF937F797CDB
:10A7400096CF997D7C96D3633BC092C4BF937F79AB
:10A750007D94D2997D7D94D6633DC093C2BF947F92
:10A76000797E93D4997D7E93D86340C094BFBF9582
:10A770007F797F91D7997D7F91DB6342C094BDBF84
:10A78000957F798090DA997D8090DE6344C095BB97
:10A79000BF967F79818EDC997D818EE06347C0967C
:10A7A000B8BF977F79828DDF997D828DE36349C041
:10A7B00096B6BF977F79838BE2997D838BE6634B57
:10A7C000C097B4BF987F79848AE4997D848AE863CE
:10A7D0004EC097B1BF987F798588E7997D8588EBD2
:10A7E0006350C098AFBF997F798687EA997D868745
:10A7F000EE6352C099ADBF9A7F798785EC997D87CA
:10A8000085F06355C099AABF9A7F798884EF997DB6
:10A810008884F36357C09AA8BF9B7F798982F29995
:10A820007D8982F6635AC09BA5BF9C7F798B80F19E
:10A83000997D8B80F5635BC09CA4BF9D7F798F7BE6
:10A84000EE997D8F7BF2635EC09EA1BF9F7F799161
:10A8500079ED997D9179F16360C09F9FBFA07F7969
:10A860009376EB997D9376EF6362C0A19DBFA27F43
:10A87000799574EA997D9574EE6364C0A29BBFA339
:10A880007F799771E8997D9771EC6366C0A399BF52
:10A89000A47F79996FE7997D996FEB6368C0A5975D
:10A8A000BFA67F799B6CE5997D9B6CE9636AC0A626
:10A8B00095BFA77F799D6AE4997D9D6AE8636CC026
:10A8C000A793BFA87F799F67E2997D9F67E6636E34
:10A8D000C0A991BFAA7F79A165E1997DA165E563D2
:10A8E00070C0AA8FBFAB7F79A362DF997DA362E3BB
:10A8F0006372C0AB8DBFAC7F79A560DE997DA5602A
:10A90000E26374C0AD8BBFAE7F79A75DDC997DA794
:10A910005DE06376C0AE89BFAF7F79A95BDB997DCF
:10A92000A95BDF6378C0AF87BFB07F79AB58D99997
:10A930007DAB58DD637AC0B185BFB27F79A75AD6A7
:10A94000997DA75ADA6379C0B086BFB17F79A75ADB
:10A95000D6997DA75ADA6379C0B086BFB17F79A74F
:10A960005AD6997DA75ADA6379C0B086BFB17F798C
:10A97000A75AD6997DA75ADA6379C0B086BFB17F4E
:10A9800079A75AD6997DA75ADA6379C0B086BFB144
:10A990007F79A75AD6997DA75ADA6379C0B086BF66
:10A9A000B17F79A75AD6997DA75ADA6379C0B08664
:10A9B000BFB17F79A75AD6997DA75ADA6379C0B01B
:10A9C00086BFB17F79A75AD6997DA75ADA6379C035
:10A9D000B086BFB17F79A75AD6997DA75ADA637935
:10A9E000C0B086BFB17F79A75AD6997DA75ADA63DE
:10A9F00079C0B086BFB17F79A75AD6997DA75ADAB8
:10AA00006379C0B086BFB17F79A75AD6997DA75A1E
:10AA1000DA6379C0B086BFB17F79A75AD6997DA78E
:10AA20005ADA6379C0B086BFB17F79A75AD6997DCB
:10AA3000A75ADA6379C0B086BFB17F79A75AD69991
:10AA40007DA75ADA6379C0B086BFB17F03020202E4
:10AA500003030202020303030303030302030202CC
:10AA600002030302020203030303030303020302BC
:10AA700002020303020202030303030303030203AC
:10AA8000020202030302020203030303030303029D
:10AA9000030202020303020202030303030303038C
:10AAA000020302020203030202020303030303037D
:10AAB000030203020202030302020203030303036D
:10AAC000030302030202020303020202030303035D
:10AAD000030303020302020203030202020303034D
:10AAE000030303030203020202030302020203033D
:10AAF000030303030302030202020303020202032D
:10AB0000030303030303020302020203030202021C
:10AB1000030303030303030203020202030302020B
:10AB200002030303030303030203020202030302FB
:10AB300002020303030303030302030202020303EB
:10AB400002020203030303030303020302020203DC
:10AB500003020202030303030303030203030303C9
:10AB600003030303030303030303030302030303B6
:10AB700003030303030303030303030303020303A6
:10AB80000303030303030303030303030303020396
:10AB90000303030303030303030303030303030286
:10ABA0000303030303030303030303030303030375
:10ABB0000203030303030303030303030303030366
:10ABC0000302030303030303030303030303030356
:10ABD0000303020303030303030303030303030346
:10ABE0000303030203030303030303030303030336
:10ABF0000303030302030303030303030303030326
:10AC00000303030303020303030303030303030315
:10AC10000303030303030203030303030303030305
:10AC200003030303030303020303030303030303F5
:10AC300003030303030303030203030303030303E5
:10AC400003030303030303030302030303030303D5
:10AC500003030303030303030303020303030303C5
:10AC600003030303030303030303030203000000BE
:10AC700003030000000300030000030002030000C0
:10AC800000030300000003000300000300020300B0
:10AC900000000303000000030003000003000203A0
:10ACA0000000000303000000030003000003000293
:10ACB0000300000003030000000300030000030082
:10ACC0000203000000030300000003000300000370
:10ACD0000002030000000303000000030003000063
:10ACE0000300020300000003030000000300030050
:10ACF0000003000203000000030300000003000340
:10AD00000000030002030000000303000000030032
:10AD1000030000030002030000000303000000031F
:10AD20000003000003000203000000030300000012
:10AD300003000300000300020300000003030000FF
:10AD400000030003000003000203000000030300EF
:10AD500000000300030000030002030000000303DF
:10AD600000000003000300000300020300000003D2
:10AD700003000000030003000003000203000000C2
:10AD800003030000000300030000030002030000AF
:10AD9000000303000000030003000003000203009F
:10ADA000000003030000000300030000030002038F
:10ADB0000000000303000000030003000003000282
:10ADC0000300000003030000000300030000030071
:10ADD000020300000003030000000300030000035F
:10ADE0000002030000000303000000030003000052
:10ADF000030002030000000303000000030003003F
:10AE0000000300020300000003030000000300032E
:10AE10000000030002030000000303000000030021
:10AE2000030000030002030000000303000000030E
:10AE30000003000003000203000000030300000001
:10AE400003000300000300020300000003030000EE
:10AE500000030003000003000203000000030300DE
:10AE600000000300030000030002030000000303CE
:10AE700000000003000300000300020300000003C1
:10AE800003000000030003000003000203000000B1
:10AE90000303000000030203020203020203000096
:10AEA0000003030000000302030202030202030086
:10AEB0000000030300000003020302020302020376
:10AEC0000000000303000000030203020203020269
:10AED0000300000003030000000302030202030258
:10AEE0000203000000030300000003020302020348
:10AEF0000202030000000303000000030203020239
:10AF00000302020300000003030000000302030227
:10AF10000203020203000000030300000003020317
:10AF20000202030202030000000303000000030208
:10AF300003020203020203000000030300000003F7
:10AF400002030202030202030000000303000000E8
:10AF500003020302020302020300000003030000D5
:10AF600000030203020203020203000000030300C5
:10AF700000000302030202030202030000000303B5
:10AF800000000003020302020302020300000003A8
:10AF90000300000003020302020302020300000098
:10AFA0000303000000030203020203020203000085
:10AFB0000003030000000302030202030202030075
:10AFC0000000030300000003020302020302020365
:10AFD0000000000303000000030203020203020258
:10AFE0000300000003030000000302030202030247
:10AFF0000203000000030300000003020302020337
:10B000000202030000000303000000030203020227
:10B010000302020300000003030000000302030216
:10B020000203020203000000030300000003020306
:10B0300002020302020300000003030000000302F7
:10B0400003020203020203000000030300000003E6
:10B0500002030202030202030000000303000000D7
:10B0600003020302020302020300000003030000C4
:10B0700000030203020203020203000000030300B4
:10B0800000000302030202030202030000000303A4
:10B090000000000302030202030202030000000397
:10B0A0000300000003020302020302020302020281
:10B0B000030302020203020302020302020302026A
:10B0C000020303020202030203020203020203025A
:10B0D000020203030202020302030202030202034A
:10B0E000020202030302020203020302020302023B
:10B0F000030202020303020202030203020203022A
:10B100000203020202030302020203020302020319
:10B11000020203020202030302020203020302020A
:10B1200003020203020202030302020203020302F9
:10B1300002030202030202020303020202030203E9
:10B1400002020302020302020203030202020302DA
:10B1500003020203020203020202030302020203C9
:10B1600002030202030202030202020303020202BA
:10B1700003020302020302020302020203030202A9
:10B180000203020302020302020302020203030299
:10B190000202030203020203020203020202030389
:10B1A000020202030203020203020203020202037A
:10B1B0000302020203020302020302020303030367
:10B1C0000303030303030202020202020003030358
:10B1D0000303030303030302020202020200030348
:10B1E0000303030303030303020202020202000338
:10B1F0000303030303030303030202020202020028
:10B200000303030303030303030302020202020214
:10B210000003030303030303030303020202020206
:10B2200002000303030303030303030302020202F6
:10B2300002020003030303030303030303020202E6
:10B2400002020200030303030303030303030202D6
:10B2500002020202000303030303030303030302C6
:10B2600002020202020003030303030303030303B6
:10B2700002020202020200030303030303030303A7
:10B280000302020202020200030303030303030397
:10B290000303020202020202000303030303030387
:10B2A0000303030202020202020003030303030377
:10B2B0000303030302020202020200030303030367
:10B2C00003030303030202020202020079A95ADA0D
:10B2D000997DA95ADE6379C0B086BFB17F79A95A3A
:10B2E000DA997DA95ADE6379C0B086BFB17F79A9AA
:10B2F0005ADA997DA95ADE6379C0B086BFB17F79E9
:10B30000A95ADA997DA95ADE6379C0B086BFB17FA8
:10B3100079A95ADA997DA95ADE6379C0B086BFB19E
:10B320007F79A95ADA997DA95ADE6379C0B086BFC0
:10B33000B17F79A95ADA997DA95ADE6379C0B086BE
:10B34000BFB17F79A95ADA997DA95ADE6379C0B075
:10B3500086BFB17F79A95ADA997DA95ADE6379C08F
:10B36000B086BFB17F79A95ADA997DA95ADE63798F
:10B37000C0B086BFB17F79A960DA997DA960DE632C
:10B3800079C0B086BFB17F79A96DDA997DA96DDEEC
:10B390006379C0B086BFB17F79A973DB997DA9734A
:10B3A000DF6379C0B086BFB17F79A97ADB997DA9C7
:10B3B0007ADF6379C0B086BFB17F79A981DB997DDF
:10B3C000A981DF6379C0B086BFB17F79A987DC9995
:10B3D0007DA987E06379C0B086BFB17F79A98EDC93
:10B3E000997DA98EE06379C0B086BFB17F79A994B9
:10B3F000DC997DA994E06379C0B086BFB17F79A95B
:10B400009BDD997DA99BE16379C0B086BFB17F794F
:10B41000A9A2DD997DA9A2E16379C0B086BFB17F01
:10B4200079A9A8DD997DA9A8E16379C0B086BFB1EB
:10B430007F79A9AFDE997DA9AFE26379C0B086BFFD
:10B44000B17F79A9B5DE997DA9B5E26379C0B086EF
:10B45000BFB17F79A9BCDE997DA9BCE26379C0B098
:10B4600086BFB17F79A9C3DF997DA9C3E36379C0A2
:10B47000B086BFB17F79A9C9DF997DA9C9E3637996
:10B48000C0B086BFB17F79A9D0DF997DA9D0E36331
:10B4900079C0B086BFB17F79A9D6E0997DA9D6E4FD
:10B4A0006379C0B086BFB17F79A9DDE0997DA9DD60
:10B4B000E46379C0B086BFB17F79A9E4E1997DA941
:10B4C000E4E56379C0B086BFB17F79A7E2E1997DF9
:10B4D000A7E2E56376C0B089BFB17F79A3DDE199CA
:10B4E0007DA3DDE5636FC0AF90BFB07F79A1DAE0E7
:10B4F000997DA1DAE4636BC0AE94BFAF7F799FD72B
:10B50000E0997D9FD7E46367C0AD98BFAE7F799D1A
:10B51000D5E0997D9DD5E46363C0AC9CBFAD7F79D8
:10B520009BD2DF997D9BD2E3635FC0ABA0BFAC7FB2
:10B530007999CFDF997D99CFE3635BC0AAA4BFABB4
:10B540007F7997CCDF997D97CCE36357C0A9A8BFDB
:10B55000AA7F7995CADE997D95CAE26353C0A8ACEB
:10B56000BFA97F7992C7DE997D92C7E2634FC0A7DA
:10B57000B0BFA87F7990C4DE997D90C4E2634CC0CF
:10B58000A7B3BFA87F798EC1DD997D8EC1E16348E5
:10B59000C0A6B7BFA77F798CBFDD997D8CBFE16363
:10B5A00044C0A5BBBFA67F798ABCDD997D8ABCE17A
:10B5B0006340C0A4BFBFA57F7988B9DC997D88B9F5
:10B5C000E0633CC0A3C3BFA47F7986B6DC997D86C7
:10B5D000B6E06338C0A2C7BFA37F7984B4DC997D8D
:10B5E00084B4E06334C0A1CBBFA27F7982B1DB9980
:10B5F0007D82B1DF6330C0A0CFBFA17F7980AEDB99
:10B60000997D80AEDF632CC09FD3BFA07F797DABD7
:10B61000DA997D7DABDE6328C09ED7BF9F7F797BA3
:10B62000ABD6997D7BABDA6328C09ED7BF9F7F796D
:10B6300076ABCD997D76ABD26328C09ED7BF9F7F76
:10B640007973ABC9997D73ABCE6328C09ED7BF9F7A
:10B650007F7971ABC4997D71ABCA6328C09ED7BF97
:10B660009F7F796EABBF997D6EABC66328C09ED7B6
:10B67000BF9F7F796BABBB997D6BABC26328C09ECC
:10B68000D7BF9F7F7969ABB6997D69ABBE6328C090
:10B690009ED7BF9F7F7966ABB2997D66ABBA6328B0
:10B6A000C09ED7BF9F7F7963ABAD997D63ABB66317
:10B6B00028C09ED7BF9F7F7960ABA8997D60ABB152
:10B6C0006328C09ED7BF9F7F7961ABA7997D61AB8F
:10B6D000B0632BC09ED4BF9F7F7964ABA4997D6477
:10B6E000ABAD6332C09ECDBF9F7F7966ABA2997D23
:10B6F00066ABAB6335BF9ECABE9F7F7968ABA0992E
:10B700007D68ABA96339BF9EC6BE9F7F796AAB9E39
:10B71000997D6AABA7633CBE9EC3BD9F7F796CAB2E
:10B720009C997D6CABA56340BE9EBFBD9F7F796D2C
:10B73000AB9A997D6DABA36343BE9EBCBD9F7F79E1
:10B740006FAB98997D6FABA16347BD9EB8BC9F7FDF
:10B750007971AB96997D71AB9F634ABD9EB5BC9FD5
:10B760007F7973AB94997D73AB9D634EBC9EB1BBE7
:10B770009F7F7975AB93997D75AB9C6352BC9EADF1
:10B78000BB9F7F7977AB91997D77AB9A6355BC9ED0
:10B79000AABB9F7F7979AB8F997D79AB986359BBB1
:10B7A0009EA6BA9F7F797AAB8D997D7AAB96635CC2
:10B7B000BB9EA3BA9F7F797CAB8B997D7CAB946356
:10B7C00060BA9E9FB99F7F797EAB89997D7EAB924F
:10B7D0006363BA9E9CB99F7F7980AB87997D80AB6C
:10B7E000906367BA9E98B99F7F7982AB85997D8275
:10B7F000AB8E636AB99E95B89F7F7984AB83997D40
:10B8000084AB8C636EB99E91B89F7F7986AB81992A
:10B810007D86AB8A6372B89E8DB79F7F798CAD832E
:10B82000997D8CAD8C6372B89E8DB79F7F7998B1EE
:10B8300088997D98B1916372B89E8DB79F7F799EEC
:10B84000B38B997D9EB3946372B89E8DB79F7F79B9
:10B85000A4B68D997DA4B6966372B89E8DB79F7F6E
:10B8600079AAB890997DAAB8996372B89E8DB79F4E
:10B870007F79B0BA93997DB0BA9C6372B89E8DB748
:10B880009F7F79B6BD95997DB6BD9E6372B89E8D3A
:10B89000B79F7F79BCBF98997DBCBFA16372B89EEA
:10B8A0008DB79F7F79C2C19B997DC2C1A46372B8D5
:10B8B0009E8DB79F7F79C8C49E997DC8C4A76372C7
:10B8C000B89E8DB79F7F79C6BDA2997DC6BDAA637C
:10B8D00072B89F8DB7A07F79C2AFAA997DC2AFB170
:10B8E0006373B9A18CB8A27F79C0A8AE997DC0A8B6
:10B8F000B56373B9A28CB8A37F79BEA1B2997DBE9E
:10B90000A1B86374BAA38BB9A47F79BC9AB6997DA8
:10B91000BC9ABC6374BAA58BB9A67F79BA93BA995D
:10B920007DBA93C06375BBA68ABAA77F79B78BBE71
:10B93000997DB78BC46375BCA78ABBA87F79B58492
:10B94000C2997DB584C76376BCA889BBA97F79B34A
:10B950007DC6997DB37DCB6376BDA989BCAA7F796D
:10B96000B176CA997DB176CF6377BDAB88BCAC7F29
:10B9700079AF6FCE997DAF6FD26377BEAC88BDAD26
:10B980007F79AD68D2997DAD68D66378BEAD87BD4D
:10B99000AE7F79AB61D6997DAB61DA6378BFAE8754
:10B9A000BEAF7F79A859DB997DA859DE6379C0B015
:10B9B00086BFB17F030303030303030303030303EE
:10B9C0000303030303030303030303030303030347
:10B9D0000303030303030303030303030303030337
:10B9E0000303030303030303030303030303030327
:10B9F0000303030303030303030303030303030317
:10BA00000303030303030303030303030303030306
:10BA100003030303030303030303030303030303F6
:10BA200003030303030303030303030303030303E6
:10BA300003030303030303030303030303030303D6
:10BA400003030303030303030303030303030303C6
:10BA500003030303030303030303030303030300B9
:10BA600000000303000000030303030303030303B5
:10BA700000000003030000000303030303030303A8
:10BA80000300000003030000000303030303030398
:10BA90000303000000030300000003030303030388
:10BAA0000303030000000303000000030303030378
:10BAB0000303030300000003030000000303030368
:10BAC0000303030303000000030300000003030358
:10BAD0000303030303030000000303000000030348
:10BAE0000303030303030300000003030000000338
:10BAF0000303030303030303000000030300000028
:10BB00000303030303030303030000000303000014
:10BB10000003030303030303030300000003030004
:10BB200000000303030303030303030000000303F4
:10BB300000000003030303030303030300000003E7
:10BB400003000000030303030303030303000000D7
:10BB500003030000000303030303030303030000C4
:10BB600000030300000003030303030303030300B4
:10BB700000000303000000030303030303030303A4
:10BB80000000000303000000030303030303030397
:10BB90000300000003030000000303030303030387
:10BBA0000303000000030300000003030303030377
:10BBB0000303030202020303020202030003000064
:10BBC0000300030302020203030202020300030054
:10BBD0000003000303020202030302020203000344
:10BBE0000000030003030202020303020202030037
:10BBF0000300000300030302020203030202020324
:10BC00000003000003000303020202030302020216
:10BC10000300030000030003030202020303020205
:10BC200002030003000003000303020202030302F5
:10BC300002020300030000030003030202020303E5
:10BC400002020203000300000300030302020203D6
:10BC500003020202030003000003000303020202C6
:10BC600003030202020300030000030003030202B5
:10BC700002030302020203000300000300030302A5
:10BC80000202030302020203000300000300030395
:10BC90000202020303020202030003000003000386
:10BCA0000302020203030202020300030000030076
:10BCB0000303020202030302020203000300000363
:10BCC0000003030202020303020202030003000056
:10BCD0000300030302020203030202020300030043
:10BCE0000003000303020202030302020203000333
:10BCF0000000030003030202020303020202030026
:10BD0000030000030003030002000303000200031A
:10BD1000000300000300030300020003030002000D
:10BD200003000300000300030300020003030002FA
:10BD300000030003000003000303000200030300EC
:10BD400002000300030000030003030002000303DA
:10BD500000020003000300000300030300020003CD
:10BD600003000200030003000003000303000200BD
:10BD700003030002000300030000030003030002AA
:10BD8000000303000200030003000003000303009C
:10BD9000020003030002000300030000030003038A
:10BDA000000200030300020003000300000300037D
:10BDB0000300020003030002000300000000000073
:10BDC0000303000200030300020003000000000060
:10BDD0000003030002000303000200030000000050
:10BDE0000000030300020003030002000300000040
:10BDF0000000000303000200030300020003000030
:10BE0000000000000303000200030300020003001F
:10BE1000000000000003030002000303000200030F
:10BE20000000000000000303000200030300020002
:10BE300003000000000000030300020003030002EF
:10BE400000030000000000000303000200030300E1
:10BE500002000300000000000003030002000303CF
:10BE600000020003000000000000030300020003C2
:10BE700003000200030000000000000303000200B2
:10BE8000030300020003000000000000030300029F
:10BE90000003030002000300000000000003030091
:10BEA000020003030002000300000000000003037F
:10BEB0000002000303000200030000000000000372
:10BEC0000300020003030002000300000000000062
:10BED000030300020003030002000300000000004F
:10BEE000000303000200030300020003000000003F
:10BEF000000003030002000303000200030000002F
:10BF00000000000303000000030300000003000022
:10BF10000000000003030000000303000000030012
:10BF20000000000000030300000003030000000302
:10BF300000000000000003030000000303000000F5
:10BF400003000000000000030300000003030000E2
:10BF500000030000000000000303000000030300D2
:10BF600000000300000000000003030000000303C2
:10BF700000000003000000000000030300000003B5
:10BF800003000000030000000000000303000000A5
:10BF90000303000000030000000000000303000092
:10BFA0000003030000000300000000000003030082
:10BFB0000000030300000003030303030303030360
:10BFC0000000000303000000030303030303030353
:10BFD0000300000003030000000303030303030343
:10BFE0000303000000030300000003030303030333
:10BFF0000303030000000303000000030303030323
:10C000000303030300000003030000000303030312
:10C010000303030303000000030300000003030302
:10C0200003030303030300000003030000000303F2
:10C0300003030303030303000000030300000003E2
:10C0400003030303030303030000000303000000D2
:10C0500003030303030303030300000003030000BF
:10C0600000030303030303030303000000030300AF
:10C07000000003030303030303030300000003039F
:10C080000000000303030303030303030000000392
:10C0900003000000030303030303030379AC68D226
:10C0A000997DAC68D66379C0B086BFB17F79AF7433
:10C0B000CC997DAF74D06379C0B086BFB17F79B1C0
:10C0C0007DC7997DB17DCB6379C0B086BFB17F79E3
:10C0D000B386C2997DB386C66379C0B086BFB17F8F
:10C0E00079B58EBE997DB58EC26379C0B086BFB179
:10C0F0007F79B795BA997DB795BE6379C0B086BF91
:10C10000B17F79B89CB6997DB89CBA6379C0B08686
:10C11000BFB17F79BAA2B2997DBAA2B66379C0B035
:10C1200086BFB17F79BBA8AF997DBBA8B36379C047
:10C13000B086BFB17F79BDAEAB997DBDAEAF63793F
:10C14000C0B086BFB17F79BEB4A8997DBEB4AC63E0
:10C1500079C0B086BFB17F79BFB9A5997DBFB9A9B4
:10C160006379C0B086BFB17F79C0BFA2997DC0BFDF
:10C17000A66379C0B086BFB17F79C1C49F997DC1E4
:10C18000C4A36379C0B086BFB17F79C2C99C997DD1
:10C19000C2C9A06379C0B086BFB17F79C3CE999977
:10C1A0007DC3CE9D6379C0B086BFB17F79C4D3967D
:10C1B000997DC4D39A6379C0B086BFB17F79C5D762
:10C1C00093997DC5D7976379C0B086BFB17F79C693
:10C1D000DC90997DC6DC946379C0B086BFB17F796D
:10C1E000C7E18D997DC7E1916379C0B086BFB17F0A
:10C1F00079C5E18A997DC5E18E6379C0B086BFB10A
:10C200007F79C1E283997DC1E2876379C0B086BF3F
:10C21000B17F79BEE37F997DBEE3836379C0B08649
:10C22000BFB17F79BCE47B997DBCE47F6379C0B00A
:10C2300086BFB17F79B9E578997DB9E57C6379C02E
:10C24000B086BFB17F79B7E674997DB7E678637938
:10C25000C0B086BFB17F79B4E770997DB4E77463ED
:10C2600079C0B086BFB17F79B2E76C997DB2E770D3
:10C270006379C0B086BFB17F79B0E868997DB0E8D6
:10C280006C6379C0B086BFB17F79ADE965997DAD4A
:10C29000E9696379C0B086BFB17F79ABEA61997D06
:10C2A000ABEA656379C0B086BFB17F79A8EB5D99D1
:10C2B0007DA8EB616379C0B086BFB17F79A6EC59E8
:10C2C000997DA6EC5D6379C0B086BFB17F79A3ED9F
:10C2D00055997DA3ED596379C0B086BFB17F799E32
:10C2E000E655997D9EE6596374C0B08BBFB17F79E6
:10C2F00094D855997D94D859636AC0B095BFB17FE1
:10C30000798ED055997D8ED0596365C0B09ABFB1F2
:10C310007F7989C955997D89C959635FC0B0A0BF2C
:10C32000B17F7983C255997D83C259635AC0B0A544
:10C33000BFB17F797EBA55997D7EBA596355C0B039
:10C34000AABFB17F7978B355997D78B359634FC04F
:10C35000B0B0BFB17F7973AC55997D73AC59634A66
:10C36000C0B0B5BFB17F796EA455997D6EA45963F5
:10C3700045C0B0BABFB17F79689D55997D689D5918
:10C380006340C0B0BFBFB17F79639655997D639616
:10C3900059633AC0B0C5BFB17F795D8E55997D5D57
:10C3A0008E596335C0B0CABFB17F79588755997D22
:10C3B0005887596330C0B0CFBFB17F79527F55994C
:10C3C0007D527F59632AC0B0D5BFB17F79527F5566
:10C3D000997D527F596337C0ABC8BFAC7F79527F1C
:10C3E00055997D527F596352C0A1ADBFA27F79524A
:10C3F0007F55997D527F59635FC09CA0BF9D7F7917
:10C40000527F55997D527F59636DC09792BF987F37
:10C4100079527F55997D527F59637AC09285BF9337
:10C420007F79527F55997D527F596388C08D77BF40
:10C430008E7F79527F55997D527F596396C0876967
:10C44000BF887F79527956997D52795A6396C08711
:10C4500069BF887F79516D59997D516D5D6396C033
:10C460008769BF887F7950675B997D50675F639666
:10C47000C08769BF887F7950615D997D5061616334
:10C4800096C08769BF887F794F5A5F997D4F5A63FD
:10C490006396C08769BF887F794E5461997D4E54F9
:10C4A000656396C08769BF887F794D4E63997D4DDE
:10C4B0004E676396C08769BF887F794D4864997DD0
:10C4C0004D48686396C08769BF887F794C426699FA
:10C4D0007D4C426A6396C08769BF887F794B3B6811
:10C4E000997D4B3B6C6396C08769BF887F794B35DC
:10C4F0006A997D4B356E6396C08769BF887F794A9C
:10C500002F6C997D4A2F706396C08769BF887F79A9
:10C5100049296E997D4929726396C08769BF887FD2
:10C5200079482270997D4822746396C08769BF88D4
:10C530007F794D2475997D4D24796395C0896ABFB3
:10C540008A7F79572980997D5729846392C08D6DA0
:10C55000BF8E7F795C2C86997D5C2C8A6391C08F1D
:10C560006EBF907F79612F8B997D612F8F638FC014
:10C570009170BF927F79673291997D673295638E12
:10C58000C09371BF947F796C3597997D6C359B63AF
:10C590008CC09673BF977F7971389D997D7138A152
:10C5A000638BC09874BF997F79763BA2997D763B67
:10C5B000A66389C09A76BF9B7F797C3EA8997D7CD3
:10C5C0003EAC6387C09C78BF9D7F798141AE997DE9
:10C5D0008141B26386C09E79BF9F7F798644B399BB
:10C5E0007D8644B76384C0A07BBFA17F798B47B9A8
:10C5F000997D8B47BD6383C0A37CBFA47F79904A9C
:10C60000BF997D904AC36381C0A57EBFA67F7996FE
:10C610004DC5997D964DC96380C0A77FBFA87F791E
:10C620009B50CA997D9B50CE637EC0A981BFAA7FD3
:10C6300079A053D0997DA053D4637DC0AB82BFACA9
:10C640007F79A556D6997DA556DA637BC0AD84BFA8
:10C65000AE7F79AB59DC997DAB59E06379C0B08688
:10C66000BFB17F00020202020202020202020303C1
:10C670000303030302020202020202020202020395
:10C680000303030303020202020202020202020285
:10C690000303030303030202020202020202020274
:10C6A0000203030303030302020202020202020264
:10C6B0000202030303030303020202020202020254
:10C6C0000202020303030303030202020202020244
:10C6D0000202020203030303030302020202020234
:10C6E0000202020202030303030303020202020224
:10C6F0000202020202020303030303030202020214
:10C700000202020202020203030303030302020203
:10C7100002020202020202020303030303030202F3
:10C7200002020202020202020203030303030302E3
:10C7300002020202020202020202030303030303D3
:10C7400002020202020202020202020303030303C4
:10C7500003020202020202020202020203030303B4
:10C7600003030202020202020202020202030303A4
:10C770000303030202020202020202020202030394
:10C780000303030302020202020202020202020384
:10C790000303030303020202020202020202020274
:10C7A0000303030303030202020202020202020263
:10C7B000020303030303030202030303020203034E
:10C7C000030203030303030302020303030202033E
:10C7D000030302030303030303020203030302022E
:10C7E000030303020303030303030202030303021D
:10C7F000020303030203030303030302020303030D
:10C8000002020303030203030303030302020303FD
:10C8100003020203030302030303030303020203ED
:10C8200003030202030303020303030303030202DD
:10C8300003030302020303030203030303030302CC
:10C8400002030303020203030302030303030303BC
:10C8500002020303030202030303020303030303AD
:10C86000030202030303020203030302030303039D
:10C87000030302020303030202030303020303038D
:10C88000030303020203030302020303030203037D
:10C89000030303030202030303020203030302036D
:10C8A000030303030302020303030202030303025D
:10C8B000030303030303020203030302020303034C
:10C8C000020303030303030202030303020203033D
:10C8D000030203030303030302020303030202032D
:10C8E000030302030303030303020203030302021D
:10C8F000030303020303030303030202030303020C
:10C9000002030303020303030303030202030303FB
:10C9100002020303030203030303030302020303EC
:10C9200003020203030302030303030303020203DC
:10C9300003030202030303020303030303030202CC
:10C9400003030302020303030203030303030302BB
:10C9500002030303020203030302030303030303AB
:10C96000020203030302020303030203030303039C
:10C97000030202030303020203030302030303038C
:10C98000030302020303030202030303020303037C
:10C99000030303020203030302020303030203036C
:10C9A000030303030202030303020203030302035C
:10C9B000030303030302020303030202030303024C
:10C9C000030303030303020203030302020303033B
:10C9D000020303030303030202030303020203032C
:10C9E000030203030303030302020303030202031C
:10C9F000030302030303030303020203030302020C
:10CA000003030302030303030303020203030302FA
:10CA100002030303020303030303030202030303EA
:10CA200002020303030203030303030302020303DB
:10CA300003020203030302030303030303020203CB
:10CA400003030202030303020303030303030202BB
:10CA500003030302020303030203030303030302AA
:10CA6000020303030202030303020303030303039A
:10CA7000020203030302020303030203030303038B
:10CA8000030202030303020203030302030303037B
:10CA9000030302020303030202030303020303036B
:10CAA000030303020203030302020303030203035B
:10CAB000030303030202030303020203030302034B
:10CAC000030303030302020303030202030303023B
:10CAD000030303030303020203030302020303032A
:10CAE000020303030303030202030303020203031B
:10CAF000030203030303030302020303030202030B
:10CB000003030203030303030302020303030202FA
:10CB100003030302030303030303020203030302E9
:10CB200002030303020303030303030202030303D9
:10CB300002020303030203030303030302020303CA
:10CB400003020203030302030303030303020203BA
:10CB500003030202030303020303030303030202AA
:10CB60000303030202030303020303030303030299
:10CB70000203030302020303030203030303030389
:10CB8000020203030302020303030203030303037A
:10CB9000030202030303020203030302030303036A
:10CBA000030302020303030202030303020303035A
:10CBB000030303020203030302020303030203034A
:10CBC000030303030202030303020203030302033A
:10CBD000030303030302020303030202030303022A
:10CBE0000303030303030202030303020203030319
:10CBF000020303030303030202030303020203030A
:10CC000003020303030303030202030303020203F9
:10CC100003030203030303030302020303030202E9
:10CC200003030302030303030303020079A95ADA8F
:10CC3000997DA95ADE6379C0B086BFB17F79A95AC0
:10CC4000DA997DA95ADE6379C0B086BFB17F79A930
:10CC50005ADA997DA95ADE6379C0B086BFB17F796F
:10CC6000A95ADA997DA95ADE6379C0B086BFB17F2F
:10CC700079A95ADA997DA95ADE6379C0B086BFB125
:10CC80007F79A95ADA997DA95ADE6379C0B086BF47
:10CC9000B17F79A95ADA997DA95ADE6379C0B08645
:10CCA000BFB17F79A95ADA997DA95ADE6379C0B0FC
:10CCB00086BFB17F79A95ADA997DA95ADE6379C016
:10CCC000B086BFB17F79A95ADA997DA95ADE637916
:10CCD000C0B086BFB17F79A95ADA997DA95ADE63BF
:10CCE00079C0B086BFB17F79A95ADA997DA95ADE99
:10CCF0006379C0B086BFB17F79A95ADA997DA95A04
:10CD0000DE6379C0B086BFB17F79A95ADA997DA96F
:10CD10005ADE6379C0B086BFB17F79A95ADA997DAE
:10CD2000A95ADE6379C0B086BFB17F79A95ADA9972
:10CD30007DA95ADE6379C0B086BFB17F79A855DA84
:10CD4000997DA855DE637CC0B183BFB27F79A54BC6
:10CD5000DA997DA54BDE6382C0B37DBFB47F79A431
:10CD600046DA997DA446DE6386C0B579BFB67F7981
:10CD7000A241DA997DA241DE6389C0B676BFB77F52
:10CD800079A03CDA997DA03CDE638DC0B872BFB952
:10CD90007F799F36DA997D9F36DE6390C0B96FBF89
:10CDA000BA7F799D31DA997D9D31DE6394C0BB6B8A
:10CDB000BFBC7F799B2CDA997D9B2CDE6397C0BC2E
:10CDC00068BFBD7F799A27DA997D9A27DE639AC07A
:10CDD000BD65BFBE7F799822DA997D9822DE639E79
:10CDE000C0BF61BFC07F79971CDA997D971CDE6355
:10CDF000A1C0C05EBFC17F799517DA997D9517DE16
:10CE000063A5C0C25ABFC37F799312DA997D93128A
:10CE1000DE63A8C0C357BFC47F79920DDA997D92B3
:10CE20000DDE63ACC0C553BFC67F799008DA997D2B
:10CE30009008DE63AFC0C650BFC77F798E02DA9913
:10CE40007D8E02DE63B3C0C84CBFC97F798E02DA23
:10CE5000997D8E02DE63B3C0C64CBFC77F798E0258
:10CE6000DA997D8E02DE63B4C0C14BBFC27F798E7A
:10CE700002DA997D8E02DE63B4C0BE4BBFBF7F79FC
:10CE80008E02DA997D8E02DE63B5C0BB4ABFBC7FDD
:10CE9000798E02DA997D8E02DE63B5C0B84ABFB9D9
:10CEA0007F798E02DA997D8E02DE63B6C0B549BF06
:10CEB000B67F798E02DA997D8E02DE63B6C0B24902
:10CEC000BFB37F798E02DA997D8E02DE63B7C0AF81
:10CED00048BFB07F798E02DA997D8E02DE63B7C0DB
:10CEE000AC48BFAD7F798E02DA997D8E02DE63B8E1
:10CEF000C0A947BFAA7F798E02DA997D8E02DE63D0
:10CF0000B8C0A647BFA77F798E02DA997D8E02DE70
:10CF100063B9C0A346BFA47F798E02DA997D8E02E1
:10CF2000DE63B9C0A046BFA17F798E02DA997D8EFB
:10CF300002DE63BAC09D45BF9E7F798E02DA997D7D
:10CF40008E02DE63BAC09A45BF9B7F798E02DA9962
:10CF50007D8E02DE63BBC09744BF987F798E02DA74
:10CF6000997D8E02DE63BAC09A45BF9B7F798E029F
:10CF7000DA997D8E02DE63B8C0A047BFA17F798EAB
:10CF800002DA997D8E02DE63B6C0A349BFA47F7921
:10CF90008E02DA997D8E02DE63B5C0A74ABFA87FF4
:10CFA000798E02DA997D8E02DE63B3C0AA4CBFABE4
:10CFB0007F798E02DA997D8E02DE63B2C0AD4DBFFD
:10CFC000AE7F798E02DA997D8E02DE63B0C0B14FFA
:10CFD000BFB27F798E02DA997D8E02DE63AFC0B474
:10CFE00050BFB57F798E02DA997D8E02DE63AEC0C6
:10CFF000B751BFB87F798E02DA997D8E02DE63ACBD
:10D00000C0BB53BFBC7F798E02DA997D8E02DE638E
:10D01000ABC0BE54BFBF7F798E02DA997D8E02DE2F
:10D0200063A9C0C156BFC27F798E02DA997D8E0294
:10D03000DE63A8C0C557BFC67F798E02DA997D8EA0
:10D0400002DE63A6C0C859BFC97F798E02DA997D16
:10D050008E02DE63A5C0CB5ABFCC7F798E02DA99EF
:10D060007D8E02DE63A3C0CF5CBFD07F798E02DAF3
:10D07000997D8E02DE63A4C0CC5BBFCD7F798E022A
:10D08000DA997D8E02DE63A6C0C659BFC77F798E4E
:10D0900002DA997D8E02DE63A8C0C357BFC47F79D0
:10D0A0008E02DA997D8E02DE63A9C0BF56BFC07FB3
:10D0B000798E02DA997D8E02DE63ABC0BC54BFBDAF
:10D0C0007F798E02DA997D8E02DE63ACC0B953BFE0
:10D0D000BA7F798E02DA997D8E02DE63AEC0B551D9
:10D0E000BFB67F798E02DA997D8E02DE63AFC0B261
:10D0F00050BFB37F798E02DA997D8E02DE63B0C0B5
:10D10000AF4FBFB07F798E02DA997D8E02DE63B2B7
:10D11000C0AB4DBFAC7F798E02DA997D8E02DE63A3
:10D12000B3C0A84CBFA97F798E02DA997D8E02DE4A
:10D1300063B5C0A54ABFA67F798E02DA997D8E02BB
:10D14000DE63B6C0A149BFA27F798E02DA997D8ED7
:10D1500002DE63B8C09E47BF9F7F798E02DA997D59
:10D160008E02DE63B9C09B46BF9C7F798E02DA993E
:10D170007D8E02DE63BBC09744BF987F798E02DA52
:10D18000997D8E02DE63BAC09A45BF9B7F798E027D
:10D19000DA997D8E02DE63B8C0A047BFA17F798E89
:10D1A00002DA997D8E02DE63B6C0A349BFA47F79FF
:10D1B0008E02DA997D8E02DE63B5C0A74ABFA87FD2
:10D1C000798E02DA997D8E02DE63B3C0AA4CBFABC2
:10D1D0007F798E02DA997D8E02DE63B2C0AD4DBFDB
:10D1E000AE7F798E02DA997D8E02DE63B0C0B14FD8
:10D1F000BFB27F798E02DA997D8E02DE63AFC0B452
:10D2000050BFB57F798E02DA997D8E02DE63AEC0A3
:10D21000B751BFB87F798E02DA997D8E02DE63AC9A
:10D22000C0BB53BFBC7F798E02DA997D8E02DE636C
:10D23000ABC0BE54BFBF7F798E02DA997D8E02DE0D
:10D2400063A9C0C156BFC27F798E02DA997D8E0272
:10D25000DE63A8C0C557BFC67F798E02DA997D8E7E
:10D2600002DE63A6C0C859BFC97F798E02DA997DF4
:10D270008E02DE63A5C0CB5ABFCC7F798E02DA99CD
:10D280007D8E02DE63A3C0CF5CBFD07F798E02DAD1
:10D29000997D8E02DE63A4C0CC5BBFCD7F798E0208
:10D2A000DA997D8E02DE63A6C0C659BFC77F798E2C
:10D2B00002DA997D8E02DE63A8C0C357BFC47F79AE
:10D2C0008E02DA997D8E02DE63A9C0BF56BFC07F91
:10D2D000798E02DA997D8E02DE63ABC0BC54BFBD8D
:10D2E0007F798E02DA997D8E02DE63ACC0B953BFBE
:10D2F000BA7F798E02DA997D8E02DE63AEC0B551B7
:10D30000BFB67F798E02DA997D8E02DE63AFC0B23E
:10D3100050BFB37F798E02DA997D8E02DE63B0C092
:10D32000AF4FBFB07F798E02DA997D8E02DE63B295
:10D33000C0AB4DBFAC7F798E02DA997D8E02DE6381
:10D34000B3C0A84CBFA97F798E02DA997D8E02DE28
:10D3500063B5C0A54ABFA67F798E02DA997D8E0299
:10D36000DE63B6C0A149BFA27F798E02DA997D8EB5
:10D3700002DE63B8C09E47BF9F7F798E02DA997D37
:10D380008E02DE63B9C09B46BF9C7F798E02DA991C
:10D390007D8E02DE63BBC09744BF987F798E02DA30
:10D3A000997D8E02DE63BAC09A45BF9B7F798E025B
:10D3B000DA997D8E02DE63B8C0A047BFA17F798E67
:10D3C00002DA997D8E02DE63B6C0A349BFA47F79DD
:10D3D0008E02DA997D8E02DE63B5C0A74ABFA87FB0
:10D3E000798E02DA997D8E02DE63B3C0AA4CBFABA0
:10D3F0007F798E02DA997D8E02DE63B2C0AD4DBFB9
:10D40000AE7F798E02DA997D8E02DE63B0C0B14FB5
:10D41000BFB27F798E02DA997D8E02DE63AFC0B42F
:10D4200050BFB57F798E02DA997D8E02DE63AEC081
:10D43000B751BFB87F798E02DA997D8E02DE63AC78
:10D44000C0BB53BFBC7F798E02DA997D8E02DE634A
:10D45000ABC0BE54BFBF7F798E02DA997D8E02DEEB
:10D4600063A9C0C156BFC27F798E02DA997D8E0250
:10D47000DE63A8C0C557BFC67F798E02DA997D8E5C
:10D4800002DE63A6C0C859BFC97F798E02DA997DD2
:10D490008E02DE63A5C0CB5ABFCC7F798E02DA99AB
:10D4A0007D8E02DE63A3C0CF5CBFD07F798E02DAAF
:10D4B000997D8E02DE63A4C0CC5BBFCD7F798E02E6
:10D4C000DA997D8E02DE63A6C0C659BFC77F798E0A
:10D4D00002DA997D8E02DE63A8C0C357BFC47F798C
:10D4E0008E02DA997D8E02DE63A9C0BF56BFC07F6F
:10D4F000798E02DA997D8E02DE63ABC0BC54BFBD6B
:10D500007F798E02DA997D8E02DE63ACC0B953BF9B
:10D51000BA7F798E02DA997D8E02DE63AEC0B55194
:10D52000BFB67F798E02DA997D8E02DE63AFC0B21C
:10D5300050BFB37F798E02DA997D8E02DE63B0C070
:10D54000AF4FBFB07F798E02DA997D8E02DE63B273
:10D55000C0AB4DBFAC7F798E02DA997D8E02DE635F
:10D56000B3C0A84CBFA97F798E02DA997D8E02DE06
:10D5700063B5C0A54ABFA67F798E02DA997D8E0277
:10D58000DE63B6C0A149BFA27F798E02DA997D8E93
:10D5900002DE63B8C09E47BF9F7F798E02DA997D15
:10D5A0008E02DE63B9C09B46BF9C7F798E02DA99FA
:10D5B0007D8E02DE63BBC09744BF987F798E04DA0C
:10D5C000997D8E04DE63B9C09746BF987F798F0935
:10D5D000DA997D8F09DE63B5C0984ABF997F79904B
:10D5E0000CDA997D900CDE63B3C0994CBF9A7F79B9
:10D5F000910FDA997D910FDE63B1C09A4EBF9B7F88
:10D60000799211DA997D9211DE63AFC09A50BF9B77
:10D610007F799314DA997D9314DE63ADC09B52BF7A
:10D620009C7F799317DA997D9317DE63ABC09C5486
:10D63000BF9D7F79941ADA997D941ADE63A9C09D03
:10D6400056BF9E7F79951CDA997D951CDE63A7C035
:10D650009E58BF9F7F79961FDA997D961FDE63A53E
:10D66000C09E5ABF9F7F799722DA997D9722DE6309
:10D67000A3C09F5CBFA07F799825DA997D9825DEAD
:10D6800063A1C0A05EBFA17F799827DA997D982712
:10D69000DE639FC0A160BFA27F79992ADA997D9944
:10D6A0002ADE639DC0A162BFA27F799A2DDA997D9F
:10D6B0009A2DDE639BC0A264BFA37F799B30DA9969
:10D6C0007D9B30DE6398C0A367BFA47F799C32DA6C
:10D6D000997D9C32DE6396C0A469BFA57F799D3594
:10D6E000DA997D9D35DE6394C0A56BBFA67F799ED8
:10D6F00038DA997D9E38DE6392C0A56DBFA67F792A
:10D700009E3BDA997D9E3BDE6390C0A66FBFA77FEC
:10D71000799F3DDA997D9F3DDE638EC0A771BFA8DA
:10D720007F79A040DA997DA040DE638CC0A873BFEA
:10D73000A97F79A143DA997DA143DE638AC0A875E8
:10D74000BFA97F79A246DA997DA246DE6388C0A987
:10D7500077BFAA7F79A348DA997DA348DE6386C0A4
:10D76000AA79BFAB7F79A34BDA997DA34BDE6384A3
:10D77000C0AB7BBFAC7F79A44EDA997DA44EDE634B
:10D7800082C0AC7DBFAD7F79A551DA997DA551DE10
:10D790006380C0AC7FBFAD7F79A653DA997DA65375
:10D7A000DE637EC0AD81BFAE7F79A756DA997DA7D3
:10D7B00056DE637CC0AE83BFAF7F79A859DA997D0E
:10D7C000A859DE637AC0AF85BFB07F79A95CDA99CA
:10D7D0007DA95CDE6377C0B088BFB17F030202021F
:10D7E000030302020203030303030303020302020F
:10D7F00002030302020203030303030303020302FF
:10D8000002020303020202030303030303030203EE
:10D8100002020203030202020303030303030302DF
:10D8200003020202030302020203030303030303CE
:10D8300002030202020303020202030303030303BF
:10D8400003020302020203030202020303030303AF
:10D85000030302030202020303020202030303039F
:10D86000030303020302020203030202020303038F
:10D87000030303030203020202030302020203037F
:10D88000030303030302030202020303020202036F
:10D89000030303030303020302020203030202025F
:10D8A000030303030303030203020202030302024E
:10D8B000020303030303030302030202020303023E
:10D8C000020203030303030303020302020203032E
:10D8D000020202030303030303030203020202031F
:10D8E0000302020203030303030303020300000213
:10D8F0000303000002030003000003000203000012
:10D9000002030300000203000300000300020300FF
:10D9100000020303000002030003000003000203EF
:10D9200000000203030000020300030000030002E2
:10D9300003000002030300000203000300000300D1
:10D9400002030000020303000002030003000003BF
:10D9500000020300000203030000020300030000B2
:10D96000030002030000020303000002030003009F
:10D97000000300020300000203030000020300038F
:10D980000000030002030000020303000002030082
:10D99000030000030002030000020303000002036F
:10D9A0000003000003000203000002030300000262
:10D9B0000300030000030002030000020303000051
:10D9C000020300030000030002030000020303003F
:10D9D000000203000300000300020300000203032F
:10D9E0000000020300030000030002030000020322
:10D9F0000300000203000300000300020300000212
:10DA00000303000002030003000003000203000000
:10DA100002030300000203000300000300020300EE
:10DA200000020303000002030003000003000203DE
:10DA300000000203030000020300030000030002D1
:10DA400003000002030300000203000300000300C0
:10DA500002030000020303000002030003000003AE
:10DA600000020300000203030000020300030000A1
:10DA7000030002030000020303000002030003008E
:10DA8000000300020300000203030000020300037E
:10DA90000000030002030000020303000002030071
:10DAA000030000030002030000020303000002035E
:10DAB0000003000003000203000002030300000251
:10DAC0000300030000030002030000020303000040
:10DAD000020300030000030002030000020303002E
:10DAE000000203000300000300020300000203031E
:10DAF0000000020300030000030002030000020311
:10DB00000300000203000300000300020300000200
:10DB100003030000020300030000030002030000EF
:10DB200002030300000203000300000300020300DD
:10DB300000020303000002030003000003000203CD
:10DB400000000203030000020300030000030002C0
:10DB500003000002030300000203000300000300AF
:10DB6000020300000203030000020300030000039D
:10DB70000002030000020303000002030003000090
:10DB8000030002030000020303000002030003007D
:10DB9000000300020300000203030000020300036D
:10DBA0000000030002030000020303000002030060
:10DBB000030000030002030000020303000002034D
:10DBC0000003000003000203000002030300000240
:10DBD000030003000003000203000002030300002F
:10DBE000020300030000030002030000020303001D
:10DBF000000203000300000300020300000203030D
:10DC000000000203000300000300020300000203FF
:10DC100003000002030003000003000203000002EF
:10DC200003030000020300030000030002030000DE
:10DC300002030300000203000300000300020300CC
:10DC400000020303000002030003000003000203BC
:10DC500000000203030000020300030000030002AF
:10DC6000030000020303000002030003000003009E
:10DC7000020300000203030000020300030000038C
:10DC8000000203000002030300000203000300007F
:10DC9000030002030000020303000002030003006C
:10DCA000000300020300000203030000020300035C
:10DCB000000003000203000002030300000203004F
:10DCC000030000030002030000020303000002033C
:10DCD000000300000300020300000203030000022F
:10DCE000030003000003000203000002030300001E
:10DCF000020300030000030002030000020303000C
:10DD000000020300030000030002030000020303FB
:10DD100000000203000300000300020300000203EE
:10DD200003000002030003000003000203000002DE
:10DD300003030000020300030000030002030000CD
:10DD400002030300000203000300000300020300BB
:10DD500000020303000002030003000003000203AB
:10DD6000000002030300000203000300000300029E
:10DD7000030000020303000002030003000003008D
:10DD8000020300000203030000020300030000037B
:10DD9000000203000002030300000203000300006E
:10DDA000030002030000020303000002030003005B
:10DDB000000300020300000203030000020300034B
:10DDC000000003000203000002030300000203003E
:10DDD000030000030002030000020303000002032B
:10DDE000000300000300020300000203030000021E
:10DDF000030003000003000203000002030300000D
:10DE000002030003000003000203000002030300FA
:10DE100000020300030000030002030000020303EA
:10DE200000000203000300000300020300000203DD
:10DE300003000002030003000003000203000002CD
:10DE400003030000020300030000030002030000BC
:10DE500002030300000203000300000300020300AA
:10DE6000000203030000020300030000030002039A
:10DE7000000002030300000203000300000300028D
:10DE8000030000020303000002030003000003007C
:10DE9000020300000203030000020300030000036A
:10DEA000000203000002030300000203000300005D
:10DEB000030002030000020303000002030003004A
:10DEC000000300020300000203030000020300033A
:10DED000000003000203000002030300000203002D
:10DEE000030000030002030000020303000002031A
:10DEF000000300000300020300000203030000020D
:10DF000003000300000300020300000203030000FB
:10DF100002030003000003000203000002030300E9
:10DF200000020300030000030002030000020303D9
:10DF300000000203000300000300020300000203CC
:10DF400003000002030003000003000203000002BC
:10DF500003030000020300030000030002030000AB
:10DF60000203030000020300030000030002030099
:10DF70000002030300000203000300000300020389
:10DF8000000002030300000203000300000300027C
:10DF9000030000020303000002030003000003006B
:10DFA0000203000002030300000203000300000359
:10DFB000000203000002030300000203000300004C
:10DFC0000300020300000203030000020300030039
:10DFD0000003000203000002030300000203000329
:10DFE000000003000203000002030300000203001C
:10DFF0000300000300020300000203030000020309
:10E0000000030000030002030000020303000002FB
:10E0100003000300000300020300000203030000EA
:10E0200002030003000003000203000002030300D8
:10E0300000020300030000030002030000020303C8
:10E0400000000203000300000300020300000203BB
:10E0500003000002030003000003000203000002AB
:10E06000030300000203000300000300020300009A
:10E070000203030000020300030000030002030088
:10E080000002030300000203000300000300020378
:10E09000000002030300000203000300000300026B
:10E0A000030000020303000002030003000003005A
:10E0B0000203000002030300000203000300000348
:10E0C000000203000002030300000203000300003B
:10E0D0000300020300000203030000020300030028
:10E0E0000003000203000002030300000203000318
:10E0F000000003000203000002030300000203000B
:10E1000003000003000203000002030300000203F7
:10E1100000030000030002030000020303000002EA
:10E1200003000300000300020300000203030000D9
:10E1300002030003000003000203000002030300C7
:10E1400000020300030000030002030000020303B7
:10E1500000000203000300000300020300000203AA
:10E160000300000203000300000300020303030294
:10E170000303030302030303030303030203030371
:10E180000203030303020303030303030302030362
:10E190000302030303030203030303030303020352
:10E1A0000303020303030302030303030303030242
:10E1B0000303030203030303020303030303030331
:10E1C0000203030302030303030203030303030322
:10E1D0000302030303020303030302030303030312
:10E1E0000303020303030203030303020303030302
:10E1F00003030302030303020303030302030303F2
:10E2000003030303020303030203030303020303E1
:10E2100003030303030203030302030303030203D1
:10E2200003030303030302030303020303030302C1
:10E2300003030303030303020303030203030303B0
:10E2400002030303030303030203030302030303A1
:10E250000302030303030303030203030302030391
:10E260000303020303030303030302030303020381
:10E270000303030203030303030303020303030271
:10E280000303030302030303030303030203030360
:10E290000203030303020303030303030302030351
:10E2A0000302030303030203030303030303020341
:10E2B0000303020303030302030303030303030231
:10E2C0000303030203030303020303030303030320
:10E2D0000203030302030303030203030303030311
:10E2E0000302030303020303030302030303030301
:10E2F00003030203030302030303030203030303F1
:10E3000003030302030303020303030302030303E0
:10E3100003030303020303030203030303020303D0
:10E3200003030303030203030302030303030203C0
:10E3300003030303030302030303020303030302B0
:10E34000030303030303030203030302030303039F
:10E350000203030303030303020303030203030390
:10E360000302030303030303030203030302030380
:10E370000303020303030303030302030303020370
:10E380000303030203030303030303027CA75AD816
:10E390009780A860D66179BDB486C1B17F7CA75A49
:10E3A000D89780A860D66179BDB486C1B17F7CA7BB
:10E3B0005AD89780A860D66179BDB486C1B17F7CF8
:10E3C000A75AD89780A860D66179BDB486C1B17FBD
:10E3D0007CA75AD89780A860D66179BDB486C1B1B0
:10E3E0007F7CA75AD89780A860D66179BDB486C1D2
:10E3F000B17F7CA75AD89780A860D66179BDB486D2
:10E40000C1B17F7CA75AD89780A860D66179BDB486
:10E4100086C1B17F7CA75AD89780A860D66179BDA4
:10E42000B486C1B17F7CA75AD89780A860D661799D
:10E43000BDB486C1B17F7CA35AD99780A860D6614C
:10E4400079BDB486C1B17F7C9B5ADC9780A860D629
:10E45000617ABDB485C1B17F7C975ADD9780A86091
:10E46000D6617BBDB484C1B17F7C935ADF9780A80D
:10E4700060D6617CBDB483C1B17F7C8F5AE0978048
:10E48000A860D6617CBDB483C1B17F7C8B5AE29712
:10E4900080A860D6617DBDB482C1B17F7C875AE31C
:10E4A0009780A860D6617EBDB481C1B17F7C835A5C
:10E4B000E59780A860D6617FBDB480C1B17F7C7FC5
:10E4C0005AE69780A860D6617FBDB480C1B17F7CD9
:10E4D0007B5AE89780A860D66180BDB47FC1B17FC8
:10E4E0007C775AE99780A860D66181BDB47EC1B1BE
:10E4F0007F7C735AEB9780A860D66182BDB47DC1E2
:10E50000B17F7C6F5AEC9780A860D66182BDB47DE4
:10E51000C1B17F7C6B5AEE9780A860D66183BDB491
:10E520007CC1B17F7C675AEF9780A860D66184BDBB
:10E53000B47BC1B17F7C635AF19780A860D66185B6
:10E54000BDB47AC1B17F7C5F5AF29780A860D66172
:10E5500085BDB47AC1B17F7C5B5AF49780A860D640
:10E560006186BDB479C1B17F7C575AF59780A860A8
:10E57000D66187BDB478C1B17F7C535AF79780A824
:10E5800060D66188BDB477C1B17F7C535AF797805C
:10E59000A460D7618BBDB474C1B17F7C535AF79727
:10E5A000809C60DA6191BDB46EC1B17F7C535AF733
:10E5B00097809860DB6194BDB46BC1B17F7C535A86
:10E5C000F797809461DD6197BDB468C1B17F7C53DA
:10E5D0005AF797809061DE619ABDB465C1B17F7CC6
:10E5E000535AF797808C61E0619DBDB462C1B17FE1
:10E5F0007C535AF797808861E161A0BDB45FC1B1D7
:10E600007F7C535AF797808462E361A3BDB45CC1F9
:10E61000B17F7C535AF797808062E461A6BDB459FC
:10E62000C1B17F7C535AF797807C62E661A9BDB483
:10E6300056C1B17F7C535AF797807862E761ACBDD1
:10E64000B453C1B17F7C535AF797807463E961AFCB
:10E65000BDB450C1B17F7C535AF797807063EA61B3
:10E66000B2BDB44DC1B17F7C535AF797806C63EC57
:10E6700061B5BDB44AC1B17F7C535AF797806863D6
:10E68000ED61B8BDB447C1B17F7C535AF797806440
:10E6900064EF61BBBDB444C1B17F7C535AF797802E
:10E6A0006064F061BEBDB441C1B17F7C535AF7973D
:10E6B000805C64F261C1BDB43EC1B17F7C535AF746
:10E6C00097805864F361C4BDB43BC1B17F7C535A99
:10E6D000F797805465F561C7BDB438C1B17F7C53ED
:10E6E0005AF797805465F561BEBDB541C1B27F7CD4
:10E6F000535AF797805465F561ACBDB753C1B47FE9
:10E700007C535AF797805465F561A3BDB85CC1B5D9
:10E710007F7C535AF797805465F5619ABDBA65C1FD
:10E72000B77F7C535AF797805465F56191BDBB6EF6
:10E73000C1B87F7C535AF797805465F56188BDBC9A
:10E7400077C1B97F7C535AF797805465F5617FBDD7
:10E75000BD80C1BA7F7C535AF797805465F56176C6
:10E76000BDBF89C1BC7F7C535AF797805465F56162
:10E770006DBDC092C1BD7F7C535AF797805465F53B
:10E780006164BDC19BC1BE7F7C535AF797805465BD
:10E79000F5615BBDC2A4C1BF7F7C535AF79780541B
:10E7A00065F56152BDC4ADC1C17F7C535AF79780F6
:10E7B0005465F56149BDC5B6C1C27F7C535AF79710
:10E7C000805465F56140BDC6BFC1C37F7C535AF715
:10E7D00097805465F56137BDC7C8C1C47F7C535A63
:10E7E000F797805465F5612EBDC9D1C1C67F7C53B2
:10E7F0005AF797805465F56125BDCADAC1C77F7C99
:10E80000535AF797805465F5611CBDCBE3C1C87FAF
:10E810007C535AF797805465F56113BDCCECC1C9A0
:10E820007F7C535AF797805465F5610ABDCEF5C1D8
:10E83000CB7F7C535FF19780546AEF610CBDCAF3C4
:10E84000C1C77F7C5369E497805474E26110BDC2F4
:10E85000EFC1BF7F7C536EDE97805479DC6112BDBF
:10E86000BEEDC1BB7F7C5373D79780547ED56114B6
:10E87000BDBAEBC1B77F7C5378D197805483CF6109
:10E8800016BDB6E9C1B37F7C537DCA97805488C852
:10E890006118BDB2E7C1AF7F7C5382C49780548DAD
:10E8A000C2611ABDAEE5C1AB7F7C5387BD97805472
:10E8B00092BB611CBDAAE3C1A77F7C538CB7978034
:10E8C0005497B5611EBDA6E1C1A37F7C5391B0975B
:10E8D00080549CAE6120BDA2DFC19F7F7C5391B06C
:10E8E0009780549CAE6126BBA2D9BF9F7F7C539179
:10E8F000B09780549CAE6132B7A2CDBB9F7F7C5352
:10E9000091B09780549CAE6138B5A2C7B99F7F7C07
:10E910005391B09780549CAE613EB3A2C1B79F7F24
:10E920007C5391B09780549CAE6144B1A2BBB59F1B
:10E930007F7C5391B09780549CAE614AAFA2B5B32F
:10E940009F7F7C5391B09780549CAE6150ADA2AF35
:10E95000B19F7F7C5391B09780549CAE6156ABA21F
:10E96000A9AF9F7F7C5391B09780549CAE615CA906
:10E97000A2A3AD9F7F7C5391B09780549CAE6162FF
:10E98000A7A29DAB9F7F7C5691AD9780579CAB61B2
:10E9900062A7A29DAB9F7F7C5C91A797805D9CA5A1
:10E9A0006162A7A29DAB9F7F7C5F91A49780609CD2
:10E9B000A26162A7A29DAB9F7F7C6291A1978063B9
:10E9C0009C9F6162A7A29DAB9F7F7C65919E978073
:10E9D000669C9C6162A7A29DAB9F7F7C68919B9780
:10E9E00080699C996162A7A29DAB9F7F7C6B919887
:10E9F00097806C9C966162A7A29DAB9F7F7C6E9175
:10EA00009597806F9C936162A7A29DAB9F7F7C715D
:10EA100091929780729C906162A7A29DAB9F7F7C30
:10EA200074918F9780759C8D6162A7A29DAB9F7F2B
:10EA30007C768F9297807799906163A8A29CAC9F17
:10EA40007F7C7B8A9997807C93976165AAA39AAE15
:10EA5000A07F7C7D879D97807E909B6166ABA4990B
:10EA6000AFA17F7C8084A19780818D9F6167ACA5D9
:10EA700098B0A27F7C8382A59780848AA36169ADC8
:10EA8000A696B1A37F7C857FA997808687A7616AB8
:10EA9000AEA695B2A37F7C887CAC97808984AA615E
:10EAA0006BAFA794B3A47F7C8B79B097808C81AE39
:10EAB000616CB0A893B4A57F7C8D77B497808E7E6F
:10EAC000B2616DB1A992B5A67F7C9074B897809120
:10EAD0007BB6616FB3AA90B7A77F7C9371BC978018
:10EAE0009478BA6170B4AA8FB8A77F7C956EC097EE
:10EAF000809675BE6171B5AB8EB9A87F7C986CC4E9
:10EB000097809972C26172B6AC8DBAA97F7C9B69FD
:10EB1000C797809C6FC56173B7AD8CBBAA7F7C9D86
:10EB200066CB97809E6CC96175B8AE8ABCAB7F7CA2
:10EB3000A063CF9780A169CD6176B9AE89BDAB7F67
:10EB40007CA361D39780A466D16177BAAF88BEAC4D
:10EB50007F7CA55ED79780A663D56178BBB087BF61
:10EB6000AD7F7CA85BDB9780A960D96179BCB18659
:10EB7000C0AE7F7CAB58DF9780AC5DDD617BBEB201
:10EB800084C2AF7F7CA75AD89780A860D66179BD30
:10EB9000B486C1B17F7CA75AD89780A860D6617926
:10EBA000BDB486C1B17F7CA75AD89780A860D661D2
:10EBB00079BDB486C1B17F7CA75AD89780A860D6AA
:10EBC0006179BDB486C1B17F7CA75AD89780A8600F
:10EBD000D66179BDB486C1B17F7CA75AD89780A889
:10EBE00060D66179BDB486C1B17F7CA75AD89780C1
:10EBF000A860D66179BDB486C1B17F7CA75AD89789
:10EC000080A860D66179BDB486C1B17F7CA75AD88F
:10EC10009780A860D66179BDB486C1B17F7CA75AC0
:10EC2000D89780A860D66179BDB486C1B17F03034F
:10EC300003030303030303030303030303030303A4
:10EC40000303030303030303030303030303030394
:10EC50000303030303030303030303030303030384
:10EC60000303030303030303030303030303030374
:10EC70000303030303030303030303030303030364
:10EC80000303030303030303030303030303030354
:10EC90000303030303030303030303030303030344
:10ECA0000303030303030303030303030303030334
:10ECB0000303030303030303030303030303030324
:10ECC0000303030303030303030303030303030314
:10ECD0000303030303030303030103020303010309
:10ECE00002030103030103030303010302030301FE
:10ECF00003020301030301030303030103020303EC
:10ED000001030203010303010303030301030203DD
:10ED100003010302030103030103030303010302CD
:10ED200003030103020301030301030303030103BC
:10ED300002030301030203010303010303030301AD
:10ED4000030203030103020301030301030303039B
:10ED5000010302030301030203010303010303038D
:10ED6000030103020303010302030103030103037D
:10ED7000030301030203030103020301030301036D
:10ED8000030303010302030301030203010303015D
:10ED9000030303030103020303010302030103034B
:10EDA000010303030301030203030103020301033D
:10EDB000030103030303010302030301030203012D
:10EDC000030301030303030103020303010302031B
:10EDD000010303010303030301030203030103020D
:10EDE00003010303010303030301030203030103FC
:10EDF00002030103030103030303010302030301ED
:10EE000003020301030301030303030103020303DA
:10EE100001030203010303010303030301030203CC
:10EE200003010302030103030103030303010202BD
:10EE300003030102020301030301030303030102AD
:10EE4000020303010202030103030103030303019D
:10EE5000020203030102020301030301030303038C
:10EE6000010202030301020203010303010303037E
:10EE7000030102020303010202030103030103036E
:10EE8000030301020203030102020301030301035E
:10EE9000030303010202030301020203010303014E
:10EEA000030303030102020303010202030103033C
:10EEB000010303030301020203030102020301032E
:10EEC000030103030303010202030301020203011E
:10EED000030301030303030102020303010202030C
:10EEE00001030301030303030102020303010202FE
:10EEF00003010303010303030301020203030102ED
:10EF000002030103030103030303010202030301DC
:10EF100002020301030301030303030102020303CB
:10EF200001020203010303010303030301020203BD
:10EF300003010202030103030103030303010202AD
:10EF4000030301020203010303010303030301029C
:10EF5000020303010202030103030103030303018C
:10EF6000020203030102020301030301030303037B
:10EF7000010202030301020203010303010303036D
:10EF80000301020203030102020301030101030161
:10EF9000030301020203030102020301030101034F
:10EFA0000103030102020303010202030103010141
:10EFB000030103030102020303010202030103012F
:10EFC000010301030301020203030102020301031F
:10EFD0000101030103030102020303010202030111
:10EFE00003010103010303010202030301020203FF
:10EFF00001030101030103030102020303010202F1
:10F0000003010301010301030301020203030102DF
:10F0100002030103010103010303010202030301CF
:10F0200002020301030101030103030102020303BE
:10F0300001020203010301010301030301020203B0
:10F0400003010202030103010103010303010202A0
:10F05000030301020203010301010301030301028F
:10F06000020303010202030103010103010303017F
:10F07000020203030102020301030101030103036E
:10F080000102020303010202030103010103010360
:10F090000301020203030102020301030101030150
:10F0A000030301020203030102020301030101033E
:10F0B0000103030102020303010202030103010130
:10F0C000030103030102020303010202030103011E
:10F0D0000103010303010101030301010103010312
:10F0E0000101030103030101010303010101030104
:10F0F00003010103010303010101030301010103F2
:10F1000001030101030103030101010303010101E3
:10F1100003010301010301030301010103030101D1
:10F1200001030103010103010303010101030301C1
:10F1300001010301030101030103030101010303B1
:10F1400001010103010301010301030301010103A3
:10F150000301010103010301010301030301010193
:10F160000303010101030103010103010303010181
:10F170000103030101010301030101030103030171
:10F180000101030301010103010101010101030365
:10F190000101010303010101030101010101010357
:10F1A0000301010103030101010301010101010147
:10F1B0000303010101030301010103010101010135
:10F1C0000103030101010303010101030101010125
:10F1D0000101030301010103030101010301010115
:10F1E0000101010303010101030301010103010105
:10F1F00001010101030301010103030101010301F5
:10F2000001010101010303010101030301010103E4
:10F2100001010101010103030101010303010101D6
:10F2200003010101010101030301010103030101C4
:10F2300001030301030301030303010101030301AC
:10F24000010103030103030103030301010103039C
:10F25000010101030301030301030303010101038E
:10F26000030101010303010303010303030101017E
:10F27000030301010103030103030103030301016C
:10F28000010303010101030301030301030303015C
:10F29000010103030101010303010303010303034C
:10F2A000010101030301010103030103030103033E
:10F2B000030101010303010101030301030301032E
:10F2C000030301010103030101010303010303011E
:10F2D000030303010101030301010103030303030A
:10F2E00003030303010101030301010103030303FA
:10F2F00003030303030101010303010101030303EA
:10F3000003030303030301010103030101010303D9
:10F3100003030303030303010101030301010103C9
:10F3200003030303030303030101010303010101B9
:10F3300003030303030303030301010103030101A7
:10F340000103030303030303030301010103030197
:10F350000101030303030303030303010101030387
:10F360000101010303030303030303030101010379
:10F370000301010103030303030303030301010169
:10F380000303010101030303030303030303010157
:10F390000103030101010303030303030303030147
:10F3A0000101030301010103030303030303030337
:10F3B0000101010303010101030303030303030329
:10F3C0000301010103030101010303030303030319
:10F3D0000303010101030301010103030303030309
:10F3E00003030301010103030101010303030303F9
:10F3F00003030303010101030301010103030303E9
:10F4000003030303030101010303010101030303D8
:10F4100003030303030301010103030101010303C8
:10F4200003030303030303010101030301010103B8
:10F4300003030303030303030101010303010101A8
:10F440000303030303030303030101010303010196
:10F450000103030303030303030301010103030186
:10F460000101030303030303030303010101030376
:10F470000101010303030303030303030101010368
:10F480000301010103030303030303030301010158
:10F490000303010101030303030303030303010146
:10F4A0000103030101010303030303030303030136
:10F4B0000101030301010103030303030303030326
:10F4C0000101010303010101030303030303030318
:10F4D0000000F894EE27ECBBF1E0F5BFE5BFE09348
:10F4E0006C00EBBFF8E1F1BDF0E1F1BD8DE0A2E011
:10F4F000BB27ED938A95E9F780E090E1A0E0B1E0C9
:10F50000ED930197E9F7E0EDF4EF05901590BF0159
:10F51000F001309751F0A591B591859195910590A5
:10F520000D920197E1F7FB01F0CFEFEFEDBFE0E1C6
:10F53000EEBFC0E0D5E00C949D7A2BD1E7E0EA93D2
:10F54000C7D1EFE0EA93D4D102D0FECFFFCFE3D111
:10F55000CC24CC2041F4E5D1EAE0F0E0FA93EA9340
:10F560000E941A7DF6CFDDD1D6D1E2E1F0E0FA9328
:10F57000EA9302D1D6D1DAD1A3D0D3D1D7D1E1D178
:10F58000E0D1DED0CED1D2D1E2D1E1D1E0D1E4D010
:10F59000C8D1CCD1E9D0E4E1F0E0FA93EA93E4D029
:10F5A000C0D1C4D1A7D0BDD1E4EFF1E0FA93EA9382
:10F5B0000E941A7DE8EEF3E0FA93EA930E941A7D26
:10F5C000D2CF08950A9300E0E981E295E07FEE0F43
:10F5D000AB81EA2B0E2FA33009F4BFD1AB81A83049
:10F5E00009F4BBD1AB81A43019F4EA81EA50EA8373
:10F5F000AB81A83009F4B5D1AB81A93009F4B1D100
:10F60000EFEFEA935CD10A935AD1EA81EA9357D19A
:10F61000EA81E027EF77EA9352D181E38A95F1F707
:10F62000EE27FF270881249608950E944A7D00E076
:10F6300010E06E807F80442455244614570410F057
:10F6400094D11AC000E010E00131E0E01E078CF414
:10F6500092D1AB85BC85EA0FFB1FE49198D1AA85B6
:10F66000BB85EA0FFB1FE491EA93ACDF0F5F1F4FEE
:10F67000EBCF7BD196D1E1CF0E944F7D2C960895A0
:10F68000E881E03039F493D1ADBC9CBC44245524CE
:10F69000BB2415C0E13061F48FD1EE27FF27FDBDFB
:10F6A000ECBD44245524E1E0BE2EEE27E7BF07C0A1
:10F6B000E23011F481D103C0E33009F478D106C1FE
:10F6C000E1E08E2EECEFF8E1FA93EA93E4EAFBE155
:10F6D00077D181D180D17FD17ED17DD17CD17BD1B9
:10F6E0007AD1E4E4F6E2FA93EA93E0E4FAE284D130
:10F6F00088244DC0E1E08E2EE4E2F8E4FA93EA9328
:10F70000ECECFAE45DD183D182D181D180D17FD17B
:10F710007ED17DD17CD1ECE6F5E5FA93EA93E8E67B
:10F72000F9E56AD1882433C0ECE8F0E0FA93EA9373
:10F73000E4E1F1E0FA93EA93E8E0F0E06FD127C06A
:10F74000ECE3FEE2FA93EA93E6E3F5E3FA93EA9355
:10F75000E9E6F0E063D11BC0E4EEF7E8FA93EA9340
:10F76000EEEDFDE862D113C0E0E3FCE3FA93EA9327
:10F77000EAE2F2E45AD10BC0ECE9F1E0FA93EA9341
:10F78000ECE4FDE0FA93EA93E0EBF0E047D1229657
:10F790000895EE27EBBBEABBE8BBE7BBE5BBE4BBE8
:10F7A000E3E0E2BBEE27E1BBE3B9E2B9E09362003C
:10F7B000E0936100E0936500EFEFE0936400EE27D3
:10F7C000E0BFE3BFE2BFE1BFEFBDEEBDEDBDECBD0D
:10F7D000EBBDEABDE9BDE8BDE0937900E0937800B8
:10F7E000E5BDE4BDE3BDE0938B00E0938A00E093C8
:10F7F0008900E0938800E0938700E0938600E0931F
:10F800008500E0938400E0938300E0938200EAE0C7
:10F81000E0936A00EE27EABFE3E0E9BFE8BFEE2726
:10F82000E7BFE0937D00E0E8E8B9EE27E0BD78941B
:10F8300008950E94267DEE27EA9322DFE1E0CE2E96
:10F84000E0916500AFEFEA27E09365000E94347D08
:10F8500018950E94267D0E94347D18950E94267D71
:10F860000E944A7D00E010E04614570420F0E1E0D9
:10F87000EA9306DF1EC000E010E00131E0E01E0761
:10F88000ACF479D0A0910005B0910105EA0FFB1FFF
:10F89000E4917DD0A0910205B0910305EA0FFB1F12
:10F8A000E491EA938FDE0F5F1F4FE7CF7AD0ADBCB4
:10F8B0009CBC0E944F7D24960E94347D1895E09157
:10F8C0009B00E072E1F3E881E0939C0021960895AB
:10F8D000F894EE27EBB9E8E1EAB9E6E0E0939500A9
:10F8E000EE27E0939000E881E9B978942196089595
:10F8F000F894EE27E0939B00E8E1E0939A00E6E0BD
:10F90000E0939D00EE27E0939800E881E093990052
:10F91000789421960895E0EDF7E0FA93EA930C9439
:10F920001A7DECE3F0E0FA93EA93FECEE4EFF1E027
:10F93000FA93EA930E941A7DE4E1F0E0FA93EA93E5
:10F940000895FEDEE4E1F0E0FA93EA93089504DF1F
:10F95000E4E1F0E0FA93EA930895EA81EB5FEA8349
:10F960000895EA81E550EA830895EC81FD81FA93D8
:10F97000EA930C941A7DE02FF12FEA93A42DB52D74
:10F98000E1E1F0E00E94427DE00FF11F0895EA936B
:10F99000A42DB52DE1E1F0E00E94427DE00FF11FC2
:10F9A0000895E42DF52D31964E2E5F2E0895E4E056
:10F9B000E7BFE5E0EEBD0895EE27E7BFEEBD089591
:10F9C000FA93EA93E8E2F0E0FA93EA93EE81FF819A
:10F9D000FA93EA932ACEECE4FEE1FA93EA93E8E4A0
:10F9E000F2E2FA93EA93ECE3F0E0FA93EA93EE8121
:10F9F000FF81FA93EA9319CEFA93EA93ECE3F0E0ED
:10FA0000FA93EA93EE81FF81FA93EA930ECEE4E74C
:10FA1000FDE4FA93EA93E0E7F1E5EECFFA93EA9397
:10FA2000EE81FF81FA93EA9300CEFA93EA93EAE536
:10FA3000F0E0F4CFE991F991309639F086E69EE056
:10FA40000197F1F7A8953197C9F708950A921A928C
:10FA5000FA926A937A938A939A93AA93BA93EA93BF
:10FA6000FA930FB60A92089509900FBEF991E991A1
:10FA7000B991A9919991899179916991F990199088
:10FA800009900895FA9FF02DEB9FF00DEA9FE02D6D
:10FA9000F10D08953A932A931A930A9308953B819E
:10FAA0002A81198108810895FFFFFFFFFFFFFFFFF3
:10FAB000FFFFFFFFFFFFFFFFFFFFFFFFFFFFFFFF56
:10FAC000FFFFFFFFFFFFFFFFFFFFFFFFFFFFFFFF46
:10FAD000FFFFFFFFFFFFFFFFFFFFFFFFFFFFFFFF36
:10FAE000FFFFFFFFFFFFFFFFFFFFFFFFFFFFFFFF26
:020000021000EC
:00000001FF
